:100000000C94004C0C94214C0C9439D40C94214C3D
:100010000C94214C0C94214C0C94214C0C94214CAC
:100020000C94214C0C94214C0C94214C0C9464D6CF
:100030000C94214C0C94214C0C94D9B60C94214C6A
:100040000C94214C0C94214C0C94214C0C94214C7C
:100050000C94214C0C94214C0C94214C0C94214C6C
:100060000C94214C0C9453D40C94E2D30C94214C5A
:100070000C94ACCD0C944ECD0C948ACD0C94214CA8
:100080000C9404D50C94214C0C94214C0C94214CD0
:100090000C94214C0C94214C0C94214C0C94214C2C
:1000A0000C94214C0C94214C0C94214C0C9458BE73
:1000B0000C94FCBE0C94214C0C94214C0C94CAB8AA
:1000C0000C94214C0C94214C0C94214C0C94214CFC
:1000D0000C94214C0C94214C0C94214C0C94214CEC
:1000E0000C9450A90C94214C0C94214C0C94214C50
:1000F0000C94214C0C94214C0C94214C0C94214CCC
:100100000C942FBE0C94D3BE0C9406BE0C94AABEC5
:100110000C94214C0C94214C0C94214C0C94214CAB
:100120000C94214C0C94214C0C94214C0C94214C9B
:100130000C94214C0C942EB80C94214C0C94214C12
:100140000C94214C0C94214C0C94214C0C94214C7B
:100150000C94214C0C94214C0C9446A90C94214CE9
:100160000C94214C0C94214C0C94214C0C94214C5B
:100170000C94214C0C94214C0C94214C0C94214C4B
:100180000C94214C0C94214C0C94214C0C94214C3B
:100190000C94214C0C94214C0C94214C0C94214C2B
:1001A0000C9481BE0C9425BF0C94214C0C94214CD2
:1001B0000C947CB80C94214C0C94214C0C94214C44
:1001C0000C94214C0C94214C0C94214C0C94214CFB
:1001D0000C94214C0C94214C0C94214C0C94214CEB
:1001E0000C94214C0C94214C65756F757975837551
:1001F0008E752C7B2C7B2C7B2C7B2C7B94752C7B09
:100200002C7B2C7B2C7B2C7B2C7B9675A075AA756C
:10021000B475BE752C7B2C7B2C7B2C7B2C7B2C7B98
:10022000C8752C7B1E762C7B2C7B2C7B2C7B2C7B13
:100230002C7B2C7B5D762C7B13792C7B2C7B2C7B75
:100240002C7B2C7B2C7B2C7B2C7B13792C7B2C7B91
:100250002C7B8A768F769976A376A576AF76BA765A
:100260002C7BC5762C7B2C7B02772C7B2C7B2C7BF0
:100270002C7B2C7B2C7B2C7B2C7B2C7B2C7B2C7B46
:100280002C7B2C7B2C7B2C7B0C772C7B2C7B2C7B5A
:100290002C7B2C7B2C7B2C7B2C7B2C7B1677207750
:1002A0002A7773777D7796779677A077AA77B47752
:1002B000BE77C877CD77D777E1772A7B2A7B2A7BF1
:1002C0002A7B2A7B2A7B2A7B2A7B2A7B2A7B2A7B06
:1002D0002A7B2A7B2A7B2A7B2A7B2A7B2A7B2A7BF6
:1002E0002A7BA0772A7B2A7B2A7B2A7B2A7B2A7B74
:1002F0002A7B2A7B2A7B2A7B2A7B2A7B2A7B2A7BD6
:100300002A7B2A7B2A7BEB77F577FF7709782A7B94
:100310002A7B2A7B2A7B2A7B2A7B2A7B2A7B96774D
:10032000B77A787A7C7A847A607A647A6C7A707A2E
:10033000907AA37AAB7AAF7AB37A0F7B887A847893
:100340009578A6782C7B2C7B1E7856752C7BB778FD
:10035000C878D97813798777FB782C7B2F782C7B1A
:10036000EA78407813782C7B2C7B2C7B5178627850
:1003700073789FBDA7BDAFBDB7BDBFBDC7BDCFBD66
:10038000D7BDCAC027C02FC037C03FC047C04FC06D
:1003900057C05FC067C06FC077C07FC087C08FC0C5
:1003A000AFC0AFC0AFC0AFC0AFC0AFC0AFC0AFC0D5
:1003B000AFC0AFC0AFC0AFC0AFC0AFC0AFC0AFC0C5
:1003C000AFC0AFC0AFC0AFC0AFC0AFC0AFC0AFC0B5
:1003D000AFC0AFC0AFC0AFC0AFC0AFC0AFC0AFC0A5
:1003E000AFC0AFC0AFC097C09FC0AFC0AFC0AFC0BD
:1003F000AFC0AFC0AFC0AFC0AFC0AFC0AFC0AFC085
:10040000AFC0AFC0AFC0AFC0AFC0AFC0AFC0AFC074
:10041000AFC0AFC0AFC0AFC0AFC0AFC0AFC0AFC064
:10042000AFC0AFC0AFC0AFC0AFC0AFC0AFC0AFC054
:10043000AFC0AFC0AFC0AFC0AFC0AFC0AFC0AFC044
:10044000AFC0AFC0AFC0AFC0A7C0084AD73B3BCE1C
:10045000016E84BCBFFDC12F3D6C74319ABD5683C3
:100460003DDA3D00C77F11BED9E4BB4C3E916BAA7B
:10047000AABE000000803F05A84CCDB2D44EB938CA
:1004800036A9020C50B9918688083CA6AAAA2ABEB1
:10049000000000803F07634236B79BD8A71A39682F
:1004A0005618AEBAAB558C1D3CB7CC5763BD6DED3D
:1004B000FD753EF6177231BF000000803F08000056
:1004C00000BE922449123EABAAAA2ABECDCCCC4C87
:1004D0003E00000080BEABAAAAAA3E00000000BFFA
:1004E000000000803F0000000000084178D3BB43BB
:1004F00087D1133D190E3CC3BD4282AD2B3E68EC43
:100500008276BED98FE1A93E4C80EFFFBE01C4FFC9
:100510007F3F0000000000000C9444B00C94887AE7
:100520000C94525B0C9415C00C946C7A0C94645B24
:100530000C9420680C94A1C40C94A9AA0C949FBD9F
:100540000C94647A0C94125F0C945BBD0C9495AA85
:100550000C940C600C94E26B0C94EA5E0C946A5B55
:100560000C943FC00C9469CC0C94EE5E0C945171C9
:100570000C9462780C94D85F0C94A26C0C94666214
:100580000C94374C0C946FC00C94BDBC0C94F7BF0A
:100590000C94AFBD0C942D4C0C946CAB0C947B5B09
:1005A0000C940E5E0C941E5F0C94025C0C94234C15
:1005B0000C94FB780C94F5770C948FC00C94BA6172
:1005C0000C94B5AA0C944FC00C94F5820C943F8502
:1005D0000C9440B00C94DE610C941E760C94DB6796
:1005E0000C94365E0C94025F0C94CD770C94FCCB8B
:1005F0000C94286D0C9460680C940E5F0C94A767A3
:100600000C94F85F0C94585B0C9499870C949A5B4B
:100610000C942C7B0C9499760C941CB00C9455D0B3
:100620000C9440780C94756F0C9472BD0C9438B097
:100630000C9458D10C945FC00C94F45F0C944D5FF3
:100640000C94BB5B0C94944F0C946DCA0C940A5F91
:100650000C947EC50C949B5C0C94C7BD0C9496774F
:100660000C94285E0C94455B0C941A5F0C94F05F1C
:100670000C949ABB0C946F750C94175D0C94865B6C
:100680000C9409780C9425630C949C580C945E5B34
:100690000C940F7B0C94225F0C94EA780C94A37654
:1006A0000C94AF7A0C9487C00C94AF760C94AA7516
:1006B0000C9472670C94A7C00C94BFBD0C94E45FBB
:1006C0000C9476BD0C9456750C94D9780C946ABD34
:1006D0000C94AC950C947D6F0C94E07C0C94D45BE2
:1006E0000C946C5F0C94A55B0C94FF720C941677C1
:1006F0000C942E5F0C9464830C94764C0C943CB058
:100700000C94E25E0C94B77C0C94715C0C94A1AADE
:100710000C9427C00C94D7770C94AA770C946FB1E3
:100720000C94A7BD0C9400B00C94D3D10C94877793
:100730000C94BE770C94576C0C94AFC00C94517809
:100740000C94FF770C948F760C948A760C9492BC60
:100750000C949CAE0C94BA760C946A670C9452BDBF
:100760000C94045D0C94CAC00C946EBD0C9488C4A7
:100770000C94B9AA0C94B76C0C9411C00C9498AE5C
:100780000C94635E0C9476670C9467C00C94F65ED0
:100790000C94907A0C949DAA0C943D5E0C94C878AD
:1007A0000C9477C00C9402770C94C7660C944EBDE1
:1007B0000C94B1AA0C94FC5F0C94917D0C946E6720
:1007C0000C94D45F0C94445E0C945D760C94847805
:1007D0000C94EA640C94AB7A0C94874C0C947FC014
:1007E0000C947C7A0C94AB660C94F7BC0C949661D8
:1007F0000C941E780C94B2CA0C94847A0C94A5764E
:100800000C94C5760C943C610C94E87C0C94CFBDA0
:100810000C94787A0C9465750C944F720C943E622B
:100820000C9468830C945CAE0C9414600C94BE75AC
:100830000C94FE620C94DD5D0C94EFCE0C94667DFE
:100840000C945E630C9421D10C94C1D00C9455BBD4
:100850000C9410600C9440620C94FE5E0C94B7787B
:100860000C94286C0C94B77A0C9413780C94BDC437
:100870000C9437C00C9498B10C942FC00C94A37AAC
:100880000C94B4770C9495780C949FC00C942A77B0
:100890000C9494750C94DC7C0C9489C40C94E9CC75
:1008A0000C94825E0C9405620C94D5620C946E7B61
:1008B0000C9497C00C94C8770C94DFBB0C9473789D
:1008C0000C94647C0C94A6BC0C948B620C943A5CE3
:1008D0000C94DE5E0C9492610C94D7BD0C94156759
:1008E0000C94EB770C94E65E0C945EAE0C94206056
:1008F0000C9483750C945F6B0C94F25E0C9460AE58
:100900000C942B600C94707A0C94B7BD0C94C16756
:100910000C94FBCC0C94065F0C941FBD0C94666782
:100920000C94B0620C94265F0C948F5B0C9413793A
:100930000C94B05B0C94BD720C9447C00C949675EB
:100940000C94A0770C948E750C9400600C94855DCB
:100950000C942A7B0C94BC7C0C9482D30C94EC7C7D
:100960000C94705B0C947D770C9420770C94C1CF21
:100970000C94BC7D0C94E1770C9437D20C94165FE8
:100980000C9499AA0C94A6780C946C830C94ADAA40
:100990000C9456BD0C9457C00C9479750C94A068B7
:1009A0000C94DAC40C9403530C9434720C940C77AA
:1009B0000C9408600C94E05F0C948F5F0C94FA5ECA
:1009C0000C94095E0C942A5F0C94E85F0C942F78C9
:1009D0000C9404600C94B37A0C94705F0C94C875FA
:1009E0000C94B4750C94F5670C94EB5B0C94A5AA6D
:1009F0000C94EBAF0C94756C0C94A0750C94EC5F9C
:100A00000C94DC5F0C94E47C0C9496AE0C94D45C57
:100A10000C947E7B0C94277D0C9473770C942F5E42
:100A20000C94607A0C948ACC0C94F1BF5B257325EE
:100A3000735D20257320257320706F736974696F4F
:100A40006E2531382E336625730A005B25732573B6
:100A50005D202573202573206F66667365742532CB
:100A6000302E336625730A005B257325735D2025C0
:100A700073207A65726F206261636B6F66662531E1
:100A8000392E336625730A005B257325735D202597
:100A900073206C61746368206261636B6F666625A6
:100AA00031382E336625730A005B257325735D206C
:100AB0002573206C617463682076656C6F6369745C
:100AC000792531332E306625732F6D696E0A005BF0
:100AD000257325735D20257320736561726368201B
:100AE00076656C6F636974792531322E30662573B3
:100AF0002F6D696E0A005B257325735D20257320B9
:100B0000737769746368206D617825313764205B81
:100B1000303D6F66662C313D686F6D696E672C32B3
:100B20003D6C696D69742C333D6C696D69742B681B
:100B30006F6D696E675D0A005B257325735D202507
:100B40007320737769746368206D696E253137642B
:100B5000205B303D6F66662C313D686F6D696E6756
:100B60002C323D6C696D69742C333D6C696D697410
:100B70002B686F6D696E675D0A005B257325735D79
:100B8000202573207261646975732076616C7565C8
:100B90002532302E346625730A005B257325735D7C
:100BA000202573206A756E6374696F6E20646576A4
:100BB000696174696F6E2531342E3466257320287F
:100BC0006C61726765722069732066617374657207
:100BD000290A005B257325735D202573206A6572E1
:100BE0006B20686F6D696E672531362E3066257310
:100BF0002F6D696E5E33202A2031206D696C6C691F
:100C00006F6E0A005B257325735D202573206A656E
:100C1000726B206D6178696D756D2531352E30668A
:100C200025732F6D696E5E33202A2031206D696C2B
:100C30006C696F6E0A005B257325735D2025732038
:100C400074726176656C206D696E696D756D2531A4
:100C5000372E336625730A005B257325735D2025C7
:100C6000732074726176656C206D6178696D756D45
:100C70002531372E336625730A005B257325735D96
:100C80002025732076656C6F63697479206D6178B7
:100C9000696D756D2531312E306625732F6D696E46
:100CA0000A005B257325735D2025732066656564E6
:100CB00072617465206D6178696D756D2531312EB5
:100CC000306625732F6D696E0A005B257325735D91
:100CD0002025732061786973206D6F646525313834
:100CE000642025730A005B6D615D20206D696E20B4
:100CF000617263207365676D656E742531382E33BC
:100D00006625730A005B736C5D2020736F66742028
:100D10006C696D697420656E61626C652531326441
:100D20000A005B63745D202063686F7264616C20ED
:100D3000746F6C6572616E63652531372E3466257C
:100D4000730A005B6A615D20206A756E6374696F67
:100D50006E20616363656C65726174696F6E2538BE
:100D60002E306625730A005B6764695D20646566E2
:100D700061756C742067636F646520646973746166
:100D80006E6365206D6F6465253264205B303D477E
:100D900039302C313D4739315D0A005B6770615D48
:100DA0002064656661756C742067636F646520708C
:100DB00061746820636F6E74726F6C253364205B9E
:100DC000303D4736312C313D4736312E312C323DC6
:100DD0004736345D0A005B67636F5D20646566615A
:100DE000756C742067636F646520636F6F72642035
:100DF00073797374656D253364205B312D3620283B
:100E00004735342D473539295D0A005B67756E5DBE
:100E10002064656661756C742067636F6465207516
:100E20006E697473206D6F6465253564205B303D99
:100E30004732302C313D4732315D0A005B67706CC0
:100E40005D2064656661756C742067636F646520FE
:100E5000706C616E6525313064205B303D47313701
:100E60002C313D4731382C323D4731395D0A002560
:100E70006320776F726B206F66667365743A2531F5
:100E8000322E336625730A002563206D616368691D
:100E90006E6520706F736E3A2531312E336625737F
:100EA0000A00256320706F736974696F6E3A25318B
:100EB000352E336625730A00546F6F6C206E756D86
:100EC0006265722020202020202020202025640A16
:100ED00000466565642072617465206D6F64653AD3
:100EE00020202020202025730A0044697374616E3D
:100EF0006365206D6F64653A202020202020202526
:100F0000730A0050617468204D6F64653A20202098
:100F1000202020202020202025730A00506C616EA4
:100F2000653A202020202020202020202020202062
:100F30002025730A004D6F74696F6E206D6F6465B4
:100F40003A20202020202020202025730A00436FF3
:100F50006F7264696E6174652073797374656D3A3C
:100F600020202025730A00556E6974733A202020D2
:100F700020202020202020202020202025730A004F
:100F8000486F6D696E672073746174653A20202024
:100F9000202020202025730A0046656564686F6C58
:100FA000642073746174653A20202020202025730A
:100FB0000A004D6F74696F6E2073746174653A2016
:100FC0002020202020202025730A004379636C65AF
:100FD0002073746174653A20202020202020202076
:100FE00025730A00526177206D616368696E652020
:100FF00073746174653A20202025730A004D616383
:1010000068696E652073746174653A202020202021
:10101000202025730A004C696E65206E756D62652F
:10102000723A2531302E30660A00466565642072BA
:101030006174653A2531362E336625732F6D696EDE
:101040000A0056656C6F636974793A2531372E331F
:101050006625732F6D696E0A00B0107F105F104710
:101060003935202D20756E6974732D7065722D725F
:1010700065766F6C7574696F6E206D6F646500477F
:101080003934202D20756E6974732D7065722D6D45
:10109000696E757465206D6F64652028692E652EF4
:1010A000206665656472617465206D6F64652900F2
:1010B000473933202D20696E766572736520746917
:1010C0006D65206D6F646500EC10CC1047393120E0
:1010D0002D20696E6372656D656E74616C20646944
:1010E0007374616E6365206D6F64650047393020ED
:1010F0002D206162736F6C7574652064697374610F
:101100006E6365206D6F6465003D1125110F1147F9
:101110003634202D20636F6E74696E756F75732081
:101120006D6F6465004736312E31202D2065786162
:1011300063742073746F70206D6F6465004736317F
:10114000202D2065786163742070617468206D6F54
:10115000646500771168115911473139202D2059E4
:101160005A20706C616E6500473138202D20585A26
:1011700020706C616E6500473137202D2058592052
:10118000706C616E65000312F111D811B7119011E6
:10119000473830202D2063616E63656C206D6F745D
:1011A000696F6E206D6F646520286E6F6E652061BB
:1011B00063746976652900473320202D20636F759D
:1011C0006E74657220636C6F636B77697365206101
:1011D0007263206665656400473220202D20636CB1
:1011E0006F636B7769736520617263206665656400
:1011F00000473120202D206C696E65617220666584
:10120000656400473020202D206C696E6561722076
:10121000747261766572736520287365656B290049
:10122000CA12B01296127C12621248122E12473560
:1012300039202D20636F6F7264696E61746520734D
:10124000797374656D203600473538202D20636F23
:101250006F7264696E6174652073797374656D2053
:101260003500473537202D20636F6F7264696E61DA
:1012700074652073797374656D20340047353620AA
:101280002D20636F6F7264696E617465207379736A
:1012900074656D203300473535202D20636F6F72E4
:1012A00064696E6174652073797374656D203200B2
:1012B000473534202D20636F6F7264696E617465E9
:1012C0002073797374656D203100473533202D20EC
:1012D0006D616368696E6520636F6F7264696E61CA
:1012E00074652073797374656D00FD12F712F01246
:1012F000486F6D696E6700486F6D6564004E6F746E
:1013000020486F6D65640031132C13271321131CC3
:10131000131313456E6420486F6C6400486F6C644F
:1013200000446563656C00506C616E0053796E63B8
:10133000004F666600441340133B13486F6C640013
:1013400052756E0053746F70006E1364135E135702
:101350001353134A6F6700486F6D696E67005072D0
:101360006F6265004D616368696E696E67004F6604
:101370006600A4139E13981393138F13891380137D
:1013800053687574646F776E004379636C650045CC
:101390006E640053746F7000416C61726D00526531
:1013A00061647900496E697469616C697A696E6714
:1013B0000007140114FB13F613F213EE13E913E301
:1013C00013DD13D613D213C91353687574646F7782
:1013D0006E004A6F6700486F6D696E6700437963FE
:1013E0006C650050726F626500486F6C64005275E6
:1013F0006E00456E640053746F7000416C61726DD5
:1014000000526561647900496E697469616C697A3A
:10141000696E67002E141814473231202D206D6933
:101420006C6C696D65746572206D6F646500473220
:1014300030202D20696E63686573206D6F646500D0
:1014400068145D14511448145B7261646975735DAE
:10145000005B696E686962697465645D005B7374E2
:10146000616E646172645D005B64697361626C6586
:10147000645D0082147E1479142064656700206D19
:101480006D0020696E002A2A2A204E4F5449434598
:10149000202A2A2A20526573657474696E67206257
:1014A000617564207261746520746F202573005B20
:1014B000626175645D2055534220626175642072DB
:1014C00061746525313564205B313D393630302C0F
:1014D000323D31393230302C333D33383430302CDA
:1014E000343D35373630302C353D313135323030C2
:1014F0002C363D3233303430305D0A005B72786D0B
:101500005D2073657269616C205258206D6F64654F
:1015100025313564205B303D73747265616D696E91
:10152000675F6D6F64652C313D7061636B65745FDF
:101530006D6F64655D0A005B65785D2020656E6196
:10154000626C6520666C6F7720636F6E74726F6C6F
:1015500025313064205B303D6F66662C313D584F3D
:101560004E2F584F46462C323D5254532F4354531E
:101570005D0A005B65655D2020656E61626C6520BB
:101580006563686F25313864205B303D6F66662C7B
:10159000313D6F6E5D0A005B65635D20206578708C
:1015A000616E64204C4620746F2043524C46206F7D
:1015B0006E205458253664205B303D6F66662C31B2
:1015C0003D6F6E5D0A00F915F415EE15E815E2158C
:1015D000DB15D41532333034303000313135323010
:1015E0003000353736303000333834303000313960
:1015F0003230300039363030003000737973006695
:1016000062000000000702DC7C05623E62903AF650
:1016100088DC43737973006676000000000703E0FE
:101620007C05623E62943AEC51783F7379730068AE
:1016300070000000000700E47C056225639C3A000E
:1016400000803F737973006876000000000700E8AF
:101650007C0562BC7CA03A0000004173797300698C
:1016600064000000000400EC7C647C3E628C3A0064
:10167000000000000000006E00000000000100DE1D
:101680005ED45BD562833200000000000000006C75
:10169000696E6500000100DE5EEB5BD5628332009F
:1016A0000000000000000076656C000000000244AD
:1016B0005E025C3E628C3A000000000000000066A2
:1016C00065656400000002635E3A5C3E628C3A002D
:1016D000000000000000007374617400000000E26C
:1016E0005E455B3E628C3A00000000000000006D29
:1016F00061637300000000E65E525B3E628C3A005C
:10170000000000000000006379637300000000EA3D
:101710005E585B3E628C3A00000000000000006DE5
:101720006F747300000000EE5E5E5B3E628C3A00F8
:1017300000000000000000686F6C6400000000F210
:101740005E645B3E628C3A000000000000000075A1
:101750006E697400000000FA5E705B3E628C3A00B5
:1017600000000000000000636F6F7200000000FEC8
:101770005E7B5B3E628C3A00000000000000006D62
:101780006F6D6F00000000025F865B3E628C3A0066
:1017900000000000000000706C616E000000000698
:1017A0005F8F5B3E628C3A0000000000000000701A
:1017B000617468000000000A5F9A5B3E628C3A0028
:1017C0000000000000000064697374000000000E57
:1017D0005FA55B3E628C3A000000000000000066DE
:1017E000726D6F00000000125FB05B3E628C3A00C9
:1017F00000000000000000746F6F6C000000001615
:101800005FBB5B3E628C3A000000006D706F006D44
:10181000706F780000000320609B5C3E628C3A0091
:101820000000006D706F006D706F79000000032084
:10183000609B5C3E628C3A000000006D706F006D32
:10184000706F7A0000000320609B5C3E628C3A005F
:101850000000006D706F006D706F6100000003206C
:10186000609B5C3E628C3A000000006D706F006D02
:10187000706F620000000320609B5C3E628C3A0047
:101880000000006D706F006D706F6300000003203A
:10189000609B5C3E628C3A00000000706F730070C9
:1018A0006F7378000000031460715C3E628C3A0034
:1018B000000000706F7300706F73790000000314F4
:1018C00060715C3E628C3A00000000706F730070C3
:1018D0006F737A000000031460715C3E628C3A0002
:1018E000000000706F7300706F73610000000314DC
:1018F00060715C3E628C3A00000000706F73007093
:101900006F7362000000031460715C3E628C3A00E9
:10191000000000706F7300706F73630000000314A9
:1019200060715C3E628C3A000000006F6673006F6D
:10193000667378000000032B60D45C3E628C3A0032
:101940000000006F6673006F667379000000032B60
:1019500060D45C3E628C3A000000006F6673006FDA
:1019600066737A000000032B60D45C3E628C3A0000
:101970000000006F6673006F667361000000032B48
:1019800060D45C3E628C3A000000006F6673006FAA
:10199000667362000000032B60D45C3E628C3A00E8
:1019A0000000006F6673006F667363000000032B16
:1019B00060D45C3E628C3A00000000686F6D006885
:1019C0006F6D6500000000F65E6A5B0E5E8C3A008B
:1019D000000000686F6D00686F6D780000000014F3
:1019E0006096613E62583200000000686F6D0068CA
:1019F0006F6D7900000000146096613E62593200FC
:101A0000000000686F6D00686F6D7A0000000014C0
:101A10006096613E625A3200000000686F6D006897
:101A20006F6D6100000000146096613E625B3200E1
:101A3000000000686F6D00686F6D620000000014A8
:101A40006096613E625C3200000000686F6D006865
:101A50006F6D6300000000146096613E625D3200AD
:101A60000000007072620070726265000000008801
:101A7000C496613E625E32000000007072620070C7
:101A80007262780000000388C405623E625F320023
:101A900000000070726200707262790000000388BA
:101AA000C405623E62633200000000707262007022
:101AB00072627A0000000388C405623E62673200E9
:101AC00000000070726200707262610000000388A2
:101AD000C405623E626B32000000007072620070EA
:101AE0007262620000000388C405623E626F3200C9
:101AF0000000007072620070726263000000038870
:101B0000C405623E627332000000006A6F67006ABB
:101B10006F67780000000088C49261285E7D320003
:101B20000000006A6F67006A6F6779000000008834
:101B3000C492612F5E7D32000000006A6F67006A08
:101B40006F677A0000000088C49261365E7D3200C3
:101B50000000006A6F67006A6F676100000000881C
:101B6000C492613D5E7D32000000007077720070AB
:101B70007772310000000076BDA6BC3E628C3A0050
:101B800000000070777200707772320000000076FB
:101B9000BDA6BC3E628C3A000000007077720070F7
:101BA0007772330000000076BDA6BC3E628C3A001E
:101BB00000000070777200707772340000000076C9
:101BC000BDA6BC3E628C3A0000000031000000312E
:101BD0006D61000000030052BD96614062B958007B
:101BE0000000003100000031736100000003035663
:101BF000BD056255BBC4586666E63F310000003142
:101C000074720000000B045BBD05629ABBC8585C8F
:101C10008FA24031000000316D6900000003006AAE
:101C2000BD9661DFBBBA58000000413100000031B1
:101C3000706F00000003006EBD96616662BE5800C2
:101C40000000003100000031706D000000030072E0
:101C5000BD966192BCBF58000000403200000032C7
:101C60006D61000000030052BD96614062D85800CB
:101C700000803F3200000032736100000003035611
:101C8000BD056255BBE3586666E63F320000003290
:101C900074720000000B045BBD05629ABBE7585CE0
:101CA0008FA24032000000326D6900000003006A1C
:101CB000BD9661DFBBD95800000041320000003200
:101CC000706F00000003006EBD96616662DD580013
:101CD00000803F3200000032706D0000000300728F
:101CE000BD966192BCDE5800000040330000003316
:101CF0006D61000000030052BD96614062F758001C
:101D000000004033000000337361000000030356FD
:101D1000BD056255BB02596666E63F3300000033DD
:101D200074720000000B045BBD05629ABB06597714
:101D300077074033000000336D6900000003006A3C
:101D4000BD9661DFBBF8580000004133000000334E
:101D5000706F00000003006EBD96616662FC580063
:101D60000000003300000033706D000000030072BB
:101D7000BD966192BCFD5800000040340000003464
:101D80006D61000000030052BD966140621659006B
:101D9000004040340000003473610000000303562B
:101DA000BD056255BB21596666E63F34000000342C
:101DB00074720000000B045BBD05629ABB255900DC
:101DC00000B44334000000346D6900000003006A71
:101DD000BD9661DFBB17590000004134000000349C
:101DE000706F00000003006EBD966166621B5900B3
:101DF0000000003400000034706D00000003007229
:101E0000BD966192BC1C590000004078000000782B
:101E1000616D00000003008F5F045D175D143100E9
:101E200000803F7800000078766D0000000B00D83D
:101E30005F0562156719310000C84478000000781A
:101E400066720000000B00D45F0562156715310053
:101E500000C8447800000078746E0000000B03E0B6
:101E60005F056215672131000000007800000078EE
:101E7000746D0000000B03DC5F056215671D310007
:101E800000964378000000786A6D0000000B00E4C3
:101E90005F0562855D25310000C84278000000784A
:101EA0006A680000000B00E85F0562DD5D29310013
:101EB00000C84278000000786A640000000B04EC5F
:101EC0005F056215673131CDCC4C3D78000000785C
:101ED000736E0000000300F45F9661F7BF383000B6
:101EE00000803F780000007873780000000300F85D
:101EF0005F9661F7BF39300000000078000000787D
:101F000073760000000B00FC5F0562156739310035
:101F1000007A4478000000786C760000000B000026
:101F200060056215673D310000C842780000007806
:101F30006C620000000B030460056215674131000C
:101F400000204178000000787A620000000B03084E
:101F50006005621567453100000040790000007996
:101F6000616D00000003008F5F045D175D49310063
:101F700000803F7900000079766D0000000B00D8EA
:101F80005F056215674E310000C844790000007992
:101F900066720000000B00D45F056215674A3100CD
:101FA00000C8447900000079746E0000000B03E063
:101FB0005F05621567563100000000790000007966
:101FC000746D0000000B03DC5F0562156752310081
:101FD00000E14379000000796A6D0000000B00E425
:101FE0005F0562855D5A310000C8427900000079C2
:101FF0006A680000000B00E85F0562DD5D5E31008D
:1020000000C84279000000796A640000000B04EC0B
:102010005F056215676631CDCC4C3D7900000079D3
:10202000736E0000000300F45F9661F7BF3A300062
:1020300000803F790000007973780000000300F809
:102040005F9661F7BF3B30000000407900000079E7
:1020500073760000000B00FC5F056215676E3100AF
:10206000007A4479000000796C760000000B0000D3
:10207000600562156772310000C84279000000797E
:102080006C620000000B0304600562156776310086
:1020900000204179000000797A620000000B0308FB
:1020A00060056215677A31000000407A0000007A0E
:1020B000616D00000003008F5F045D175D7E3100DD
:1020C00000803F7A0000007A766D0000000B00D897
:1020D0005F056215678331000096447A0000007A3C
:1020E00066720000000B00D45F056215677F310047
:1020F0000096447A0000007A746E0000000B03E042
:102100005F056215678B31000000007A0000007ADD
:10211000746D0000000B03DC5F05621567873100FA
:102120000096427A0000007A6A6D0000000B00E41D
:102130005F0562855D8F310000C8427A0000007A39
:102140006A680000000B00E85F0562DD5D93310006
:1021500000C8427A0000007A6A640000000B04ECB8
:102160005F056215679B31CDCC4C3D7A0000007A4B
:10217000736E0000000300F45F9661F7BF3C30000F
:102180000000007A0000007A73780000000300F875
:102190005F9661F7BF3D300000803F7A0000007A13
:1021A00073760000000B00FC5F05621567A3310029
:1021B0000016447A0000007A6C760000000B0000E4
:1021C0006005621567A7310000C8427A0000007AF6
:1021D0006C620000000B03046005621567AB310000
:1021E0000020417A0000007A7A620000000B0308A8
:1021F0006005621567AF31000000406100000061BA
:10220000616D00000003008F5F045D175DB3310056
:1022100000803F6100000061766D0000000300D87F
:102220005F05622563B8310000614561000000610F
:1022300066720000000300D45F05622563B43100BC
:102240000061456100000061746E0000000303E05E
:102250005F05621567C031000080BF61000000614A
:10226000746D0000000303DC5F05622563BC310070
:102270000080BF61000000616A6D0000000300E49F
:102280005F0562855DC4310000C8426100000061E5
:102290006A680000000300E85F0562DD5DC8310088
:1022A00000C84261000000616A640000000304ECA1
:1022B0005F05622563D031CDCC4C3D6100000061EB
:1022C00072610000000B03F05F05622563D43100EA
:1022D00000803F6100000061736E0000000300F4A5
:1022E0005F9661F7BF3E300000803F6100000061F3
:1022F00073780000000300F85F9661F7BF3F30007D
:10230000000040610000006173760000000300FCE3
:102310005F05622563D8310000164461000000614A
:102320006C760000000300006005622563DC31006C
:1023300000C84261000000616C62000000030304F9
:102340006005622563E0310000204161000000610A
:102350007A620000000303086005622563E431002F
:102360000000406200000062616D00000003008F09
:102370005F045D175DE8310000000062000000624C
:10238000766D0000000300D85F05622563ED310023
:10239000006145620000006266720000000300D424
:1023A0005F05622563E9310000614562000000625B
:1023B000746E0000000303E05F05621567F53100ED
:1023C0000080BF6200000062746D0000000303DC47
:1023D0005F05622563F131000080BF62000000628A
:1023E0006A6D0000000300E45F0562855DF931005D
:1023F00000C84262000000626A640000000300EC52
:102400005F056225630532CDCC4C3D620000006261
:1024100072610000000B03F05F0562256309320062
:1024200000803F6300000063616D00000003008FC7
:102430005F045D175D1D3200000000630000006353
:10244000766D0000000300D85F056225632232002C
:10245000006145630000006366720000000300D461
:102460005F056225631E3200006145630000006362
:10247000746E0000000303E05F056215672A3200F6
:102480000080BF6300000063746D0000000303DC84
:102490005F056225632632000080BF630000006391
:1024A0006A6D0000000300E45F0562855D2E320066
:1024B00000C84263000000636A640000000300EC8F
:1024C0005F056225633A32CDCC4C3D63000000636A
:1024D00072610000000B03F05F056225633E32006D
:1024E00000803F703100007031667271000300950A
:1024F000AA0562256395570000C84270310000703C
:102500003163736C00030099AA0562256399570033
:10251000007A447031000070316373680003009DDD
:10252000AA056225639D570000FA447031000070CF
:102530003163706C000303A1AA05622563A15700F3
:1025400000003E703100007031637068000303A525
:10255000AA05622563A557CDCC4C3E7031000070B2
:102560003177736C000300A9AA05622563A957009F
:10257000007A44703100007031777368000300AD59
:10258000AA05622563AD570000FA4470310000705F
:102590003177706C000303B1AA05622563B157005F
:1025A00000003E703100007031777068000303B5A1
:1025B000AA05622563B557CDCC4C3E703100007042
:1025C00031706F66000303B9AA05622563B957CD60
:1025D000CCCC3D673534006735347800000B030CF4
:1025E00060056215678430000000006735340067BD
:1025F00035347900000B030C6005621567883000E4
:10260000000000673534006735347A00000B030C96
:1026100060056215678C3000000000673534006784
:1026200035346100000B030C6005621567903000C3
:10263000000000673534006735346200000B030C7E
:10264000600562156794300000000067353400674C
:1026500035346300000B030C600562156798300089
:10266000000000673535006735357800000B030C36
:1026700060056215679C30000016436735350067BA
:1026800035357900000B030C6005621567A030003A
:10269000006143673535006735357A00000B030C60
:1026A0006005621567A430000000006735350067DB
:1026B00035356100000B030C6005621567A830001A
:1026C000000000673535006735356200000B030CEC
:1026D0006005621567AC30000000006735350067A3
:1026E00035356300000B030C6005621567B03000E0
:1026F000000000673536006735367800000B030CA4
:102700006005621567B43000000000673536006769
:1027100035367900000B030C6005621567B8300090
:10272000000000673536006735367A00000B030C71
:102730006005621567BC3000000000673536006731
:1027400035366100000B030C6005621567C0300070
:10275000000000673536006735366200000B030C59
:102760006005621567C430000000006735360067F9
:1027700035366300000B030C6005621567C8300036
:10278000000000673537006735377800000B030C11
:102790006005621567CC30000000006735370067C0
:1027A00035377900000B030C6005621567D03000E7
:1027B000000000673537006735377A00000B030CDF
:1027C0006005621567D43000000000673537006788
:1027D00035376100000B030C6005621567D83000C7
:1027E000000000673537006735376200000B030CC7
:1027F0006005621567DC3000000000673537006750
:1028000035376300000B030C6005621567E030008C
:10281000000000673538006735387800000B030C7E
:102820006005621567E43000000000673538006716
:1028300035387900000B030C6005621567E830003D
:10284000000000673538006735387A00000B030C4C
:102850006005621567EC30000000006735380067DE
:1028600035386100000B030C6005621567F030001D
:10287000000000673538006735386200000B030C34
:102880006005621567F430000000006735380067A6
:1028900035386300000B030C6005621567F83000E3
:1028A000000000673539006735397800000B030CEC
:1028B0006005621567FC300000000067353900676D
:1028C00035397900000B030C600562156700310093
:1028D000000000673539006735397A00000B030CBA
:1028E0006005621567043100000000673539006734
:1028F00035396100000B030C600562156708310073
:10290000000000673539006735396200000B030CA1
:1029100060056215670C31000000006735390067FB
:1029200035396300000B030C600562156710310038
:102930000000006739320067393278000001030C6B
:102940006005623E62F432000000006739320067C1
:10295000393279000001030C6005623E62F83200F2
:10296000000000673932006739327A000001030C39
:102970006005623E62FC3200000000673932006789
:10298000393261000001030C6005623E62003300D1
:102990000000006739320067393262000001030C21
:1029A0006005623E62043300000000673932006750
:1029B000393263000001030C6005623E6208330097
:1029C00000000067323800673238780000010310D9
:1029D0006005623E620C3300000000673238006719
:1029E00032387900000103106005623E6210330046
:1029F000000000673238006732387A0000010310A7
:102A00006005623E621433000000006732380067E0
:102A100032386100000103106005623E6218330025
:102A2000000000673238006732386200000103108E
:102A30006005623E621C33000000006732380067A8
:102A400032386300000103106005623E62203300EB
:102A50000000006733300067333078000001031056
:102A60006005623E62243300000000673330006777
:102A700033307900000103106005623E62283300A4
:102A8000000000673330006733307A000001031024
:102A90006005623E622C330000000067333000673F
:102AA00033306100000103106005623E6230330084
:102AB000000000673330006733306200000103100C
:102AC0006005623E62343300000000673330006707
:102AD00033306300000103106005623E623833004A
:102AE0000000006A6964006A69646100000000888F
:102AF000C4DE61FE62B33A000000006A6964006AE5
:102B00006964620000000088C4DE61FE62B73A00BA
:102B10000000006A6964006A69646300000000885C
:102B2000C4DE61FE62BB3A000000006A6964006AAC
:102B30006964640000000088C4DE61FE62BF3A0080
:102B4000000000737973006A61000000000F002E1E
:102B50005F05621567523000504348737973006314
:102B600074000000000F044D5F0562156756300ABF
:102B7000D7233C73797300736C0000000007006C6E
:102B80005F966140625A30000000007379730073F1
:102B90007400000000070011C09661F1BF2D3000E5
:102BA000000000737973006D740000000007024E8E
:102BB000BD0562BDBCB55800000040000000006DBE
:102BC0006500000000000089C41FBD1FBD8C3A00D5
:102BD000000000000000006D64000000000000899B
:102BE000C4F7BCF7BC8C3A00000000737973006531
:102BF0006A000000000700648396616662A43A00E0
:102C000000803F737973006A760000000007006857
:102C1000839661F582493D00000040737973006A34
:102C2000730000000007006C83966166624B3D00F4
:102C300000803F7379730074760000000007007E07
:102C4000C596616662285A0000803F7379730071EF
:102C50007600000000070044B09661B062EE5700B5
:102C60000000007379730073760000000007009C79
:102C7000AE96618B62FB570000803F7379730073DF
:102C80006900000000070098AEBA6160AEFC570012
:102C9000007A4373797300656300000000070066E3
:102CA0006796612068BA2900000000737973006597
:102CB000650000000007006A679661A068BB2900F4
:102CC0000000007379730065780000000007006E53
:102CD0006796616068BC290000803F737973007259
:102CE000786D0000000700726796616662BD29007A
:102CF00000803F73797300626175640000040076A0
:102D0000679661C766B8290000A040000000007304
:102D10007200000000000096AE5CAE5EAE8C3A0021
:102D20000000000000000071720000000000003888
:102D3000B0EBAF3E628C3A00000000000000007172
:102D4000690000000000003CB000B03E628C3A0018
:102D500000000000000000716F0000000000004053
:102D6000B01CB03E628C3A0000000000000000651C
:102D70007200000000000088C46CAB3E628C3A0018
:102D800000000000000000716600000000000088E4
:102D9000C49261095E8C3A000000000000000072DD
:102DA00078000000000000BDC4AB663E628C3A00B3
:102DB000000000000000006D736700000000008943
:102DC000C492613E628C3A00000000000000006383
:102DD0006C65617200000088C4035303538C3A0091
:102DE000000000000000007465737400000000889B
:102DF000C4667D15C08C3A0000000000000000642D
:102E00006566610000000088C4917D3C618C3A00D9
:102E100000000000000000626F6F74000000008876
:102E2000C4BC7DB77C8C3A00000000000000006844
:102E3000656C700000000088C4277D3E628C3A00FB
:102E40000000000000000068000000000000008892
:102E5000C4277D3E628C3A000000007379730067DE
:102E6000706C00000007001A5F96618B626830008A
:102E70000000007379730067756E00000007001E84
:102E80005F9661666269300000803F737973006706
:102E9000636F0000000700225F96614062673000A8
:102EA00000803F737973006770610000000700269F
:102EB0005F96618B626A300000004073797300672F
:102EC000646900000007002A5F966166626B30004B
:102ED00000000000000000676300000000000088A0
:102EE000C46E7B7E7B8C3A00000000000000006D09
:102EF00061000000000B04705F056215675F30CD54
:102F0000CCCC3D000000006664000000000300A17E
:102F1000C4966166624A3D000000007564610075F8
:102F200064613000000300BDC4DE61FE62483A0007
:102F3000000000756461007564613100000300BD2C
:102F4000C4DE61FE624C3A000000007564610075E9
:102F500064613200000300BDC4DE61FE62503A00CD
:102F6000000000756461007564613300000300BDFA
:102F7000C4DE61FE62543A000000007564620075B0
:102F800064623000000300BDC4DE61FE62583A0096
:102F9000000000756462007564623100000300BDCA
:102FA000C4DE61FE625C3A00000000756462007578
:102FB00064623200000300BDC4DE61FE62603A005C
:102FC000000000756462007564623300000300BD98
:102FD000C4DE61FE62643A0000000075646300753F
:102FE00064633000000300BDC4DE61FE62683A0025
:102FF000000000756463007564633100000300BD68
:10300000C4DE61FE626C3A00000000756463007506
:1030100064633200000300BDC4DE61FE62703A00EA
:10302000000000756463007564633300000300BD35
:10303000C4DE61FE62743A000000007564640075CD
:1030400064643000000300BDC4DE61FE62783A00B3
:10305000000000756464007564643100000300BD05
:10306000C4DE61FE627C3A00000000756464007595
:1030700064643200000300BDC4DE61FE62803A0079
:10308000000000756464007564643300000300BDD3
:10309000C4DE61FE62843A000000005F7465005F78
:1030A00074657800000002DAC405623E6260550073
:1030B0000000005F7465005F74657900000002DA4B
:1030C000C405623E626455000000005F7465005FE5
:1030D00074657A00000002DAC405623E6268550039
:1030E0000000005F7465005F74656100000002DA33
:1030F000C405623E626C55000000005F7465005FAD
:1031000074656200000002DAC405623E6270550018
:103110000000005F7465005F74656300000002DA00
:10312000C405623E627455000000005F7472005F67
:1031300074727800000002DAC405623E62855600AF
:103140000000005F7472005F74727900000002DAA0
:10315000C405623E628956000000005F7472005F21
:1031600074727A00000002DAC405623E628D560075
:103170000000005F7472005F74726100000002DA88
:10318000C405623E629156000000005F7472005FE9
:1031900074726200000002DAC405623E6295560055
:1031A0000000005F7472005F74726300000002DA56
:1031B000C405623E629956000000005F7473005FB0
:1031C00074733100000002DAC405623E62F05500FB
:1031D0000000005F7073005F70733100000002DA5E
:1031E000C405623E620056000000005F6373005F2A
:1031F00063733100000002DAC405623E62105600BB
:103200000000005F6573005F65733100000002DA43
:10321000C405623E622056000000005F7873005FC4
:1032200078733100000002DAC405623E6250590032
:103230000000005F6665005F66653100000002DA2D
:10324000C405623E623056000000005F7473005F88
:1032500074733200000002DAC405623E62F4550065
:103260000000005F7073005F70733200000002DACC
:10327000C405623E620456000000005F6373005F95
:1032800063733200000002DAC405623E6214560025
:103290000000005F6573005F65733200000002DAB2
:1032A000C405623E622456000000005F7873005F30
:1032B00078733200000002DAC405623E6268590089
:1032C0000000005F6665005F66653200000002DA9C
:1032D000C405623E623456000000005F7473005FF4
:1032E00074733300000002DAC405623E62F85500D0
:1032F0000000005F7073005F70733300000002DA3B
:10330000C405623E620856000000005F6373005F00
:1033100063733300000002DAC405623E621856008F
:103320000000005F6573005F65733300000002DA20
:10333000C405623E622856000000005F7873005F9B
:1033400078733300000002DAC405623E62805900DF
:103350000000005F6665005F66653300000002DA0A
:10336000C405623E623856000000005F7473005F5F
:1033700074733400000002DAC405623E62FC55003A
:103380000000005F7073005F70733400000002DAA9
:10339000C405623E620C56000000005F6373005F6C
:1033A00063733400000002DAC405623E621C5600FA
:1033B0000000005F6573005F65733400000002DA8F
:1033C000C405623E622C56000000005F7873005F07
:1033D00078733400000002DAC405623E6298590036
:1033E0000000005F6665005F66653400000002DA79
:1033F000C405623E623C5600000000000000005F11
:1034000064616D0000000088C4825E825E8C3A00B8
:1034100000000000000000736530300000020088EA
:10342000C4BA61D5620758000000000000000073B4
:103430006530310000020088C4BA61D562095800C5
:1034400000000000000000736530320000020088B8
:10345000C4BA61D5620B5800000000000000007380
:103460006530330000020088C4BA61D5620D58008F
:103470000000000000000073653034000002008886
:10348000C4BA61D5620F580000000000000000734C
:103490006530350000020088C4BA61D56211580059
:1034A0000000000000000073653036000002008854
:1034B000C4BA61D562135800000000000000007318
:1034C0006530370000020088C4BA61D56215580023
:1034D0000000000000000073653038000002008822
:1034E000C4BA61D5621758000000000000000073E4
:1034F0006530390000020088C4BA61D562195800ED
:1035000000000000000000736531300000020088F8
:10351000C4BA61D5621B58000000000000000073AF
:103520006531310000020088C4BA61D5621D5800BF
:1035300000000000000000736531320000020088C6
:10354000C4BA61D5621F580000000000000000737B
:103550006531330000020088C4BA61D56221580089
:103560000000000000000073653134000002008894
:10357000C4BA61D562235800000000000000007347
:103580006531350000020088C4BA61D56225580053
:103590000000000000000073653136000002008862
:1035A000C4BA61D562275800000000000000007313
:1035B0006531370000020088C4BA61D5622958001D
:1035C0000000000000000073653138000002008830
:1035D000C4BA61D5622B58000000000000000073DF
:1035E0006531390000020088C4BA61D5622D5800E7
:1035F0000000000000000073653230000002008807
:10360000C4BA61D5622F58000000000000000073AA
:103610006532310000020088C4BA61D562315800B9
:1036200000000000000000736532320000020088D4
:10363000C4BA61D562335800000000000000007376
:103640006532330000020088C4BA61D56235580083
:1036500000000000000000736532340000020088A2
:10366000C4BA61D562375800000000000000007342
:103670006532350000020088C4BA61D5623958004D
:103680000000000000000073653236000002008870
:10369000C4BA61D5623B580000000000000000730E
:1036A0006532370000020088C4BA61D5623D580017
:1036B000000000000000007365323800000200883E
:1036C000C4BA61D5623F58000000000000000073DA
:1036D0006532390000020088C4BA61D562415800E1
:1036E00000000000000000737973000000000088F3
:1036F000C4EA645E638C3A000000000000000070C1
:103700003100000000000088C4EA645E638C3A0067
:1037100000000000000000310000000000000088F0
:10372000C4EA645E638C3A000000000000000032CE
:103730000000000000000088C4EA645E638C3A0068
:1037400000000000000000330000000000000088BE
:10375000C4EA645E638C3A0000000000000000349C
:103760000000000000000088C4EA645E638C3A0038
:103770000000000000000078000000000000008849
:10378000C4EA645E638C3A00000000000000007927
:103790000000000000000088C4EA645E638C3A0008
:1037A000000000000000007A000000000000008817
:1037B000C4EA645E638C3A0000000000000000610F
:1037C0000000000000000088C4EA645E638C3A00D8
:1037D00000000000000000620000000000000088FF
:1037E000C4EA645E638C3A000000000000000063DD
:1037F0000000000000000088C4EA645E638C3A00A8
:103800000000000000000067353400000000008860
:10381000C4EA645E638C3A000000000000000067A8
:103820003535000000000088C4EA645E638C3A000D
:10383000000000000000006735360000000000882E
:10384000C4EA645E638C3A00000000000000006778
:103850003537000000000088C4EA645E638C3A00DB
:1038600000000000000000673538000000000088FC
:10387000C4EA645E638C3A00000000000000006748
:103880003539000000000088C4EA645E638C3A00A9
:1038900000000000000000673932000000000088CE
:1038A000C4EA645E638C3A00000000000000006718
:1038B0003238000000000088C4EA645E638C3A007D
:1038C00000000000000000673330000000000088A6
:1038D000C4EA645E638C3A00000000000000006DE2
:1038E000706F000000000088C4EA645E638C3A00D8
:1038F00000000000000000706F73000000000088EE
:10390000C4EA645E638C3A00000000000000006FAF
:103910006673000000000088C4EA645E638C3A00AD
:1039200000000000000000686F6D000000000088CB
:10393000C4EA645E638C3A0000000000000000707E
:103940007262000000000088C4EA645E638C3A0082
:103950000000000000000070777200000000008886
:10396000C4EA645E638C3A00000000000000006A54
:103970006F67000000000088C4EA645E638C3A0050
:10398000000000000000006A696400000000008878
:10399000C4EA645E638C3A00000000000000007519
:1039A0006461000000000088C4EA645E638C3A0031
:1039B0000000000000000075646200000000008844
:1039C000C4EA645E638C3A000000000000000075E9
:1039D0006463000000000088C4EA645E638C3A00FF
:1039E0000000000000000075646400000000008812
:1039F000C4EA645E638C3A00000000000000005FCF
:103A00007465000000000088C4EA645E638C3A00BC
:103A1000000000000000005F7472000000000088D9
:103A2000C4EA645E638C3A00000000000000005F9E
:103A30007473000000000088C4EA645E638C3A007E
:103A4000000000000000005F7073000000000088AC
:103A5000C4EA645E638C3A00000000000000005F6E
:103A60006373000000000088C4EA645E638C3A005F
:103A7000000000000000005F657300000000008887
:103A8000C4EA645E638C3A00000000000000005F3E
:103A90007873000000000088C4EA645E638C3A001A
:103AA000000000000000005F666500000000008864
:103AB000C4EA645E638C3A00000000000000006D00
:103AC0000000000000000088C4DB673E628C3A0002
:103AD00000000000000000710000000000000088ED
:103AE000C4C1673E628C3A00000000000000006F15
:103AF0000000000000000088C4A7673E628C3A0006
:103B00000000000000000024000000000000008809
:103B1000C4F5673E628C3A00000000486F6D696E24
:103B200067206572726F72202D202563206178698D
:103B3000732073657474696E6773206D6973636F46
:103B40006E666967757265640050726F62696E6750
:103B5000206572726F72202D202563206178697351
:103B60002063616E6E6F74206D6F76652064757270
:103B7000696E672070726F62696E67005B69645D71
:103B8000202054696E7947204944253330730A0058
:103B90005B68765D2020686172647761726520766B
:103BA000657273696F6E2531362E32660A005B6866
:103BB000705D2020686172647761726520706C614D
:103BC00074666F726D2531352E32660A005B66763B
:103BD0005D20206669726D7761726520766572730B
:103BE000696F6E2531362E32660A005B66625D2093
:103BF000206669726D77617265206275696C6425F3
:103C000031382E32660A00456E7465722024626F68
:103C10006F743D3120746F20656E74657220746816
:103C20006520626F6F74206C6F616465722E0A008C
:103C30000A0A0A2323232054696E794720424F4FF2
:103C400054204C4F414445522048656C702023233A
:103C5000230A00456E7465722024646566613D31F7
:103C600020746F20726573657420746865207379A1
:103C70007374656D20746F20746865206661637469
:103C80006F72792064656661756C742076616C75FD
:103C900065732E0A546869732077696C6C206F769F
:103CA0006572777269746520616E79206368616EF0
:103CB00067657320796F752068617665206D616432
:103CC000652E0A000A0A0A2323232054696E7947C5
:103CD00020524553544F52452044454641554C547B
:103CE000532048656C70202323230A00496E766FA9
:103CF0006B652073656C662074657374206279202F
:103D0000656E746572696E672024746573743D4EC8
:103D1000207768657265204E206973206F6E65207C
:103D20006F663A0A202024746573743D3120207335
:103D30006D6F6B6520746573740A2020247465733D
:103D4000743D322020686F6D696E672074657374EE
:103D500020202028796F75206D7573742074726926
:103D60007020686F6D696E6720737769746368652A
:103D700073290A202024746573743D3320207371E5
:103D8000756172652074657374202020286120732A
:103D90006572696573206F662073717561726573F2
:103DA000290A202024746573743D342020617263D5
:103DB000207465737420202020202028736F6D6587
:103DC000206C6172676520636972636C6573290A90
:103DD000202024746573743D3520206477656C6CF5
:103DE000207465737420202020286D6F7665732001
:103DF0007370616365642062792031207365636F3D
:103E00006E64206477656C6C73290A2020247465C5
:103E100073743D36202066656564686F6C64207439
:103E20006573742028656E746572202120616E644C
:103E3000207E20746F20686F6C6420616E64207235
:103E40006573746172742C20726573706563746934
:103E500076656C79290A202024746573743D3720B7
:103E6000204D20636F64657320746573742020286F
:103E70004D20636F64657320696E7465726D696E41
:103E8000676C65642077697468206D6F7665732947
:103E90000A202024746573743D3820204A534F4E05
:103EA00020746573742020202020286D6F74696F42
:103EB0006E20746573742072756E207573696E67F9
:103EC000204A534F4E20636F6D6D616E6473290AF3
:103ED000202024746573743D392020696E766572E4
:103EE00073652074696D6520746573740A202024DD
:103EF000746573743D313020726F74617279206D16
:103F00006F74696F6E20746573740A202024746561
:103F100073743D313120736D616C6C206D6F76650B
:103F20007320746573740A202024746573743D31A2
:103F30003220736C6F77206D6F76657320746573B4
:103F4000740A202024746573743D313320636F6FCD
:103F50007264696E6174652073797374656D206F26
:103F60006666736574207465737420284739322C33
:103F7000204735342D473539290A0A54657374733F
:103F800020617373756D6520612063656E74657261
:103F90006564205859206F726967696E20616E648C
:103FA000206174206C656173742038306D6D2063FE
:103FB0006C656172616E636520696E20616C6C2056
:103FC000646972656374696F6E730A5465737473A0
:103FD00020617373756D65205A2068617320617468
:103FE000206C656173742034306D6D20706F73695F
:103FF000697469766520636C656172616E63650AD8
:104000005465737473207374617274207769746873
:104010002061204730205830205930205A30206D00
:104020006F76650A486F6D696E67206973207468E2
:104030006520657863657074696F6E2E204E6F2001
:10404000696E697469616C20706F736974696F6EF1
:10405000206F7220636C656172616E6365206973A5
:1040600020617373756D65640A000A0A0A232323AD
:104070002054696E79472053454C4620544553548B
:104080002048656C70202323230A00456163682063
:104090002420636F6D6D616E642061626F766520B0
:1040A000616C736F20646973706C617973207468DC
:1040B0006520746F6B656E20666F72206561636842
:1040C0002073657474696E6720696E205B205D20C3
:1040D000627261636B6574730A546F2076696577E9
:1040E0002073657474696E677320656E74657220E1
:1040F0006120746F6B656E3A0A0A2020243C746F4D
:104100006B656E3E0A0A466F72206578616D706C51
:1041100065202479667220746F20646973706C6105
:1041200079207468652059206D6178206665656422
:1041300020726174650A0A546F2075706461746539
:104140002073657474696E677320656E7465722080
:10415000746F6B656E20657175616C732076616C30
:1041600075653A0A0A2020243C746F6B656E3E3DEB
:104170003C76616C75653E0A0A466F72206578610F
:104180006D706C6520247966723D38303020746F14
:1041900020736574207468652059206D61782066ED
:1041A000656564207261746520746F20383030203A
:1041B0006D6D2F6D696E7574650A466F7220636F41
:1041C0006E66696775726174696F6E20646574618B
:1041D000696C73207365653A2068747470733A2F44
:1041E0002F6769746875622E636F6D2F73796E74B3
:1041F0006865746F732F54696E79472F77696B699F
:104200002F54696E79472D436F6E666967757261C9
:1042100074696F6E0A00546865736520636F6D6D15
:10422000616E6473206172652061637469766520D4
:10423000666F7220636F6E66696775726174696F0D
:104240006E3A0A2020247379732053686F772073A5
:10425000797374656D202867656E6572616C2920BD
:1042600073657474696E67730A20202431202020DE
:1042700053686F77206D6F746F722031207365748F
:1042800074696E677320286F722077686174657631
:104290006572206D6F746F7220796F752077616E13
:1042A0007420312C322C332C34290A2020247820FD
:1042B000202053686F7720582061786973207365D8
:1042C0007474696E677320286F72207768617465F3
:1042D000766572206178697320796F752077616ED9
:1042E0007420782C792C7A2C612C622C63290A207A
:1042F00020246D20202053686F7720616C6C206D26
:104300006F746F722073657474696E67730A20200E
:10431000247120202053686F7720616C6C206178B5
:1043200069732073657474696E67730A2020246F43
:1043300020202053686F7720616C6C206F66667355
:1043400065742073657474696E67730A2020242471
:1043500020202053686F7720616C6C207365747423
:10436000696E67730A2020246820202053686F77C5
:1043700020746869732068656C702073637265656A
:104380006E0A0A000A0A0A2323232054696E794719
:1043900020434F4E46494755524154494F4E2048BD
:1043A000656C70202323230A000A466F722064651F
:1043B0007461696C65642054696E794720696E6622
:1043C0006F207365653A2068747470733A2F2F6795
:1043D00069746875622E636F6D2F73796E7468658A
:1043E000746F732F54696E79472F77696B692F0A41
:1043F000466F7220746865206C6174657374206602
:1044000069726D77617265207365653A20687474AE
:1044100070733A2F2F6769746875622E636F6D2F02
:1044200073796E746865746F732F54696E79470A77
:10443000506C65617365206C6F6720616E792069CF
:10444000737375657320617420687474703A2F2FCC
:104450007777772E73796E746865746F732E636FD8
:104460006D2F666F72756D730A486176652066758B
:104470006E0A000A4E6F74653A2054696E794720BF
:1044800067656E657261746573206175746F6D61C7
:1044900074696320737461747573207265706F72D0
:1044A00074732062792064656661756C740A54685F
:1044B00069732063616E2062652064697361626C58
:1044C000656420627920656E746572696E67202468
:1044D00073763D300A536565207468652077696B93
:1044E000692062656C6F7720666F72206D6F7265F0
:1044F0002064657461696C732E0A00546865736585
:1045000020636F6D6D616E647320617265206163FD
:10451000746976652066726F6D2074686520636FBC
:104520006D6D616E64206C696E653A0A205E78205C
:10453000202020202020202020202020526573656C
:10454000742028636F6E74726F6C207829202D2080
:10455000736F6674776172652072657365740A2083
:10456000203F202020202020202020202020204DFF
:10457000616368696E6520706F736974696F6E201E
:10458000616E642067636F6465206D6F64656C2085
:1045900073746174650A20202420202020202020AC
:1045A00020202020202053686F7720616E642073C4
:1045B000657420636F6E66696775726174696F6E8A
:1045C0002073657474696E67730A2020212020208F
:1045D0002020202020202020202046656564686F50
:1045E0006C64202D2073746F70206D6F74696F6E12
:1045F00020776974686F7574206C6F73696E6720BB
:10460000706F736974696F6E0A20207E20202020ED
:104610002020202020202020204379636C65205317
:1046200074617274202D20726573746172742066D7
:10463000726F6D2066656564686F6C640A2020681F
:104640002020202020202020202020202053686FA0
:104650007720746869732068656C70207363726575
:10466000656E0A2020246820202020202020202081
:1046700020202053686F7720636F6E6669677572BC
:104680006174696F6E2068656C7020736372656514
:104690006E0A20202474657374202020202020209E
:1046A00020204C6973742073656C662D7465737477
:1046B000730A202024746573743D4E20202020202E
:1046C000202052756E2073656C662D74657374209E
:1046D0004E0A202024686F6D653D31202020202067
:1046E000202052756E206120686F6D696E672063AF
:1046F00079636C650A202024646566613D31202061
:104700002020202020526573746F726520616C6CCC
:104710002073657474696E677320746F20226661FC
:1047200063746F7279222064656661756C74730AB4
:10473000000A0A0A2323232054696E79472048651A
:104740006C70202323230A005B6A735D20206A7348
:104750006F6E2073657269616C697A652073747914
:104760006C65253964205B303D72656C61786564E9
:104770002C313D7374726963745D0A005B6A765D07
:1047800020206A736F6E20766572626F7369747928
:1047900025313564205B303D73696C656E742C3156
:1047A0003D666F6F7465722C323D6D657373616722
:1047B00065732C333D636F6E666967732C343D6C93
:1047C000696E656E756D2C353D766572626F7365C9
:1047D0005D0A005B656A5D2020656E61626C652024
:1047E0006A736F6E206D6F646525313364205B30B2
:1047F0003D746578742C313D4A534F4E5D0A000C70
:10480000590659FF58FA58F158E658DB58CF58C3A3
:1048100058B5589E588F5882587658625855584007
:10482000582C582958265817580258ED57DE57CE9D
:1048300057BC57A55788576B5752573C572B57199A
:10484000570C57FA56E056DD56DA56D756D456D19D
:1048500056CE56CB56C856C556C256BF56BC56B98C
:1048600056B656B356B056AD56AA56A756A456A13C
:10487000569E569B569856955692568F568C5689EC
:10488000568656835680567D567A5677567456719C
:10489000566E566B566856655662565F565C56594C
:1048A000565656535650564D564A564756445641FC
:1048B000563E561A56FA55E055C655AC5588556BB6
:1048C0005553553D552355FF54E254D054B0549997
:1048D0005480545E54455427540B54F353E153C34E
:1048E00053AE53AA53A653A2539E539A5396539230
:1048F000538E538A53865382537E537A5376537220
:10490000536E5354533A5327530B53F952E252C147
:1049100052B0529052705256523C522552F251C5EA
:1049200051A55183515D5136511A51FB50E150C789
:1049300050A2507950615036500A50D44F9F4F8D3D
:104940004F7B4F6C4F594F404F1E4F0C4FFA4EE864
:104950004ED64EC44EB24EA04E8E4E7C4E6A4E582F
:104960004E464E344E224E1E4E1A4E164E124E0ECD
:104970004E0A4E064E024EFE4DFA4DF64DF24DEEEB
:104980004DEA4DE64DE24DDE4DDA4DD64DD24DBEEF
:104990004DA04D844D594D344D0F4D0B4D074D03DA
:1049A0004DFF4CFB4CF74CF34CEF4CEB4CE74CE31E
:1049B0004CDF4CDB4CD74CC34CA74C8B4C6F4C534F
:1049C0004C374C1B4CFF4BE34BC74BAB4B8F4B73E4
:1049D0004B6F4B6B4B674B634B5F4B5B4B574B4387
:1049E0004B1B4BF44ACE4AA14A7B4A4E4A4A4A469E
:1049F0004A424A2F4A0E4AF9494A6F6767696E6709
:104A0000206379636C65206661696C65640050722F
:104A10006F626520656E64706F696E7420697320C3
:104A20007374617274696E6720706F696E74005080
:104A3000726F6265206379636C65206661696C657D
:104A40006400323439003234380032343700486F71
:104A50006D696E67204572726F72202D20486F6DF0
:104A6000696E67207377697463686573206D697315
:104A7000636F6E6669677572656400486F6D696E15
:104A800067204572726F72202D204E6567617469D0
:104A90007665206C61746368206261636B6F666623
:104AA00000486F6D696E67204572726F72202D200D
:104AB00054726176656C206D696E2026206D617878
:104AC00020617265207468652073616D6500486FB0
:104AD0006D696E67204572726F72202D204C617473
:104AE00063682076656C6F63697479206973207AD6
:104AF00065726F00486F6D696E67204572726F72E4
:104B0000202D205365617263682076656C6F636940
:104B10007479206973207A65726F00486F6D696ED1
:104B200067204572726F72202D20426164206F727F
:104B3000206E6F20617869732073706563696669A0
:104B4000656400486F6D696E67206379636C6520EA
:104B50006661696C65640032333900323338003283
:104B600033370032333600323335003233340032DB
:104B7000333300536F6674206C696D6974206578F7
:104B8000636565646564202D2043206D6178005362
:104B90006F6674206C696D697420657863656564FF
:104BA0006564202D2043206D696E00536F6674206C
:104BB0006C696D6974206578636565646564202D32
:104BC0002042206D617800536F6674206C696D69B6
:104BD00074206578636565646564202D2042206DCE
:104BE000696E00536F6674206C696D697420657816
:104BF000636565646564202D2041206D61780053F4
:104C00006F6674206C696D6974206578636565648E
:104C10006564202D2041206D696E00536F667420FD
:104C20006C696D6974206578636565646564202DC1
:104C3000205A206D617800536F6674206C696D692D
:104C400074206578636565646564202D205A206D45
:104C5000696E00536F6674206C696D6974206578A5
:104C6000636565646564202D2059206D617800536B
:104C70006F6674206C696D6974206578636565641E
:104C80006564202D2059206D696E00536F66742075
:104C90006C696D6974206578636565646564202D51
:104CA0002058206D617800536F6674206C696D69BF
:104CB00074206578636565646564202D2058206DD7
:104CC000696E00536F6674206C696D697420657835
:104CD0006365656465640032313900323138003211
:104CE0003137003231360032313500323134003262
:104CF0003133003231320032313100323130003262
:104D0000303900323038003230370032303600541B
:104D1000726170657A6F696420706C616E6E657225
:104D2000206661696C656420746F20636F6E7665C0
:104D3000726765004C696D69742073776974636884
:104D400020686974202D2053687574646F776E2015
:104D50006F63637572726564004D616368696E6547
:104D600020697320616C61726D6564202D20436F32
:104D70006D6D616E64206E6F742070726F63657309
:104D8000736564004D6F7665206C6573732074687D
:104D9000616E206D696E696D756D2074696D650059
:104DA0004D6F7665206C657373207468616E206D3D
:104DB000696E696D756D206C656E67746800476516
:104DC0006E657269632054696E7947206572726FEF
:104DD0007200313939003139380031393700313911
:104DE0003600313935003139340031393300313949
:104DF0003200313931003139300031383900313841
:104E00003800313837003138360031383500313824
:104E10003400313833003138320031383100313824
:104E200030005420776F726420697320696E766158
:104E30006C6964005420776F7264206973206D6917
:104E40007373696E67005220776F726420697320F4
:104E5000696E76616C6964005220776F72642069B4
:104E600073206D697373696E67005120776F726488
:104E700020697320696E76616C6964005120776FD8
:104E80007264206973206D697373696E67004C20CA
:104E9000776F726420697320696E76616C69640053
:104EA0004C20776F7264206973206D697373696E2B
:104EB00067004820776F726420697320696E76619D
:104EC0006C6964004820776F7264206973206D6993
:104ED0007373696E67004520776F72642069732071
:104EE000696E76616C6964004520776F7264206931
:104EF00073206D697373696E67004420776F726405
:104F000020697320696E76616C6964004420776F54
:104F10007264206973206D697373696E6700502035
:104F2000776F7264206973206E6F742061207661E0
:104F30006C696420746F6F6C206E756D62657200B1
:104F40005020776F7264206973206E6F7420616ED9
:104F500020696E7465676572005020776F726420F7
:104F60006973206E65676174697665005020776F9C
:104F70007264206973207A65726F005020776F72B7
:104F80006420697320696E76616C696400502077D3
:104F90006F7264206973206D697373696E67004175
:104FA00072632073706563696669636174696F6EAB
:104FB000206572726F72202D20656E64706F696E4D
:104FC00074206973207374617274696E6720706FE6
:104FD000696E74004172632073706563696669630A
:104FE0006174696F6E206572726F72202D2072611C
:104FF0006469757320617263206F7574206F662019
:10500000746F6C6572616E636500417263207370CA
:105010006563696669636174696F6E206572726F3A
:1050200072202D206D697373696E67206F666673D9
:105030006574287329004172632073706563696623
:1050400069636174696F6E206572726F72202D20C2
:105050006D697373696E6720617869732865732958
:105060000041726320737065636966696361746986
:105070006F6E206572726F72005370696E646C653A
:10508000206D757374206265207475726E696E6729
:1050900020666F72207468697320636F6D6D616E36
:1050A00064005370696E646C65206D757374206262
:1050B00065206F666620666F72207468697320636E
:1050C0006F6D6D616E64005370696E646C65205322
:1050D00020776F726420697320696E76616C6964F1
:1050E000005370696E646C65205320776F72642082
:1050F0006973206D697373696E67005370696E64BC
:105100006C652073706565642065786365656465AA
:1051100064206D6178696D756D005370696E646CA3
:10512000652073706565642062656C6F77206D69BA
:105130006E696D756D0050726F6772616D6D65643B
:1051400020706F696E742073616D652061732063D8
:10515000757272656E7420706F696E740043757439
:1051600074657220636F6D70656E736174696F6EC4
:105170002063616E6E6F7420626520656E61626C83
:105180006564005265717565737465642076656C3D
:105190006F636974792065786365656473206C69F1
:1051A0006D697473004730206F72204731206D7530
:1051B00073742062652061637469766520666F721E
:1051C0002047353300526F746172792061786573BE
:1051D0002063616E6E6F7420626520757365642054
:1051E00077697468207468697320636F6D6D616E90
:1051F0006400496E76657273652074696D65206D13
:105200006F64652063616E6E6F74206265207573D4
:1052100065642077697468207468697320636F6DB2
:105220006D616E64004665656472617465206E6FC1
:1052300074207370656369666965640053656C65A5
:105240006374656420706C616E6520697320696E9B
:1052500076616C69640053656C6563746564207085
:105260006C616E65206973206D697373696E670088
:10527000417869732074617267657420706F736917
:1052800074696F6E20697320696E76616C69640061
:10529000417869732074617267657420706F7369F7
:1052A00074696F6E206973206D697373696E67002E
:1052B000417869732069732064697361626C656405
:1052C000004178697320697320696E76616C696446
:1052D00020666F72207468697320636F6D6D616EF4
:1052E0006400417869732063616E6E6F742062653B
:1052F0002070726573656E74004178697320776FF2
:105300007264206D697373696E670047636F6465CB
:10531000206D6F64616C2067726F75702076696FA5
:105320006C6174696F6E004D20636F646520756EEB
:10533000737570706F727465640047636F64652085
:10534000636F6D6D616E6420756E737570706F72D2
:105350007465640047656E657269632047636F64B6
:105360006520696E707574206572726F72003132DB
:1053700039003132380031323700313236003132C3
:1053800035003132340031323300313232003132C3
:1053900031003132300031313900313138003131B2
:1053A00037003131360031313500313134004A5364
:1053B0004F4E20737472696E6720746F6F206C6F2C
:1053C0006E67004A534F4E20696E70757420686195
:1053D0007320746F6F206D616E79207061697273D4
:1053E000004A534F4E2073796E7461782065727253
:1053F0006F7200496E7075742076616C75652072ED
:10540000616E6765206572726F7200496E707574A7
:105410002065786365656473206D6178696D756D6D
:105420002076616C756500496E707574206C6573CB
:1054300073207468616E206D696E696D756D20767C
:10544000616C756500496E7075742065786365657B
:105450006473206D6178206C656E67746800436FBB
:105460006D6D616E64206E6F74206163636570742E
:10547000656420617420746869732074696D6500C7
:10548000506172616D657465722063616E6E6F74D8
:10549000206265207265616400506172616D65749F
:1054A000657220697320726561642D6F6E6C79007E
:1054B000556E737570706F72746564206E756D6271
:1054C0006572206F72204A534F4E207479706500C8
:1054D000426164206E756D62657220666F726D61E7
:1054E0007400496E76616C6964206F72206D616C26
:1054F000666F726D656420636F6D6D616E640055DB
:105500006E7265636F676E697A656420636F6D6D37
:10551000616E64206F7220636F6E666967206E61D2
:105520006D650047656E65726963206173736572AE
:1055300074696F6E206661696C757265004D656D8A
:105540006F7279206661756C74206465746563742C
:10555000656400537461636B206F766572666C6F6F
:105560007720646574656374656400436F6E74725C
:105570006F6C6C657220617373657274696F6E20F5
:105580006661696C7572650043616E6F6E69636117
:105590006C206D616368696E6520617373657274F8
:1055A000696F6E206661696C75726500506C616E22
:1055B0006E657220617373657274696F6E206661C7
:1055C000696C7572650053746570706572206173E3
:1055D00073657274696F6E206661696C75726500BF
:1055E000456E636F64657220617373657274696F71
:1055F0006E206661696C75726500494F2073756233
:105600002D73797374656D20617373657274696F3E
:105610006E206661696C75726500436F6E666967BE
:10562000207375622D73797374656D206173736572
:105630007274696F6E206661696C757265003839C5
:105640000038380038370038360038350038340034
:1056500038330038320038310038300037390037FD
:1056600038003737003736003735003734003733E6
:105670000037320037310037300036390036380015
:1056800036370036360036350036340036330036CD
:1056900032003631003630003539003538003537C4
:1056A00000353600353500353400353300353200ED
:1056B00035310035300034390034380034370034A7
:1056C00036003435003434003433003432003431A1
:1056D00000343000333900333800333700333600BC
:1056E00042616420737461747573207265706F72A7
:1056F000742073657474696E6700506572736973A2
:1057000074656E6365206572726F7200466C6F61BE
:1057100074206973204E414E00466C6F617420699D
:105720007320696E66696E697465004D6F766520D9
:1057300074696D65206973204E414E004D6F76652A
:105740002074696D6520697320696E66696E69747D
:10575000650047656E65726963206578636570747E
:10576000696F6E207265706F7274004661696C6556
:105770006420746F2067657420706C616E6E657252
:10578000206275666665720053797374656D206179
:105790006C61726D202D207368757474696E67205A
:1057A000646F776E00496E697469616C697A6174BF
:1057B000696F6E206661696C75726500526561641F
:1057C0002D6F6E6C79206164647265737300496E2D
:1057D00076616C6964204164647265737300446926
:1057E00076696465206279207A65726F00466C6F15
:1057F0006174696E6720706F696E74206572726F74
:105800007200496E7465726E616C2072616E6765BC
:10581000206572726F7200496E7465726E616C20E1
:105820006572726F720031390031380046756E63EF
:1058300074696F6E206973207374756262656400A9
:10584000456E746572696E6720626F6F74206C6F4D
:105850006164657200496E697469616C697A696E28
:1058600067004275666665722066756C6C202D2037
:10587000666174616C004275666665722066756C5F
:105880006C0042756666657220656D707479004EB5
:105890006F207375636820646576696365004D6188
:1058A000782066696C652073697A65206578636520
:1058B000656465640046696C65206E6F74206F7066
:1058C000656E00456E64206F662066696C650045F4
:1058D0006E64206F66206C696E650048617264209A
:1058E0007265736574005465726D696E6174656488
:1058F00000436F6D706C657465004E6F6F7000458E
:10590000616761696E004572726F72004F4B005B98
:105910007031706F665D2070776D2070686173659F
:10592000206F66662020202531352E3366205B30BF
:105930002E2E315D0A005B70317770685D207077C4
:105940006D20636377207068617365206869253115
:10595000352E3366205B302E2E315D0A005B7031B0
:1059600077706C5D2070776D20636377207068615D
:105970007365206C6F2531352E3366205B302E2EFB
:10598000315D0A005B70317773685D2070776D2040
:105990006363772073706565642068692531352EEF
:1059A00030662052504D0A005B703177736C5D2079
:1059B00070776D20636377207370656564206C6F0A
:1059C0002531352E30662052504D0A005B70316310
:1059D00070685D2070776D206377207068617365F3
:1059E000206869202531352E3366205B302E2E311C
:1059F0005D0A005B703163706C5D2070776D2063B1
:105A000077207068617365206C6F202531352E33E7
:105A100066205B302E2E315D0A005B703163736847
:105A20005D2070776D2063772073706565642068F2
:105A300069202531352E30662052504D0A005B70AA
:105A40003163736C5D2070776D20637720737065B0
:105A50006564206C6F202531352E30662052504D04
:105A60000A005B70316672715D2070776D2066721E
:105A7000657175656E63792020202531352E30667D
:105A800020487A0A0053595354454D205245414409
:105A900059004C6F6164696E6720636F6E66696759
:105AA000732066726F6D20454550524F4D00496E10
:105AB000697469616C697A696E6720636F6E666983
:105AC000677320746F2050726F626F74697820461C
:105AD00069726562616C6C205639302070726F6635
:105AE000696C65007B226572223A7B226662223AEB
:105AF00025302E32662C227374223A25642C226DB6
:105B00007367223A222573227D7D0A007B65723AF3
:105B10007B66623A25302E32662C73743A25642CEB
:105B20006D73673A222573227D7D0A005B71765D75
:105B300020207175657565207265706F72742076AE
:105B40006572626F73697479253764205B303D6FCD
:105B500066662C313D73696E676C652C323D7472DC
:105B600069706C655D0A00716F3A25640A0071699D
:105B70003A25640A0071723A25640A005B73765D07
:105B80002020737461747573207265706F72742055
:105B9000766572626F73697479253664205B303D77
:105BA0006F66662C313D66696C74657265642C3273
:105BB0003D766572626F73655D0A005B73695D2097
:105BC0002073746174757320696E74657276616C8C
:105BD0002531342E3066206D730A004D6F746F725C
:105BE00020256320706F77657220656E61626C6539
:105BF000642073746174653A25322E30660A005B46
:105C0000257325735D206D257320706F7765722075
:105C10006D616E6167656D656E7425313064205B02
:105C2000303D64697361626C65642C313D616C77F1
:105C3000617973206F6E2C323D696E206379636CDD
:105C4000652C333D7768656E206D6F76696E675D94
:105C50000A005B257325735D206D257320706F6CC2
:105C6000617269747925313864205B303D6E6F72E2
:105C70006D616C2C313D726576657273655D0A00ED
:105C80005B257325735D206D2573206D6963726FCD
:105C9000737465707325313664205B312C322C347B
:105CA0002C385D0A005B257325735D206D257320FC
:105CB00074726176656C20706572207265766F6CA7
:105CC0007574696F6E2531302E346625730A005B5A
:105CD000257325735D206D257320737465702061B5
:105CE0006E676C652532302E336625730A005B259E
:105CF0007325735D206D2573206D617020746F2096
:105D00006178697325313564205B303D582C313D15
:105D1000592C323D5A2E2E2E5D0A005B6D745D208B
:105D2000206D6F746F722069646C652074696D6595
:105D30006F75742531342E3266205365630A004E28
:105D40005D4A5D455D2064656700206D6D002069DA
:105D50006E005B73745D20207377697463682074D0
:105D600079706525313864205B303D4E4F2C313DD4
:105D70004E435D0A005465737420232564206E6FC2
:105D80007420666F756E640A004E362047393220E3
:105D9000583735205930205A300A4E372046353092
:105DA000302E300A4E3820473159302E3239315A90
:105DB0002D322E3139380A4E39205837342E3736A5
:105DC0003759302E3035385A2D322E3335350A4E6C
:105DD0003130205837342E373039592D302E30306D
:105DE000305A2D322E3337310A4E31312058373464
:105DF0002E3532395A2D322E3236340A4E31322077
:105E00005837342E36333459302E3130355A2D32FE
:105E10002E3331390A4E3133205837342E3834334B
:105E200059302E3331345A2D322E3138330A4E3117
:105E300034205837352E30303059302E3437315ADF
:105E40002D322E3132360A4E31352059302E36352C
:105E5000305A2D322E3130300A4E313620583734F8
:105E60002E37383359302E3433345A2D322E3133C5
:105E7000310A4E3137205837342E35363659302EC8
:105E80003231375A2D322E3234340A4E31382058BE
:105E900037342E333530592D302E3030305A2D32A4
:105EA0002E3138320A4E3139205837342E313730BE
:105EB0005A2D322E3134340A4E3230205837342E97
:105EC00034323959302E3235395A2D322E31363559
:105ED0000A4E3231205837342E35333359302E3371
:105EE00036335A2D322E3139310A4E32322058375C
:105EF000342E36383959302E3531395A2D322E312B
:105F000031340A4E3233205837342E383434593035
:105F10002E3637345A2D322E3039360A4E3234204E
:105F20005837352E30303059302E3833305A2D32E4
:105F30002E3131340A4E32352059312E3031305A1B
:105F40002D322E3134340A4E3236205837342E3723
:105F5000383759302E3739375A2D322E3039380AE2
:105F60004E3237205837342E36323859302E3633A9
:105F7000385A2D322E3130380A4E323820583734C4
:105F80002E34363959302E3437385A2D322E313599
:105F9000370A4E3239205837342E33303959302EA3
:105FA0003331395A2D322E3131300A4E33302058A8
:105FB00037342E30343459302E3035335A2D322E7A
:105FC0003130380A4E3331205837332E3939305971
:105FD000302E3030305A2D322E3037370A4E333291
:105FE000205837332E3831315A2D312E3934370A73
:105FF0004E3333205837332E39373359302E31361C
:10600000325A2D322E3037390A4E33342058373435
:106010002E32343359302E3433325A2D322E30381A
:10602000340A4E3335205837342E34353959302E12
:106030003634395A2D322E3135370A4E3336205800
:1060400037342E36373659302E3836355A2D322ED3
:106050003130390A4E3337205837342E38333859D7
:10606000312E3032375A2D322E3131310A4E3338FB
:10607000205837352E30303059312E3138395A2D9D
:10608000322E3136300A4E33392059312E333639DB
:106090005A2D322E3139340A4E3430205837342EAE
:1060A00038343259312E3231315A2D322E31333487
:1060B0000A4E3431205837342E36383459312E3088
:1060C00035335A2D322E3132300A4E343220583781
:1060D000342E34323159302E3739305A2D322E3158
:1060E00037360A4E3433205837342E333136593050
:1060F0002E3638345A2D322E3133370A4E3434206E
:106100005837342E31353859302E3532365A2D32F3
:106110002E3037370A4E3435205837332E3934373E
:1061200059302E3331365A2D322E3036370A4E340E
:1061300036205837332E38393459302E3236335AC8
:106140002D322E3034360A4E3437205837332E371E
:10615000333759302E3130355A2D312E3931380AF6
:106160004E3438205837332E36333159302E3030B4
:10617000305A2D312E3837320A4E343920583733C1
:106180002E3435325A2D312E3831350A4E353020E5
:106190005837332E36363559302E3231345A2D3168
:1061A0002E3931340A4E3531205837332E383235B6
:1061B00059302E3337345A2D322E3032380A4E357C
:1061C00032205837332E38373959302E3432375A37
:1061D0002D322E3037360A4E3533205837342E3094
:1061E000393259302E3634315A2D322E3039340A64
:1061F0004E3534205837342E33303659302E38351A
:10620000345A2D322E3139320A4E35352058373432
:106210002E35313959312E3036385A2D322E31340F
:10622000310A4E3536205837342E37333359312E14
:106230003238315A2D322E3134330A4E3537205808
:1062400037342E38343059312E3338385A2D322ED7
:106250003137340A4E3538205837342E38393359CF
:10626000312E3434325A2D322E3136390A4E3539E8
:10627000205837352E30303059312E3534385A2D9C
:10628000322E3132310A4E36302059312E373238E3
:106290005A2D322E3037360A4E3631205837342EAA
:1062A00038343359312E3537315A2D322E3133307F
:1062B0000A4E3632205837342E37333859312E347F
:1062C00036365A2D322E3139350A4E36332058376C
:1062D000342E34373659312E3230345A2D322E3155
:1062E00034370A4E3634205837342E32313559304F
:1062F0002E3934335A2D322E3230320A4E36352072
:106300005837332E39303059302E3632385A2D32F4
:106310002E3130310A4E3636205837332E38343845
:1063200059302E3537365A2D322E3039360A4E3600
:1063300037205837332E35383659302E3331345ACA
:106340002D312E3931330A4E3638205837332E331B
:10635000373759302E3130355A2D312E3830380AF2
:106360004E3639205837332E32373259302E3030AE
:10637000305A2D312E3738370A4E373020583733C0
:106380002E3138325A2D312E3738370A4E373120D8
:106390005837332E3039325A2D312E3735300A4E98
:1063A0003732205837332E34313059302E3331388C
:1063B0005A2D312E3836380A4E3733205837332E7F
:1063C00037383159302E3638395A2D322E3038364A
:1063D0000A4E3734205837342E30393959312E305F
:1063E00030375A2D322E3232340A4E373520583754
:1063F000342E32303559312E3131335A2D322E323E
:1064000031310A4E3736205837342E33363459312D
:106410002E3237325A2D322E3137360A4E37372048
:106420005837342E36323959312E3533375A2D32CA
:106430002E3139310A4E3738205837342E3638321B
:1064400059312E3539305A2D322E3137370A4E37E1
:1064500039205837342E38393459312E3830325AA1
:106460002D322E3036360A4E3830205837352E3001
:10647000303059312E3930385A2D322E3034360AD8
:106480004E38312059322E3038375A2D322E303591
:10649000310A4E3832205837342E38333959312E9C
:1064A0003932375A2D322E3036320A4E3833205890
:1064B00037342E36373959312E3736365A2D322E5B
:1064C0003133360A4E3834205837342E3632355967
:1064D000312E3731335A2D322E3137300A4E38357E
:1064E000205837342E35373259312E3635395A2D1A
:1064F000322E3138300A4E3836205837342E333564
:106500003859312E3434355A2D322E3135370A4E22
:106510003837205837342E31393759312E32383404
:106520005A2D322E3139350A4E3838205837342E0C
:1065300030393059312E3137375A2D322E323435E9
:106540000A4E3839205837332E39383359312E30E6
:1065500037305A2D322E3232350A4E3930205837E4
:10656000332E38323359302E3931305A2D322E31C4
:1065700033380A4E3931205837332E3339345930B5
:106580002E3438325A2D312E3931370A4E393220D5
:106590005837332E31383059302E3236385A2D3163
:1065A0002E3832350A4E3933205837322E393636A6
:1065B00059302E3035345A2D312E3731310A4E397B
:1065C00034205837322E393133592D302E30303077
:1065D0005A2D312E3639330A4E3935205837322E5E
:1065E0003733335A2D312E3634360A4E3936205849
:1065F00037322E39393759302E3236345A2D312E22
:106600003735330A4E3937205837332E3236305922
:10661000302E3532375A2D312E3930320A4E393834
:10662000205837332E36323959302E3839365A2DD4
:10663000322E3037370A4E3939205837332E383416
:106640003059312E3130375A2D322E3232340A4EF3
:10665000313030205837332E38393359312E3136D6
:10666000305A2D322E3234350A4E313031205837DF
:106670003559305A300A004E312054314D360A4EC9
:1066800032204731370A4E33204732310A4E382004
:1066900046313830300A4E392047310A4E313030D9
:1066A0002047393220582D32352E313737592D3386
:1066B000342E303732205A2D312E303030202854AD
:1066C000454D502C2052454D4F5645204C41544588
:1066D00052290A4E33343320582D32352E35393570
:1066E000592D33342E3334390A4E33343420582D57
:1066F00032352E373031592D33342E3433360A4E5D
:1067000033343520582D32352E373931592D333425
:106710002E3532300A4E33343620582D32352E384D
:106720003634592D33342E3630310A4E3334372037
:10673000582D32352E393230592D33342E363739E3
:106740000A4E33343820582D32352E393630592DF3
:1067500033342E3735340A4E33343920582D323500
:106760002E393832592D33342E3832360A4E3335DD
:106770003020582D32352E393837592D33342E38B4
:1067800039350A4E33353120582D32352E393736CA
:10679000592D33342E3936310A4E33353220582DA7
:1067A00032352E393438592D33352E3032330A4EA6
:1067B00033353320582D32352E393033592D33357A
:1067C0002E3038320A4E33353420582D32352E389B
:1067D0003431592D33352E3133380A4E3335352087
:1067E000582D32352E373633592D33352E31393039
:1067F0000A4E33353620582D32352E363639592D3E
:1068000033352E3233390A4E33353720582D323551
:106810002E353539592D33352E3238340A4E33352D
:106820003820582D32352E343333592D33352E330D
:1068300032350A4E33353920582D32352E32393122
:10684000592D33352E3336330A4E33363020582DFA
:1068500032352E313334592D33352E3339370A4EF4
:1068600033363120582D32342E393633592D3335C5
:106870002E3432380A4E33363220582D32342E37E9
:106880003737592D33352E3435350A4E33363320CC
:10689000582D32342E353737592D33352E3437377E
:1068A0000A4E33363420582D32342E333637592D94
:1068B00033352E3439360A4E33363520582D32349E
:1068C0002E313434592D33352E3531310A4E33368D
:1068D0003620582D32332E393039592D33352E3557
:1068E00032320A4E33363720582D32332E36363177
:1068F000592D33352E3532390A4E33363820582D3E
:1069000032332E343033592D33352E3533320A4E4F
:1069100033363920582D32332E313333592D333518
:106920002E3533320A4E33373020582D32322E383E
:106930003533592D33352E3532370A2F4E32353116
:106940003820473058302E333237592D33332E35D7
:1069500032315A2D312E3030300A4E323531392015
:106960004D3330004E31204732300A4E3520473407
:1069700030204731370A4E3130205431204D3036E7
:106980000A284E31352047393020473020583020F2
:106990005930205A30290A4E3230205335303030A9
:1069A000204D3033200A4E32352058302E303634C8
:1069B0002059302E333236205A300A4E3430204798
:1069C0003031204631362E300A4E35302058302EA8
:1069D0003036342059302E3332360A4E3535205871
:1069E000302E3036302059302E3239330A4E363080
:1069F0002058302E3037372059302E3236370A4E55
:106A000036352058302E3131312059302E3235373D
:106A10000A4E37302058302E3134392059302E323A
:106A200035320A4E37352058302E3138382059301B
:106A30002E3235350A4E38302058302E323237203B
:106A400059302E3236380A4E38352058302E3235ED
:106A5000372059302E3237310A4E39302058302EF7
:106A60003333352059302E3236350A4E39352058D9
:106A7000302E3431322059302E3237310A4E3130F7
:106A8000302058302E3437342059302E3238370ADF
:106A90004E3130352058302E3439312059302E3295
:106AA00038390A4E3131302058302E35313720599F
:106AB000302E3237330A4E3131352058302E3534AE
:106AC000342059302E3236330A4E3132302058308D
:106AD0002E3538302059302E3236310A4E3132358B
:106AE0002058302E3539352059302E3236330A4E63
:106AF0003133302058302E3632312059302E323753
:106B0000340A4E3133352058302E3635392059303D
:106B10002E3330360A4E3134302058302E3637334B
:106B20002059302E3333350A4E3134352058302E2B
:106B30003637392059302E3336310A4E3135302030
:106B400058302E3637382059302E3338390A4E31E6
:106B500035352058302E3637302059302E343230EB
:106B60000A4E3136302058302E3637302059302EEC
:106B70003434360A4E3136352058302E36383020EF
:106B800059302E3437340A4E3137302058302E37B2
:106B900030342059302E3439370A4E3137352058A9
:106BA000302E3733322059302E3531350A4E3138B8
:106BB000302058302E3739342059302E3533350AAD
:106BC0004E3138352058302E3837322059302E3556
:106BD00036370A4E3139302058302E393530205969
:106BE000302E3630340A4E3139352058312E30337C
:106BF000312059302E3634370A4E32303020583159
:106C00002E3134392059302E3732320A4E32303557
:106C10002058312E3330382059302E3835340A4E32
:106C20003231302058312E3433302059302E39381B
:106C3000340A4E3231352058312E34343720593011
:106C40002E3938360A4E3232302058312E3632380C
:106C50002059302E3832320A4E3232352058312EF9
:106C60003733322059302E3731340A4E3233302008
:106C700058322E3030392059302E3338310A4E32C6
:106C800033352058322E3131362059302E323636B7
:106C90000A4E3234302058322E3232382059302EBB
:106CA0003135370A4E3234352058322E32383020C2
:106CB00059302E3132330A4E3235302058322E338D
:106CC00033322059302E3039340A4E32353520587F
:106CD000322E3432332059302E3037300A4E32368D
:106CE000302058322E3438392059302E3036350A7B
:106CF0004E3236352058322E3535372059302E3029
:106D000036360A4E3237302058322E363237205936
:106D1000302E3038340A4E3237352058322E36393C
:106D2000332059302E3130390A4E32383020583223
:106D30002E3733302059302E3133330A4E32383526
:106D40002058322E3830352059302E3139300A4E05
:106D50003239302058322E3832392059302E3231E3
:106D6000360A4E3239352058322E383830205930D4
:106D70002E3239310A4E3330302058322E383834E2
:106D80002059302E3330300A4E3330352058322ED1
:106D90003839382059302E3333320A4E33313020CF
:106DA00058322E3930352059302E3336370A4E338B
:106DB00031352058322E3931302059302E34303789
:106DC0000A4E3332302058322E3930382059302E86
:106DD0003434360A4E3332352058322E3930312091
:106DE00059302E3439350A4E3333302058322E384C
:106DF00039372059302E3439350A4E33333520583F
:106E0000322E3839302059302E3532340A4E333450
:106E1000302058322E3834322059302E3630340A51
:106E20004E3334352058322E3831342059302E36F6
:106E300036350A4E3335302058322E373934205902
:106E4000302E3735300A4E3335352058322E37390B
:106E5000312059302E3833380A4E333630205832EC
:106E60002E3831392059302E3937360A4E333635DF
:106E70002058322E3833372059312E3034340A4ED0
:106E80003337302058322E3836322059312E3131B6
:106E9000320A4E3337352058322E383737205931A1
:106EA0002E3134350A4E3338302058322E393132B3
:106EB0002059312E3231370A4E3338352058322E90
:106EC0003931372059312E3232360A4E333930209B
:106ED00058322E3935312059312E3238310A4E335D
:106EE00039352058322E3937302059312E32393544
:106EF0000A4E3430302058322E3939362059312E4E
:106F00003239350A4E3430352058332E3031332063
:106F100059312E3237350A4E3431302058332E3025
:106F200032342059312E3235340A4E34313520581E
:106F3000332E3037302059312E3135310A4E34322C
:106F4000302058332E3037372059312E3133340A20
:106F50004E3432352058332E3132352059312E30CF
:106F600033390A4E3433302058332E3133382059D8
:106F7000312E3031390A4E3433352058332E3230E9
:106F8000352059302E3930380A4E343430205833B9
:106F90002E3238322059302E3739370A4E343435B4
:106FA0002058332E3336312059302E3639310A4E9F
:106FB0003435302058332E3432362059302E35397E
:106FC000320A4E3435352058332E34353620593078
:106FD0002E3534330A4E3436302058332E34373978
:106FE0002059302E3439330A4E3436352058332E5A
:106FF0003439342059302E3437320A4E3437302069
:1070000058332E3530352059302E3434360A4E342C
:1070100037352058332E3531382059302E3431371A
:107020000A4E3438302058332E3533302059302E24
:107030003339310A4E3438352058332E3536342022
:1070400059302E3330300A4E3439302058332E35F3
:1070500037372059302E3235330A4E3439352058DF
:10706000332E3536382059302E3231320A4E3530F3
:10707000302058332E3534342059302E3137360AEB
:107080004E3530352058332E3534312059302E319D
:1070900034360A4E3531302058332E3535332059A9
:1070A000302E3131390A4E3531352058332E3537AF
:1070B000362059302E3130360A4E35323020583392
:1070C0002E3539372059302E3130320A4E3532358F
:1070D0002058332E3631382059302E3130390A4E6F
:1070E0003533302058332E3633392059302E313253
:1070F000390A4E3533352058332E36353020593045
:107100002E3135390A4E3534302058332E36363349
:107110002059302E3137380A4E3534352058332E29
:107120003637382059302E3139320A4E3535302035
:1071300058332E3639392059302E3139370A4E35E9
:1071400035352058332E3732332059302E313936E9
:107150000A4E3536302058332E3736342059302EEB
:107160003137390A4E3536352058332E38303520F0
:1071700059302E3136350A4E3537302058332E38B7
:1071800038342059302E3135390A4E3537352058AC
:10719000332E3934392059302E3136350A4E3538B0
:1071A000302058332E3936362059302E3137350AB3
:1071B0004E3538352058332E3937382059302E3156
:1071C00039340A4E3539302058332E393738205962
:1071D000302E3232330A4E3539352058332E393677
:1071E000302059302E3234350A4E36303020583364
:1071F0002E3833342059302E3331310A4E36303563
:107200002058332E3736322059302E3334350A4E3B
:107210003631302058332E3732362059302E33381D
:10722000390A4E3631352058332E37303320593015
:107230002E3435380A4E3632302058332E36383216
:107240002059302E3533300A4E3632352058332E01
:107250003637392059302E3533340A4E3633302004
:1072600058332E3632362059302E3638310A4E36C3
:1072700033352058332E3536382059302E383238B1
:107280000A4E3634302058332E3434342059312EBF
:107290003038300A4E3634352058332E34303520CD
:1072A00059312E3136370A4E3635302058332E3488
:1072B00030342059312E3136370A4E363535205884
:1072C000332E3338372059312E3230380A4E363685
:1072D000302058332E3338342059312E3230380A8A
:1072E0004E3636352058332E3336352059312E322E
:1072F00036350A4E3637302058332E33353520593F
:10730000312E3238350A4E3637352058332E333445
:10731000382059312E3330380A4E36383020583321
:107320002E3333332059312E3335300A4E3638352B
:107330002058332E3332312059312E3339310A4E11
:107340003639302058332E3331312059312E3432F2
:10735000380A4E3639352058332E333339205931D7
:107360002E3432330A4E3730302058332E343430F6
:107370002059312E3430360A4E3730352058332ECE
:107380003531302059312E3430380A4E37313020E3
:1073900058332E3538352059312E3432310A4E3794
:1073A00031352058332E3631312059312E3433398E
:1073B0000A4E3732302058332E3631312059312E93
:1073C0003434310A4E3732352058332E3631352099
:1073D00059312E3434310A4E3733302058332E365B
:1073E00033362059312E3438380A4E373335205849
:1073F000332E3633342059312E3531370A4E373457
:10740000302058332E3632322059312E3534330A5B
:107410004E3734352058332E3630352059312E35FD
:1074200036330A4E3735302058332E35373620590B
:10743000312E3537350A4E3735352058332E353411
:10744000342059312E3538310A4E373630205833F2
:107450002E3437392059312E3539320A4E373635E8
:107460002058332E3435312059312E3539380A4ED3
:107470003737302058332E3338372059312E3632B3
:10748000360A4E3737352058332E333930205931AC
:107490002E3633360A4E3738302058332E353332B5
:1074A0002059312E3630320A4E3738352058332E97
:1074B0003630312059312E3539370A4E37393020A0
:1074C00058332E3636382059312E3539380A4E3752
:1074D00039352058332E3738322059312E36313253
:1074E0000A4E3830302058332E3739342059312E57
:1074F0003631380A4E3830352058332E3836382059
:1075000059312E3633360A4E3831302058332E3921
:1075100031382059312E3635350A4E38313520581C
:10752000332E3934352059312E3636370A4E38321B
:10753000302058332E3936342059312E3638350A1A
:107540004E3832352058332E3936372059312E36C1
:1075500038350A4E3833302058332E3937342059D5
:10756000312E3639390A4E3833352058332E3938D2
:10757000342059312E3732350A4E383430205833C2
:107580002E3938342059312E3735380A4E383435B3
:107590002058332E3937302059312E3739300A4EA2
:1075A0003835302058332E3934352059312E383182
:1075B000370A4E3835352058332E39313820593175
:1075C0002E3832360A4E3836302058332E3839317C
:1075D0002059312E3832370A4E3836352058332E5E
:1075E0003834322059312E3830390A4E383730206D
:1075F00058332E3739382059312E3738340A4E381F
:1076000037352058332E3734362059312E3737321C
:107610000A4E3838302058332E3639382059312E1A
:107620003736340A4E3838352058332E3633352025
:1076300059312E3736360A4E3839302058332E35E8
:1076400035332059312E3738350A4E3839352058E0
:10765000332E3437382059312E3832300A4E3930F3
:10766000302058332E3430392059312E3836340AF0
:107670004E3930352058332E3334352059312E3998
:1076800031380A4E3931302058332E3236342059B1
:10769000322E3032330A4E3931352058332E3234BF
:1076A000382059322E3035310A4E39323020583395
:1076B0002E3234302059322E3038310A4E3932359C
:1076C0002058332E3331362059322E3038360A4E78
:1076D0003933302058332E3339302059322E31305F
:1076E000340A4E3933352058332E34313420593250
:1076F0002E3132310A4E3934302058332E34333162
:107700002059322E3135330A4E3934352058332E34
:107710003433332059322E3138300A4E3935302047
:1077200058332E3432372059322E3230350A4E3902
:1077300035352058332E3431332059322E323234FD
:107740000A4E3936302058332E3339322059322EF2
:107750003234320A4E3936352058332E3333352001
:1077600059322E3234340A4E3937302058332E32C3
:1077700037382059322E3233360A4E3937352058B1
:10778000332E3235362059322E3234320A4E3938C1
:10779000302058332E3233392059322E3235310AC7
:1077A0004E3938352058332E3231312059322E326D
:1077B00038300A4E3939302058332E313734205979
:1077C000322E3335360A4E3939352058332E31357D
:1077D000392059322E3339370A4E31303030205863
:1077E000332E3135302059322E3433380A4E313071
:1077F00030352058332E3134302059322E34383140
:107800000A4E313031302058332E31333220593244
:107810002E3531300A4E313031352058332E31314A
:10782000382059322E3534330A4E31303230205818
:10783000332E3039392059322E3537360A4E313011
:1078400032352058332E3035312059322E363331EF
:107850000A4E313033302058332E303033205932F5
:107860002E3636360A4E313033352058322E3935E1
:10787000372059322E3638350A4E313034302058C0
:10788000322E3930372059322E3639390A4E3130BE
:1078900034352058322E3836302059322E37313197
:1078A0000A4E313035302058322E38313920593295
:1078B0002E3732370A4E313035352058322E373692
:1078C000382059322E3734350A4E31303630205870
:1078D000322E3731362059322E3735370A4E313075
:1078E00036352058322E3637352059322E37353737
:1078F0000A4E313037302058322E35373920593240
:107900002E3733310A4E313037352058322E353745
:10791000302059322E3732330A4E31303830205829
:10792000322E3535392059322E3732300A4E313029
:1079300038352058322E3533302059322E373031F9
:107940000A4E313039302058322E353031205932FC
:107950002E3639330A4E313039352058322E3437ED
:10796000312059322E3638330A4E313130302058DA
:10797000322E3434332059322E3636380A4E3131D5
:1079800030352058322E3339362059322E363334A2
:107990000A4E313131302058322E333534205932AD
:1079A0002E3539310A4E313131352058322E3335AA
:1079B000322059322E3539310A4E31313230205889
:1079C000322E3332352059322E3534330A4E31318E
:1079D00032352058322E3331352059322E3532315E
:1079E0000A4E313133302058322E3330372059325D
:1079F0002E3439380A4E313133352058322E32394F
:107A0000362059322E3436340A4E31313430205833
:107A1000322E3239332059322E3432370A4E313138
:107A200034352058322E3239352059322E333636FD
:107A30000A4E313135302058322E3332312059320E
:107A40002E3330330A4E313135352058322E33350E
:107A5000382059322E3234370A4E313136302058E0
:107A6000322E3431392059322E3230330A4E3131F0
:107A700036352058322E3431392059322E313739AB
:107A80000A4E313137302058322E343035205932B9
:107A90002E3135380A4E313137352058322E3336B3
:107AA000322059322E3132330A4E3131383020589B
:107AB000322E3335342059322E3130340A4E3131A2
:107AC00038352058322E3335342059322E30393162
:107AD0000A4E313139302058322E33383020593265
:107AE0002E3036350A4E313139352058322E343168
:107AF000302059322E3035310A4E31323030205854
:107B0000322E3431302059322E3034370A4E313251
:107B100030352058322E3430352059322E3032381C
:107B20000A4E313231302058322E3430382059321A
:107B30002E3031300A4E313231352058322E343128
:107B4000362059312E3939350A4E313232302058EB
:107B5000322E3433332059312E3938320A4E3132F5
:107B600032352058322E3433382059312E393633BD
:107B70000A4E313233302058322E343437205931C6
:107B80002E3934380A4E313233352058322E3436BD
:107B9000312059312E3933380A4E313234302058A1
:107BA000322E3438302059312E3933310A4E3132A9
:107BB00034352058322E3437382059312E3839395F
:107BC0000A4E313235302058322E34383720593170
:107BD0002E3837350A4E313235352058322E353071
:107BE000342059312E3835340A4E3132363020584F
:107BF000322E3532372059312E3834380A4E313250
:107C000036352058322E3534392059312E38343912
:107C10000A4E313237302058322E3537372059311D
:107C20002E3836310A4E313237352058322E363022
:107C3000342059312E3836360A4E313238302058F9
:107C4000322E3633312059312E3835340A4E313206
:107C500038352058322E3634302059312E383237CC
:107C60000A4E313239302058322E363430205931D4
:107C70002E3739320A4E313239352058322E3632CB
:107C8000392059312E3735390A4E313330302058AA
:107C9000322E3631322059312E3732370A4E3133B7
:107CA00030352058322E3537362059312E3639347A
:107CB0000A4E313331302058322E35333620593187
:107CC0002E3636320A4E313331352058322E343783
:107CD000302059312E3631360A4E31333230205869
:107CE000322E3334352059312E3535310A4E313369
:107CF00032352058322E3330372059312E3532313B
:107D00000A4E313333302058322E3236302059313A
:107D10002E3438320A4E313333352058322E323435
:107D2000332059312E3437370A4E3133343020580E
:107D3000322E3232382059312E3436390A4E313310
:107D400034352058322E3232322059312E343438E4
:107D50000A4E313335302058322E323238205931E4
:107D60002E3432350A4E313335352058322E3235E5
:107D7000342059312E3430350A4E313336302058C4
:107D8000322E3236382059312E3337330A4E3133C2
:107D900036352058322E3237392059312E3334328D
:107DA0000A4E313337302058322E33303820593193
:107DB0002E3238370A4E313337352058322E33348D
:107DC000302059312E3235340A4E31333830205874
:107DD000322E3430372059312E3230310A4E313381
:107DE00038352058322E3434312059312E31353641
:107DF0000A4E313339302058322E3435342059313F
:107E00002E3133310A4E313339352058322E343643
:107E1000302059312E3130360A4E3134303020582E
:107E2000322E3436342059312E3130320A4E31342C
:107E300030352058322E3437312059312E303336F8
:107E40000A4E313431302058322E343636205930F3
:107E50002E3937310A4E313431352058322E3435EF
:107E6000312059302E3839370A4E313432302058CB
:107E7000322E3431352059302E3739310A4E3134D3
:107E800032352058322E3430332059302E373637A1
:107E90000A4E313433302058322E3338382059309E
:107EA0002E3736350A4E313433352058322E3330A2
:107EB000362059302E3834310A4E3134343020587F
:107EC000322E3232322059302E3931310A4E31348D
:107ED00034352058322E3131342059302E3939354D
:107EE0000A4E313435302058322E3030322059315C
:107EF0002E3037360A4E313435352058312E393050
:107F0000352059312E3133390A4E3134363020582C
:107F1000312E3735342059312E3232330A4E313436
:107F200036352058312E3633372059312E323738F6
:107F30000A4E313437302058312E353832205931FD
:107F40002E3330310A4E313437352058312E353505
:107F5000382059312E3331350A4E313438302058DB
:107F6000312E3436302059312E3335320A4E3134E9
:107F700038352058312E3339392059312E333630A7
:107F80000A4E313439302058312E333338205931AC
:107F90002E3335340A4E313439352058312E3238AB
:107FA000372059312E3332390A4E3135303020588E
:107FB000312E3234382059312E3239340A4E31358F
:107FC00030352058312E3231372059312E32353468
:107FD0000A4E313531302058312E3231342059316A
:107FE0002E3235320A4E313531352058312E313767
:107FF000322059312E3139350A4E31353230205840
:10800000312E3132382059312E3133390A4E313543
:1080100032352058312E3131302059312E3131371F
:108020000A4E313533302058302E3935382059300A
:108030002E3934310A4E313533352058302E383907
:10804000312059302E3837330A4E313534302058EC
:10805000302E3832352059302E3830380A4E3135EE
:1080600034352058302E3735352059302E373437B7
:108070000A4E313535302058302E363139205930BE
:108080002E3633330A4E313535352058302E3437BD
:10809000372059302E3532360A4E31353630205899
:1080A000302E3437372059302E3532340A4E3135A0
:1080B00036352058302E3431312059302E34373671
:1080C0000A4E313537302058302E33333120593075
:1080D0002E3435340A4E313537352058302E32376C
:1080E000382059302E3432370A4E31353830205846
:1080F000302E3233312059302E3339370A4E313554
:1081000038352058302E3138332059302E33373916
:108110000A4E313539302058302E31333520593020
:108120002E3336350A4E313539352058302E30371A
:10813000362059302E3334310A4E3136303520470F
:108140003030204633302E300A4E31363130204D1B
:108150003035200A4E3136313520473930205830FD
:10816000205930205A300A4E31363135204D3330C7
:108170000A28456E64206F6620434E432050726F7C
:108180006772616D2900284D53472A2A2A2A204DFB
:108190006963726F737465702054657374205B76C5
:1081A000315D202A2A2A2A290A47303020473137D0
:1081B0002047323120473430204734392047383087
:1081C000204739300A6730783079307A300A7B229C
:1081D000316D69223A317D0A7B22326D69223A3152
:1081E0007D0A7B22336D69223A317D0A7B22346D10
:1081F00069223A317D0A6730207831300A7B22319A
:108200006D69223A327D0A78300A7B22316D69220B
:108210003A347D0A7831300A7B22316D69223A384E
:108220007D0A78300A6730207931300A7B22326D3E
:1082300069223A327D0A79300A7B22326D69223A0C
:10824000347D0A7931300A7B22326D69223A387DD9
:108250000A79300A6730207A31300A7B22336D691F
:10826000223A327D0A7A300A7B22336D69223A340F
:108270007D0A7A31300A7B22336D69223A387D0AD1
:108280007A300A6730206131300A7B22346D6922EE
:108290003A327D0A61300A7B22346D69223A347D9C
:1082A0000A6131300A7B22346D69223A387D0A61D5
:1082B000300A6D3200284D53472A2A2A2A20436F5C
:1082C0006F7264696E617465206F6666736574733E
:1082D0002074657374205B76315D202A2A2A2A294E
:1082E0000A67303067313767323167343067343985
:1082F0006738306739300A6735340A673932783081
:1083000079307A300A663630300A284D53472A2AA7
:108310002A2A207465737420473932206F66667389
:108320006574732A2A2A2A290A286D73675374658B
:108330007020313A204D6F76652066726F6D203067
:108340002C3020746F2033302C30206D6D20696EFE
:1083500020706F736974697665205820646972654E
:108360006374696F6E290A286D7367537465702092
:10837000323A205265736574206F726967696E20A6
:10838000746F20302E30207573696E672047393244
:10839000290A286D73675374657020333A204D6F36
:1083A000766520746F2032302C302E2053686F7524
:1083B0006C64206D6F7665203230206D6D20696EA3
:1083C00020706F73697469766520582064697265DE
:1083D0006374696F6E20616E642073746174757369
:1083E000207265706F72742073686F756C6420738F
:1083F000746172742066726F6D20302C30290A28E7
:108400006D73675374657020343A204D6F76652024
:10841000746F20302E3020202053686F756C6420DC
:108420006D6F7665203230206D6D20696E206E652F
:108430006761746976652058206469726563746940
:108440006F6E20616E642073746174757320726541
:10845000706F72742073686F756C642073746172CE
:10846000742066726F6D2032302C30290A673178A3
:1084700033300A67393278300A67317832300A6728
:1084800031783079300A2473720A67393278300AC9
:10849000673470302E350A284D53472A2A2A2A205D
:1084A0007465737420473535206F66667365747321
:1084B0002A2A2A2A290A286D736753746570203185
:1084C0003A2053657420436F6F7264696E617465FE
:1084D0002073797374656D2032205B6735355D20BC
:1084E000746F206F6666736574206F662035302C5C
:1084F0003530290A286D73675374657020323A202D
:1085000053656C6563742047353520636F6F726403
:10851000696E6174652073797374656D290A286DBD
:1085200073675374657020333A204D6F76652074FD
:108530006F20302C302E20486561642073686F7581
:108540006C64206D6F766520646961676F6E616C25
:108550006C7920696E202B5820616E64202B592085
:10856000616E6420737461747573207265706F72CC
:10857000742073686F756C64207374617274206604
:10858000726F6D20302C30290A6731304C327032D6
:108590007835307935300A6735350A673078307983
:1085A000300A673470302E350A284D53472A2A2A5C
:1085B0002A207465737420473533206162736F6CB1
:1085C000757465206F7665727269646573202A2AF6
:1085D0002A2A290A286D73675374657020313A205E
:1085E00052756E20612073717561726520696E200D
:1085F0004735352073797374656D290A286D736763
:108600005374657020323A2052756E206120737168
:108610007561726520772F473533206F76657272EA
:10862000696465290A6730783079300A67307832B2
:108630003079300A67307832307932300A673078F2
:10864000307932300A6730783079300A67347030E8
:108650002E350A6735336730783079300A6735331D
:10866000673078323079300A6735336730783230A6
:108670007932300A673533673078307932300A67BB
:1086800035336730783079300A6730783079300A9E
:10869000673470302E350A284D53472A2A2A2A205B
:1086A000746573742052657475726E20746F2068DF
:1086B0006F6D65202A2A2A2A290A286D7367537448
:1086C000657020313A2052657475726E20746F2087
:1086D000686F6D65207573696E6720473238290AA7
:1086E000286D73675374657020323A205265736544
:1086F0007420746F2047353420636F6F7264207369
:10870000797374656D290A6732380A6735340A6DE2
:10871000333000284D53472A2A2A2A20546573747F
:10872000206163637572616379206F6620736C6F7B
:1087300077206D6F766573205B76315D202A2A2A5B
:108740002A290A6735350A6730783079300A673464
:1087500070302E350A673470302E350A6731783123
:10876000306632320A6735340A6730783079300A39
:108770006D333000284D53472A2A2A2A2054657326
:108780007420766572792073686F7274206D6F76CD
:108790006573205B76315D202A2A2A2A290A6730F0
:1087A000783079300A673470302E350A6731783086
:1087B0002E3166313030300A78300A78302E310A66
:1087C00078300A78302E310A78300A78302E310A23
:1087D00078300A78302E310A78300A78302E310A13
:1087E00078300A78302E310A78300A78302E310A03
:1087F00078300A78302E310A78300A78302E310AF3
:1088000078300A78302E310A78300A78302E310AE2
:1088100078300A78302E310A78300A78302E310AD2
:1088200078300A78302E310A673470302E350A7865
:10883000300A78302E30310A78300A78302E3031D4
:108840000A78300A78302E30310A78300A78302EA3
:1088500030310A78300A78302E30310A78300A7890
:10886000302E30310A78300A78302E30310A7830A4
:108870000A78302E30310A78300A78302E30310ABA
:1088800078300A78302E30310A78300A78302E303D
:10889000310A78300A78302E30310A78300A783050
:1088A0002E30310A78300A78302E30310A6730782D
:1088B0003079300A6D3200284D53472A2A2A2A205F
:1088C000526F746172792041786973204D6F7469B9
:1088D0006F6E2054657374205B76315D202A2A2ADE
:1088E0002A290A6730306731376732316734306799
:1088F00034396738306739300A6730783079307A00
:10890000306130623063300A6735350A673078305D
:1089100079300A6633363030300A673061333630AA
:108920000A623336300A633336300A61300A623005
:108930000A63300A673161313434300A62313434C9
:10894000300A63313434300A61300A62300A6330ED
:108950000A67316131343430623732306333363054
:108960000A783079307A306130623063300A6731AA
:1089700078363061313434306237323063333630F8
:108980000A783079307A306130623063300A67318A
:108990007836307935306131343430623732306393
:1089A0003336300A783079307A3061306230633073
:1089B0000A67317836307935307832356131343480
:1089C0003062373230633336300A783079307A307B
:1089D0006130623063300A6735340A673078307945
:1089E000300A6D333000284D53472A2A2A2A20495D
:1089F0006E76657273652054696D65204D6F74697C
:108A00006F6E2054657374205B76315D202A2A2AAC
:108A10002A290A6730306731376732316734306767
:108A200034396738306739300A6735350A67307846
:108A30003079300A6739330A66302E30310A6731AF
:108A40007831300A7931300A7A31300A6131300AAE
:108A500078300A79300A7A300A61300A6731783121
:108A6000307931307A2D31306131300A67307830E9
:108A700079307A3061300A66302E310A67327831C7
:108A800030792D31307A2D32306931300A673078C3
:108A90003079307A300A6733783130792D31307A55
:108AA0002D32306931300A6730783079307A300AC7
:108AB000673278323079307A2D32306931300A6756
:108AC00030783079307A300A6733783230793069EB
:108AD00031300A6730783079307A300A673278304E
:108AE00079307A2D33306931300A67337830793014
:108AF0007A306931300A6730783079307A300A67F5
:108B0000327830793069323020284357203336307C
:108B10002064656772656573290A67337830793038
:108B2000693230202843435720333630206465674C
:108B300072656573290A6739340A6735340A673004
:108B4000783079300A6D3330007B226763223A2215
:108B500067303067313767323167343067343967AF
:108B60003830673930227D0A7B226763223A2267D8
:108B70003535227D0A7B226763223A2267307830BE
:108B80007930227D0A7B226763223A2266353030B3
:108B9000227D0A7B226763223A22284D5347737154
:108BA000756172657329227D0A7B226763223A22EE
:108BB0006730783230227D0A7B226763223A22793D
:108BC0003230227D0A7B226763223A227830227D6E
:108BD0000A7B226763223A227930227D0A7B226750
:108BE00063223A226731783130227D0A7B22676323
:108BF000223A22793130227D0A7B226763223A228F
:108C00007830227D0A7B226763223A227930227DE6
:108C10000A7B226763223A22284D534763697263B5
:108C20006C657329227D0A7B226763223A226732B0
:108C3000783130792D3130693130227D0A7B2267DD
:108C400063223A22673078307930227D0A7B2267AE
:108C500063223A226733783130792D3130693130EF
:108C6000227D0A7B226763223A226730783079308E
:108C7000227D0A7B226763223A226732783230797A
:108C800030693130227D0A7B226763223A226730C5
:108C900078307930227D0A7B226763223A2267335B
:108CA0007832307930693130227D0A7B2267632245
:108CB0003A22673078307930227D0A7B226763223E
:108CC0003A22673278307930693130227D0A7B224E
:108CD0006763223A22673378307930693130227DF8
:108CE0000A7B226763223A22673534227D0A7B227F
:108CF0006763223A22673078307930227D0A7B22FE
:108D00006763223A226D3330227D00284D53472A73
:108D10002A2A2A204D636F6465732074657374205A
:108D20005B76315D202A2A2A2A290A6735350A67A7
:108D300030783079300A6D330A673470310A6D3516
:108D40000A673470310A6D340A673470310A6D3540
:108D50000A673470310A6D370A673470310A6D3929
:108D60000A673470310A6D380A673470310A6D3918
:108D70000A663530300A67307832300A7932300A84
:108D80006D330A78300A6D340A79300A6D350A6716
:108D9000317831300A6D370A7931300A6D380A7806
:108DA000300A6D390A79300A6732783130792D31DD
:108DB000306931300A6D330A6730783079300A6DA6
:108DC000340A6733783130792D31306931300A6DAA
:108DD000350A6730783079300A6D370A6732783271
:108DE0003079306931300A6D380A6730783079303F
:108DF0000A6D390A673378323079306931300A6761
:108E000030783079300A6732783079306931300A19
:108E10006733783079306931300A6735340A673022
:108E2000783079300A6D333000284D53472A2A2A8A
:108E30002A2046656564686F6C64205465737420ED
:108E40005B76315D202A2A2A2A290A284D53472A8F
:108E50002A2A2A204D616E75616C6C7920656E74CA
:108E60006572202120616E64207E20647572696EB7
:108E700067206D6F76656D656E7420746F20746504
:108E80007374202A2A2A2A290A6735350A67307816
:108E90003079300A673470330A67303067313767AA
:108EA00032316734306734396738306739300A66B1
:108EB0003630300A6730783130307637362E3736F4
:108EC000350A783079300A6735340A673078307976
:108ED000300A6D333000284D53472A2A2A2A20446D
:108EE00077656C6C2054657374205B76315D202A45
:108EF0002A2A2A290A6730306731376732316739C1
:108F0000300A6735350A6730783079300A6635308F
:108F1000300A67307831300A673470310A67307848
:108F200032300A673470310A67307831300A67347A
:108F300070310A67307830300A673470310A793519
:108F40000A6735340A6730783079300A6D330A673A
:108F50003470310A67307831307931300A6D350A32
:108F6000673470310A67307832307932300A6D34C4
:108F70000A673470310A67307833307933300A6DDC
:108F8000380A673470310A67307834307934300AFF
:108F90006D390A673470310A673078353079353089
:108FA0000A6730783079300A6D3330002F286D73BE
:108FB000672A2A2A2A204172632054657374205B31
:108FC00076315D202A2A2A2A290A4E31206730303C
:108FD0006731376732316734306734396738306723
:108FE00039300A4E3130206730783079300A4E32CD
:108FF0003020663530300A4E3330206732783130D9
:10900000792D3130693130202843572032373020D4
:1090100064656772656573290A4E3430206730785D
:109020003079300A4E3530206733783130792D3140
:109030003069313020284343572039302064656738
:1090400072656573290A4E36302067307830793082
:109050000A4E38302067327832307930693130202A
:10906000284357203138302064656772656573295D
:109070000A4E3730206730783079300A4E38302049
:1090800067337832307930693130202843435720B4
:109090003138302064656772656573290A4E39304E
:1090A000206730783079300A4E39392046313230F5
:1090B000300A4E31303020673278307930693230C2
:1090C0002028435720333630206465677265657306
:1090D000290A4E31313020673278307930693230A8
:1090E000202843572033363020616761696E290A92
:1090F0004E313230206637303020284368616E6749
:109100006520666565642072617465207768696CA6
:109110006520696E204732206D6F74696F6E206D17
:109120006F6465290A4E31333020673278307930E8
:109130006932302028435720333630203372642080
:1091400074696D65290A4E31343020673278307980
:109150003069323020284357203336302034746849
:109160002074696D65290A4E3135302066353030FE
:109170000A4E313630206733783079307A343069AE
:1091800032302028434357203336302064656772DD
:109190006565732077697468206C696E65617220FB
:1091A00074726176656C290A4E31373020673378E6
:1091B0003079307A306932302028434357203336B3
:1091C0003020616761696E290A4E31383020663778
:1091D000303020286D73672A2A2A2A4368616E6717
:1091E0006520666565642072617465207768696CC6
:1091F0006520696E204733206D6F74696F6E206D36
:109200006F64652A2A2A2A290A4E313930206733A9
:109210007830793069323020284343572033363054
:10922000203372642074696D65290A4E3230302013
:109230006733783079306932302028434357203300
:109240003630203474682074696D65290A4E3231D5
:109250003020286D73672A2A2A2A4731382045761C
:10926000616C20746573742A2A2A2A290A4E3232C4
:1092700030204731205833302E373037205A3530A0
:109280002E37323720463530300A4E3233302047C1
:10929000313820473032205836372E373338205A6D
:1092A00032332E3631372052323520463235300AAD
:1092B0004E323430206738300A4E32353020673035
:1092C000783079307A300A4E323630206D333000C3
:1092D000284D53472A2A2A2A2053717561726573D3
:1092E000204D6F74696F6E2054657374205B763106
:1092F0005D202A2A2A2A290A6730306731376732E7
:10930000316734306734396738306739300A67304D
:10931000783079300A67307832302028747261767C
:109320006572736520612032306D6D2073717561D7
:10933000726520696E205820616E642059290A796F
:1093400032300A78300A79300A6731783130663540
:10935000303020286472617720612031306D6D20BB
:1093600073717561726520696E205820616E64208A
:10937000592061742046353030290A7931300A7815
:10938000300A79300A67307A323020287472617678
:109390006572736520612032306D6D207371756167
:1093A000726520696E205820616E64205A290A78FF
:1093B00032300A7A300A78300A67317832307932BE
:1093C000307A323066353030202866656564206139
:1093D0002032306D6D20646961676F6E616C206949
:1093E0006E20582C205920616E64205A290A78304A
:1093F00079307A300A7834307934307A3430202831
:10940000747261766572736520612034306D6D20F1
:109410006375626520696E20582C205920616E6446
:10942000205A290A78343079307A300A7830793401
:10943000307A34300A7834307934307A300A7830FF
:1094400079307A34300A78307934307A300A7834A6
:109450003079307A34300A783079307A300A6738A7
:10946000300A6730783079300A673078310A6730EF
:1094700078300A6D333000284D53472A2A2A2A2093
:10948000486F6D696E672054657374205B76315D3B
:10949000202A2A2A2A290A6732382E32783079304F
:1094A0007A300A6D333000284D53472A2A2A2A2061
:1094B000536D6F6B652054657374205B76315D204E
:1094C0002A2A2A2A290A47303020473137204732B2
:1094D000312047343020473439204738302047394D
:1094E000300A6D33673470310A6D35673470310A74
:1094F0006D34673470310A6D33673470310A6D35FD
:10950000673470310A6D37673470310A6D396734EA
:1095100070310A6D38673470310A6D390A673078F6
:109520003079307A300A673030207832300A78303B
:109530000A7932300A79300A7A32300A7A300A618E
:1095400032300A61300A47303020783230207932A8
:1095500030207A3230206132300A47303020783083
:10956000207930207A302061300A4730312066334C
:1095700030207832207932207A322061320A7830F5
:10958000207930207A302061300A673078310A67DC
:109590003078300A6D32002C000A00257300256CEB
:1095A000750025312E3066002573002C000A002539
:1095B000733A25730025733A256C750025733A2597
:1095C000312E30660025733A2573005B74765D207A
:1095D000207465787420766572626F73697479257A
:1095E000313564205B303D73696C656E742C313DA0
:1095F000766572626F73655D0A0025660A00256CE8
:10960000750A0025640A0025730A0074696E79677B
:10961000205B25735D206572723A2025733A202500
:1096200073200074696E7967205B25735D206F6B12
:109630003E2000456E64206F6620636F6D6D616E25
:10964000642066696C650A00FCCB6DCA69CC8ACC63
:10965000E9CCB2CAC1CF6DCA55D0C1D0EFCEB2CA23
:109660000000400640061040B800B8C1CF6DCA5592
:10967000D0C1D0EFCEB2CA0000400620060840B8E4
:1096800000B837D26DCA58D1D3D182D321D1A00826
:109690004006050609010837D26DCA58D1D3D1FB5F
:1096A000CCB2CAB00840060540B0308000000000CF
:1096B00000F0E0D0C0100100CF673322211F1B1340
:1096C00001016E616E00696E66004E414E494E4961
:1096D0005459494E46CDCCCC3D0AD7233C17B7D17F
:1096E0003877CC2B329595E6241FB14F0A00002025
:1096F000410000C84200401C4620BCBE4CCA1B0EA4
:109700005AAEC59D7400407A10F35A00A0724E18EC
:10971000090010A5D4E80000E87648170000E40B23
:1097200054020000CA9A3B000000E1F505000080E9
:10973000969800000040420F000000A08601000043
:1097400000102700000000E8030000000064000093
:109750000000000A00000000000100000000002CD2
:1097600076D888DC674F0823DFC1DFAE59E1B1B797
:1097700096E5E3E453C63AE651997696E8E6C28464
:1097800026EB898C9B62ED407C6FFCEFBC9C9F407C
:10979000F2BAA56FA5F490055A2AF75C936B6CF9A1
:1097A000676DC11BFCE0E40D47FEF520E6B500D077
:1097B000ED902E0300943577050080841E0800008C
:1097C000204E0A000000C80C333333330F986E125A
:1097D000831141EF8D2114893BE65516CFFEE6DB60
:1097E00018D1844B381BF77C1D901DA4BBE42420AA
:1097F0003284725E228100C9F124ECA1E53D27008C
:1098000011241FBECFEFCDBFDFE5DEBF00E00CBFF0
:1098100013E2A0E0B0E2EEE8FDEC01E00BBF02C015
:1098200007900D92A239B107D9F72AE5A2E9B3E270
:1098300001C01D92AB33B207E1F70E940E840C9475
:10984000C5E60C940000FC016081718182819381E6
:109850000E9496D86093D4320895FC016081718192
:10986000828193810E9496D86093D3320895AF92FB
:10987000BF92CF92DF92EF92FF920F931F93CF93FD
:10988000DF937B018C0188E5C82E82E3D82EE601A8
:10989000AA24A394BC2EBC18F70161917191819107
:1098A00091917F012CEA35EC47E257E30E9425DADB
:1098B00018164CF4F80140815181628173818B2D1F
:1098C0000E947C85A8820C5F1F4F2196F2E3CE3563
:1098D000DF0701F7DF91CF911F910F91FF90EF907C
:1098E000DF90CF90BF90AF900C948785FC01608192
:1098F0007181828193810E9496D86093D5326130C4
:1099000019F481E00E94837B81E00C94A47BCF93C7
:10991000DF93CDB7DEB76897CDBFDEBFFC016081B6
:109920007181828193810E9496D86093D63281E0C2
:10993000613019F40E94837B0CC00E94A47BCE018D
:10994000019628E1FC0111922A95E9F7BC010E94D9
:10995000764C6896CDBFDEBFDF91CF9108950F930F
:109960001F93CF93DF93CDB7DEB72D97CDBFDEBF6B
:1099700027E0E2EDF0E28E010F5F1F4FD80101906A
:109980000D922A95E1F7BC01660F771F680F791FCA
:10999000660F771F660F771F660F771F61507A4E2D
:1099A00045E050E0CE0108960E9435E4688570E0FD
:1099B000C8010E9463E4009739F46B8570E0C80128
:1099C0000E9463E4009711F0801B01C08FEF2D9679
:1099D000CDBFDEBFDF91CF911F910F910895EF9220
:1099E000FF920F931F93CF93DF938C01F62EE72EF8
:1099F000EC012D96FC0161857285838594850E941A
:109A000096D81F926F93DF93CF930F5E1F4F1F93D4
:109A10000F93DF93CF93EF92FF92E7E3FAE5818113
:109A20008F9380818F930E94FCE4EDB7FEB73C9644
:109A3000EDBFFEBFDF91CF911F910F91FF90EF908F
:109A400008950F931F93CF93DF93EC01162F072FE9
:109A50008C819D810E94AF4C83305CF58F3FA1F5D6
:109A600028C09E01235F3F4F9F938F938C858F93D8
:109A70008B858F938A858F9389858F933F932F93BF
:109A80006196DF93CF933F932F930F931F93809112
:109A9000385A8F938091375A8F930E94FCE48DB788
:109AA0009EB740968DBF9EBFDF91CF911F910F91C2
:109AB0000895E7E7F4E1659174914FE450E081E5A2
:109AC0009DE30E9435E4CDCFE091CE32F0E0EE0F81
:109AD000FF1FED58FB4E659174914FE450E081E516
:109AE0009DE30E9435E4BDCF0F931F93CF93DF9387
:109AF000EC01162F072F8C819D810E94AF4C833083
:109B00007CF58F3FC1F52CC0AE014F5E5F4F9E01CB
:109B1000235F3F4F9F938F938C858F938B858F937C
:109B20008A858F9389858F935F934F933F932F936C
:109B30005F934F933F932F930F931F938091385AC6
:109B40008F938091375A8F930E94FCE48DB79EB714
:109B500042968DBF9EBFDF91CF911F910F910895C7
:109B6000E7E7F4E1659174914FE450E081E59DE30E
:109B70000E9435E4C9CFE091CE32F0E0EE0FFF1F36
:109B8000ED58FB4E659174914FE450E081E59DE303
:109B90000E9435E4B9CFDF92EF92FF920F931F93AB
:109BA000CF93DF93CDB7DEB72897CDBFDEBF8B0154
:109BB000E42ED52E37E0E9EDF0E2DE0111960190BA
:109BC0000D923A95E1F728870E94AF4CF82E288530
:109BD00082E08F1518F0E22FF0E002C0E2E0F0E042
:109BE000EE0FFF1FED58FB4E659174914FE450E06E
:109BF00081E59DE30E9435E49F938F93F801838173
:109C00008F9382818F9381818F9380818F93E1E005
:109C1000F0E0EC0FFD1FEF0DF11D80811F928F937F
:109C2000DF92EF928091385A8F938091375A8F93B9
:109C30000E94FCE4CDBFDEBF2896CDBFDEBFDF9122
:109C4000CF911F910F91FF90EF90DF9008954F9269
:109C50005F926F927F92AF92BF92CF92DF92EF921C
:109C6000FF920F931F93CF93DF93C8E5D2E30DE1EB
:109C700011E35C018991813009F042C0F801C48090
:109C8000D580E680F7804080518062807380A30198
:109C90009201C701B6010E94B3D69F772CEA35EC3A
:109CA00047E257E30E9422D887FD2AC020E034E231
:109CB00044E759ECC701B6010E9425DA18165CF496
:109CC000F5012081318142815381C701B6010E9493
:109CD00025DA181604F120E034E244E759ECC30118
:109CE000B2010E9425DA18165CF4F5012081318159
:109CF00042815381C301B2010E9422D887FD0BC06B
:109D00000B5C1F4FF4E0AF0EB11C82E3CE35D807D9
:109D100009F0B0CF02C08CED01C080E0DF91CF919F
:109D20001F910F91FF90EF90DF90CF90BF90AF9079
:109D30007F906F905F904F90089580915432811181
:109D400005C0809153328093523229C0823031F461
:109D500087E0809352328091533221C0833031F4B6
:109D600089E0809352328091533219C0843031F4AB
:109D70008AE0809352328091533211C080915532E3
:109D8000813031F485E0809352328091533207C0A4
:109D9000823019F486E080935232809153328630BB
:109DA00019F08091523208958BE0809352320895D9
:109DB00080915332089580935532813059F018F0D4
:109DC000823041F0089583E892E38093813290934A
:109DD0008232089580E896E58093813290938232B2
:109DE0000895FC0184810895845B9F4FFC0180816C
:109DF0000895855B9F4FFC0180810895825B9F4F92
:109E0000FC0180810895815B9F4FFC018081089552
:109E1000875B9F4FFC01808108950C945B9ACD96DF
:109E2000FC0160817181828193810895FC016483CA
:109E300008958C5A9F4FFC01608308958F5B9F4F5C
:109E4000FC0140835183628373830895609383325E
:109E500070938432809385329093863287EE91E2BC
:109E60000C943666BF92CF92DF92EF92FF920F93DF
:109E70001F93CF93DF93D090D0327C0104EF12E395
:109E80008091CF3290E0EC01CC0FDD1FC80FD91FBD
:109E9000CC0FDD1FCC0FDD1FCC0FDD1FC459DF4CF5
:109EA00081E0D816A9F0B881A981CA80BB80409111
:109EB0004733413091F4F80120813181428153814F
:109EC0006B2F7A2F8C2D9B2D0E94B4D69B0109C03D
:109ED00020E030E080E090E004C02B2F3A2F8C2D62
:109EE0009B2DA901BC01F701458F568F678F70A389
:109EF000F4E0EF0EF11C0C5F1F4F249683E30C304F
:109F0000180771F6DF91CF911F910F91FF90EF909D
:109F1000DF90CF90BF900895835B9F4FFC016083DB
:109F200083E892E30C94324F4F925F926F927F924C
:109F30008F929F92AF92BF92CF92DF92EF92FF9259
:109F40000F931F93CF93DF93CDB7DEB76897CDBF45
:109F5000DEBF8C016091473370E080E090E00E94AA
:109F6000C4D82B013C01F801608171818281938109
:109F70000E9496D870E05B01AA0CBB1CA60EB71E0F
:109F8000AA0CBB1CAA0CBB1CAA0CBB1CC501845987
:109F90009F4C5C0104EF12E3FE0131964F01F50185
:109FA000C190D190E190F1905F01F80161917191C0
:109FB000819191918F01A30192010E94C7DA9B01C7
:109FC000AC01C701B6010E94B4D6F401619371934C
:109FD000819391934F01F3E30C301F0701F7CE01FA
:109FE00001960E943E9A83E892E30E94324F68965F
:109FF000CDBFDEBFDF91CF911F910F91FF90EF900A
:10A00000DF90CF90BF90AF909F908F907F906F9098
:10A010005F904F9008958358924369F4E62FF0E0E3
:10A02000EE0FFF1FEE0FFF1FE452FD4C60817181A8
:10A03000828193810895862F0C94339ACF92DF9278
:10A04000EF92FF920F931F93CF93DF93EC0182E384
:10A05000C338D80709F04AC070E0FB01EE0FFF1FBC
:10A06000EE0FFF1FE452FD4CC080D180E280F380F0
:10A070008091D032813059F18091CF3290E0FC0153
:10A08000EE0FFF1FE80FF91FEE0FFF1FE60FF71F80
:10A09000EE0FFF1FEE0FFF1FE459FF4C00811181EF
:10A0A000B281A381209147332130B1F4FB01EE0F3F
:10A0B000FF1FEE0FFF1FEC50FD4C208131814281CC
:10A0C0005381B8018B2F9A2F0E94B4D608C060E04C
:10A0D00070E080E090E003C0B8018B2F9A2F9B01C5
:10A0E000AC01C701B6010E94B3D603C0862F0E94FF
:10A0F000479AC55BDF4F2881211106C023E333E374
:10A100004BEC51E40E9429D8DF91CF911F910F9120
:10A11000FF90EF90DF90CF90089588E1E8E8F2E3B8
:10A12000ACEDB2E301900D928A95E1F78091CC32CB
:10A1300081110CC080918732813041F41092C0327D
:10A140001092C1321092C2321092C33208954F92CF
:10A150005F926F927F928F929F92AF92BF92CF92B7
:10A16000DF92EF92FF920F931F93CF93DF93CDB7C0
:10A17000DEB76997CDBFDEBF80915432811155C0E3
:10A1800080917932813009F050C00E940CCA81114F
:10A190004CC01092793294E8692E90E3792E26E330
:10A1A000822E912C8E010E5E1F4F30EEA32E30E2D8
:10A1B000B32E33C0F70181917F011F928F935F927D
:10A1C0004F92BF92AF921F930F930E94C7E5B801C1
:10A1D00080E593E20E949C638D839E83F6018191CA
:10A1E0009191A191B1916F018A879B87AC87BD87BF
:10A1F000CE0101960E94B360CDBFDEBF98EDE91697
:10A2000090E2F906B9F6E8E16E0E711CFFEF8F1AC5
:10A210009F0A8CE38816910441F0240183EDE82E17
:10A2200080E2F82E630188E7C8CF80E06996CDBF51
:10A23000DEBFDF91CF911F910F91FF90EF90DF90E4
:10A24000CF90BF90AF909F908F907F906F905F90D6
:10A250004F9008952F923F924F925F926F927F920C
:10A260008F929F92AF92BF92CF92DF92EF92FF9226
:10A270000F931F93CF93DF93CDB7DEB72997CDBF51
:10A28000DEBF4C015B014090D2325090D032209022
:10A29000CF32609047337090CE326B0188E892E302
:10A2A0008887998754E1E52E51E3F52E98E1299EA0
:10A2B000100111248401D6016D917D918D919D91A4
:10A2C0006D012CEA35EC47E257E30E9422D887FD66
:10A2D00080C0F70180818150823008F07AC041103F
:10A2E0004CC0F1E05F1609F1E885F985E20DF31D38
:10A2F000EC51F2408081898391819D83B281A38159
:10A30000E1E06E1217C0E885F985E459FF4F20811E
:10A31000318142815381BC018B2F9A2F0E94B4D688
:10A3200069837D838E839F8307C019821D821E826D
:10A330001F8202C0BE83AF8371100CC023E333E3DE
:10A340004BEC51E4D8016D917D918D919C910E94CF
:10A35000C7DA05C0F801608171818281938129810A
:10A360003D814E815F810E94B4D6A885B9856D93E9
:10A370007D938D939C9313972CC0A885B9858D915F
:10A380009D910D90BC91A02D89839A83AB83BC8352
:10A3900071100EC023E333E34BEC51E4F80160810C
:10A3A0007181828193810E94C7DA9B01AC0105C053
:10A3B000D8012D913D914D915C9169817A818B817C
:10A3C0009C810E94B4D6E885F9856083718382837D
:10A3D00093838885998504968887998795E3E90E04
:10A3E000F11C0C5F1F4FA885B985A459B24309F031
:10A3F00062CF6090CE327090D232F091D032F98339
:10A40000C090CF32209147332D838CE0A80EB11C31
:10A41000A3EBB1E3A887B98744E9E42E42E3F42E25
:10A42000B8E1CB9E600111248401F5016191719125
:10A43000819191915F012CEA35EC47E257E30E944C
:10A4400022D887FD8CC0A885B9858C91882309F412
:10A4500086C08150823030F4F801248435844684EB
:10A4600057843BC0611016C023E333E34BEC51E447
:10A47000D8011C966D917D918D919C911F970E94A2
:10A48000C7DA20E030E044EB53E40E94C7DA1B0156
:10A490002C010DC020E030E044EB53E4F80164856A
:10A4A0007585868597850E94C7DA1B012C012BEDE7
:10A4B0003FE049EC50E4A885B98591966D917D9176
:10A4C0008D919C9194970E94C7DA9B01AC01C201C7
:10A4D000B1010E9429D81B012C01711031C0B98132
:10A4E000B130E1F0F701EC0DFD1DEC51F240A0811F
:10A4F000B18192808380ED81E130A1F4F701E459CC
:10A50000FF4F2081318142815381BD01892D982DDA
:10A510000E94B4D6DB01982E892E04C0A0E0B0E0E2
:10A52000912C812CA2019101BD01892D982D0E94B1
:10A53000B4D6D7016D937D938D939C9313970FC0E1
:10A54000A2019101F70160817181828193810E9452
:10A55000B4D6D7016D937D938D939C931397E88523
:10A56000F985F596E887F987F4E0EF0EF11C0C5FAA
:10A570001F4F888599858255924309F056CF2996B9
:10A58000CDBFDEBFDF91CF911F910F91FF90EF9074
:10A59000DF90CF90BF90AF909F908F907F906F9003
:10A5A0005F904F903F902F90089580915030909100
:10A5B00051308F3E924111F08FE50895809104341F
:10A5C000909105348F3E9241B9F78091D8329091A5
:10A5D000D9328F3E924181F780914E3390914F3323
:10A5E0008F3E924149F78091D7569091D8568F3E31
:10A5F000924111F780919357909194578F3E9241D9
:10A60000D9F680E0089580915432811104C083E02E
:10A610008093533203C085E08093533280E00895E5
:10A62000CF93C82F0E9409B680E00E94AAB18C2F58
:10A630000E942CAB86E0809353328C2FCF910895EB
:10A640008093CD3280E008958093CE3280E00895EB
:10A650008093D23280E00895AF92BF92CF92DF9282
:10A66000EF92FF920F931F93CF93DF939FEF980F7B
:10A67000963008F041C0A090CE327A018B0198E16B
:10A68000899F60011124F601E05BFF4C6F01C0E07F
:10A69000D0E0BB24B394F7016191719181919191C4
:10A6A0007F012CEA35EC47E257E30E9425DA1816C1
:10A6B000E4F4A1100CC023E333E34BEC51E4F801C4
:10A6C00060817181828193810E94C7DA05C0F8019F
:10A6D0006081718182819381F601EC0FFD1F648F8F
:10A6E000758F868F978FB092793224960C5F1F4FAB
:10A6F000C831D10581F602C08EE601C080E0DF914D
:10A70000CF911F910F91FF90EF90DF90CF90BF906E
:10A71000AF900895CF93DF93CDB7DEB76897CDBFE5
:10A72000DEBF8093CF32682F70E080E090E00E941F
:10A73000C2D869837A838B839C831D821E821F8289
:10A74000188619861A861B861C861D861E861F86FD
:10A75000188A198A1A8A1B8A1C8A1D8A1E8A1F8ACD
:10A76000188EAE014F5F5F4FBA0184E99FE40E94EB
:10A77000BE8680E06896CDBFDEBFDF91CF910895A1
:10A78000CF93DF93E3E8F2E385E5DF011D928A953D
:10A79000E9F78AE5A0E5B3E3ED01982F19929A95C0
:10A7A000E9F7AAEAB3E3ED0119928A95E9F78FEE8A
:10A7B00092E1809350309093513080930434909381
:10A7C00005348093D8329093D93280934E3390934E
:10A7D0004F338093D7569093D85680939357909346
:10A7E0009457E0938132F093823280916930809364
:10A7F000CE32809167300E948A5380916830809376
:10A80000CD3280916A308093D13280916B308093C9
:10A81000D23281E08093CC328093483394E090939D
:10A82000873210927A3210927B3210927C3280936F
:10A830005332809352320E9448B0DF91CF910C94F2
:10A840000088CF92DF92EF92FF92CF93C82F6A01D8
:10A850007B01E82FF0E0DF01AA0FBB1FAA0FBB1F8F
:10A86000A452BD4CCD92DD92ED92FC921397EE0F67
:10A87000FF1FEE0FFF1FE857FD4CC082D182E2821E
:10A88000F382B701A6010E947185B701A6018C2F42
:10A890000E947C85CF91FF90EF90DF90CF900C9439
:10A8A00087853F924F925F926F927F928F929F9295
:10A8B000AF92BF92CF92DF92EF92FF920F931F93CE
:10A8C000CF93DF93CDB7DEB76897CDBFDEBF362E0F
:10A8D000872EA62EB72E6C0100E010E0E12CF12CA3
:10A8E0009E2CF50161917191819191915F012CEA0A
:10A8F00035EC47E257E30E9425DA18160CF050C0F9
:10A900008091CF3290E0FC01EE0FFF1FE80FF91F9E
:10A91000EE0FFF1FEE0DFF1DEE0FFF1FEE0FFF1FCF
:10A92000E459FF4C40805180628073808091CE3228
:10A9300081110EC023E333E34BEC51E4F601608157
:10A940007181828193810E94C7DA9B01AC0105C0AD
:10A95000F6012081318142815381C301B2010E94FD
:10A96000B4D6AB01BC01E1E0F0E0EC0FFD1FE00F5D
:10A97000F11F40835183628373839801205B3F4CB6
:10A98000F901E457FD4F4083518362837383E4559B
:10A99000F1094083518362837383892D0E947185FD
:10A9A000FFEFEF1AFF0A0C5F1F4F84E0C80ED11CA7
:10A9B0000831110509F094CF432D582DBE016F5F6A
:10A9C0007F4F87E39CE40E94BE8680E06896CDBFFF
:10A9D000DEBFDF91CF911F910F91FF90EF90DF903D
:10A9E000CF90BF90AF909F908F907F906F905F902F
:10A9F0004F903F9008954F925F926F927F928F9207
:10AA00009F92AF92BF92CF92DF92EF92FF920F93FD
:10AA10001F93CF93DF93CDB7DEB76897CDBFDEBF6F
:10AA200021E0209347338090CF329090CE325B016B
:10AA30006C010CED12E3882D90E07C01EE0CFF1C04
:10AA4000E80EF91EEE0CFF1CEE0CFF1CEE0CFF1CBA
:10AA5000C70184599F4C7C01F501619171918191ED
:10AA600091915F012CEA35EC47E257E30E9425DA29
:10AA7000181664F5F7012081318142815381F80174
:10AA800060817181828193810E94B3D62B013C0148
:10AA900091100EC023E333E34BEC51E4F6016081E7
:10AAA0007181828193810E94C7DA9B01AC0105C04C
:10AAB000F6012081318142815381C301B2010E949C
:10AAC000B3D6F801608F718F828F938FF4E0CF0E31
:10AAD000D11C0C5F1F4F84E0E80EF11C92E3043F91
:10AAE000190709F0B9CF682D70E080E090E00E946E
:10AAF000C2D869837A838B839C831D821E821F82C6
:10AB0000188619861A861B861C861D861E861F8639
:10AB1000188A198A1A8A1B8A1C8A1D8A1E8A1F8A09
:10AB2000188EAE014F5F5F4FBA0184E99FE40E9427
:10AB3000BE8680E06896CDBFDEBFDF91CF911F91CA
:10AB40000F91FF90EF90DF90CF90BF90AF909F90CC
:10AB50008F907F906F905F904F900895CF93DF9389
:10AB6000CDB7DEB76897CDBFDEBF109247331092E6
:10AB7000F4321092F5321092F6321092F7321092AF
:10AB8000F8321092F9321092FA321092FB3210928F
:10AB9000FC321092FD321092FE321092FF3210926F
:10ABA000003310920133109202331092033310924B
:10ABB000043310920533109206331092073310922B
:10ABC00008331092093310920A3310920B336091BC
:10ABD000CF3270E080E090E00E94C2D869837A832F
:10ABE0008B839C831D821E821F82188619861A867B
:10ABF0001B861C861D861E861F86188A198A1A8A3D
:10AC00001B8A1C8A1D8A1E8A1F8A188EAE014F5FFE
:10AC10005F4FBA0184E99FE40E94BE8680E0689697
:10AC2000CDBFDEBFDF91CF910895CF93DF93CDB736
:10AC3000DEB76897CDBFDEBF109247336091CF3249
:10AC400070E080E090E00E94C2D869837A838B83B1
:10AC50009C831D821E821F82188619861A861B8677
:10AC60001C861D861E861F86188A198A1A8A1B8AC8
:10AC70001C8A1D8A1E8A1F8A188EAE014F5F5F4F85
:10AC8000BA0184E99FE40E94BE8680E06896CDBF49
:10AC9000DEBFDF91CF910895CF93DF93CDB7DEB7BD
:10ACA0006897CDBFDEBF81E0809347336091CF329C
:10ACB00070E080E090E00E94C2D869837A838B8341
:10ACC0009C831D821E821F82188619861A861B8607
:10ACD0001C861D861E861F86188A198A1A8A1B8A58
:10ACE0001C8A1D8A1E8A1F8A188EAE014F5F5F4F15
:10ACF000BA0184E99FE40E94BE8680E06896CDBFD9
:10AD0000DEBFDF91CF910895CF93109287320E94DA
:10AD10002A5180915A30813069F488E892E30E9488
:10AD2000274EC82F882331F00E942CAB82E08093FD
:10AD3000533217C083E892E30E94324F85E080933C
:10AD4000533280915432811105C081E08093543296
:10AD50000E94A0AE83E892E30E94689A0E948D5000
:10AD6000C0E08C2FCF91089588E1ECEDF2E3ACE0E8
:10AD7000B3E301900D928A95E1F780E008950F9377
:10AD80001F93CF93DF93CDB7DEB76A97CDBFDEBFFA
:10AD90008C0181E08093D03283E892E3698F7A8FCF
:10ADA0000E94324F698D7A8DC8010E9484560E949C
:10ADB000F8858823E1F388E1E0E0F0E2DE01119616
:10ADC00001900D928A95E1F7BE016F5F7F4F8CE095
:10ADD00093E30E9484566A96CDBFDEBFDF91CF9188
:10ADE0001F910F91089588E1ECEDF2E3A4E2B3E343
:10ADF00001900D928A95E1F780E008950F931F93DB
:10AE0000CF93DF93CDB7DEB76A97CDBFDEBF8C019E
:10AE100081E08093D03283E892E3698F7A8F0E9439
:10AE2000324F698D7A8DC8010E9484560E94F88540
:10AE30008823E1F388E1E0E0F0E2DE011196019081
:10AE40000D928A95E1F7BE016F5F7F4F84E293E335
:10AE50000E9484566A96CDBFDEBFDF91CF911F91CD
:10AE60000F910895FB01DC018091CC32811111C05A
:10AE70009B01AD0160E070E080E89FE30E9429D86B
:10AE80006093C0327093C1328093C2329093C332C8
:10AE900018C08091CE32811109C023E333E34BEC1B
:10AEA00051E4CD010E94C7DAFB0101C0CD01AF0121
:10AEB000BC014093C0325093C1326093C232709350
:10AEC000C33280E008958093CC3280E0089580936F
:10AED000D13280E008956093C8327093C932809374
:10AEE000CA329093CB320E94168780E008950F9368
:10AEF0001F93CF93DF93EC018B018091CC32882399
:10AF000099F08091C0329091C132A091C232B0913B
:10AF1000C332BC01CD019F772CEA35EC47E257E301
:10AF20000E9422D887FD30C081E080938732B8012B
:10AF3000CE010E942A5180915A30813069F488E80C
:10AF400092E30E94274EC82F882331F00E942CAB39
:10AF500082E08093533219C083E892E30E94324F1B
:10AF600085E08093533280915432811105C081E095
:10AF7000809354320E94A0AE83E892E30E94689AC4
:10AF8000C82F0E948D5001C0CEE88C2FDF91CF9149
:10AF90001F910F910895CF93DF93CDB7DEB76897D8
:10AFA000CDBFDEBF682F70E080E090E00E94C2D885
:10AFB00069837A838B839C831D821E821F821886FD
:10AFC00019861A861B861C861D861E861F86188A71
:10AFD000198A1A8A1B8A1C8A1D8A1E8A1F8A188E41
:10AFE000AE014F5F5F4FBA0183E29CE40E94BE86D0
:10AFF00080E06896CDBFDEBFDF91CF910895CF93FB
:10B00000DF93CDB7DEB76897CDBFDEBF6091D43296
:10B0100070E080E090E00E94C2D869837A838B83DD
:10B020009C831D821E821F82188619861A861B86A3
:10B030001C861D861E861F86188A198A1A8A1B8AF4
:10B040001C8A1D8A1E8A1F8A188EAE014F5F5F4FB1
:10B05000BA018DE29CE40E94BE8680E06896CDBF76
:10B06000DEBFDF91CF910895CF93DF93CDB7DEB7E9
:10B070006897CDBFDEBF682F70E080E090E00E944F
:10B08000C2D869837A838B839C831D821E821F8230
:10B09000188619861A861B861C861D861E861F86A4
:10B0A000188A198A1A8A1B8A1C8A1D8A1E8A1F8A74
:10B0B000188EAE014F5F5F4FBA0186E79CE40E9495
:10B0C000BE8680E06896CDBFDEBFDF91CF91089548
:10B0D000CF93DF93CDB7DEB76897CDBFDEBF682FC4
:10B0E00070E080E090E00E94C2D869837A838B830D
:10B0F0009C831D821E821F82188619861A861B86D3
:10B100001C861D861E861F86188A198A1A8A1B8A23
:10B110001C8A1D8A1E8A1F8A188EAE014F5F5F4FE0
:10B12000BA0187E89CE40E94BE8680E06896CDBFA5
:10B13000DEBFDF91CF910895CF93FC0160817181D3
:10B14000828193810E9496D8609353321092553237
:10B1500083E892E3809381329093823280915432DB
:10B16000813011F4109254321092563210927C3287
:10B170000E94219AC0915332C430C9F40E94AE5546
:10B18000809167300E948A53809168308093CD32DD
:10B1900080916B308093D23280E00E94AAB180E02F
:10B1A0000E94685881E08093CC32C093873281E05E
:10B1B000CF910C9464AD8093443380934533809356
:10B1C0004D3380E008952CEA35EC47E257E3609177
:10B1D000F0337091F1338091F2339091F3330E9408
:10B1E00025DA1816B4F48091963390919733A09194
:10B1F0009833B0919933BC01CD019F772CEA35EC9F
:10B2000047E257E30E9422D887FF03C010924433DD
:10B2100003C081E08093443380E0089580934433F9
:10B220008091963390919733A0919833B091993350
:10B2300080933C3390933D33A0933E33B0933F33A0
:10B2400080E008952CEA35EC47E257E36091F03353
:10B250007091F1338091F2339091F3330E9425DAAB
:10B260001816B4F48091963390919733A091983347
:10B27000B0919933BC01CD019F772CEA35EC47E2C0
:10B2800057E30E9422D887FF03C01092453303C0C2
:10B2900081E08093453380E0089580934533809129
:10B2A000963390919733A0919833B09199338093CE
:10B2B000403390934133A0934233B093433380E0C3
:10B2C00008952CEA35EC47E257E36091F033709132
:10B2D000F1338091F2339091F3330E9425DA1816FE
:10B2E000B4F48091963390919733A0919833B091B4
:10B2F0009933BC01CD019F772CEA35EC47E257E347
:10B300000E9422D887FF03C010924D3303C081E012
:10B3100080934D3380E0089580934D338091963330
:10B3200090919733A0919833B0919933809349339A
:10B3300090934A33A0934B33B0934C3380E00895FD
:10B34000BC0187EE90E20C94596681E080937A32DA
:10B35000089581E080937B32089581E080937C3270
:10B3600008951F93CF93DF93CDB7DEB76897CDBF16
:10B37000DEBF0E945B9A8130C9F10E94FAD40E941C
:10B380007B8680E00E94B5AE0E94BEAF10E0812FA8
:10B390000E94339AAB01BC01812F0E9421541F5F90
:10B3A0001630A9F780E090E0A0E4B0E489839A83A6
:10B3B000AB83BC831D821E821F82188619861A8663
:10B3C0001B861C861D861E861F86188A198A1A8A65
:10B3D0001B8A1C8A1D8A1E8A1F8A188EBE016F5FF7
:10B3E0007F4FCB010E949C5880E001C08AE668969E
:10B3F000CDBFDEBFDF91CF911F91089580917A324A
:10B400008130A9F420915532213079F4809156325F
:10B4100081110BC082E08093553280E896E58093DD
:10B420008132909382322093563210927A328091F8
:10B430007B32813091F480915532882331F0823013
:10B4400061F490915632943051F40E945B9A8111CC
:10B4500004C010927B320E94B15990915632809173
:10B460007C328130C1F420917B32211114C0915083
:10B47000933088F010927C3295E0909356329093FE
:10B48000533290915432911104C0809354320E94EF
:10B49000A0AE0E94CDA280E0089585E08093533253
:10B4A00080915432811105C081E0809354320C9414
:10B4B000A0AE0895CF93DF93CDB7DEB76897CDBF29
:10B4C000DEBF80915432882311F180E090E0A0E447
:10B4D000B0E489839A83AB83BC831D821E821F8262
:10B4E000188619861A861B861C861D861E861F8650
:10B4F000188A198A1A8A1B8A1C8A1D8A1E8A1F8A20
:10B50000188EBE016F5F7F4FCB010E949C586896DA
:10B51000CDBFDEBFDF91CF910895CF93DF93CDB73D
:10B52000DEB76897CDBFDEBF80E090E0A0E4B0E476
:10B5300089839A83AB83BC831D821E821F821886F7
:10B5400019861A861B861C861D861E861F86188AEB
:10B55000198A1A8A1B8A1C8A1D8A1E8A1F8A188EBB
:10B56000AE014F5F5F4FBA018CE998E50E94BE863D
:10B570006896CDBFDEBFDF91CF910895CF93DF9363
:10B58000CDB7DEB76897CDBFDEBF80E090E0A0E822
:10B59000B0E489839A83AB83BC831D821E821F82A1
:10B5A000188619861A861B861C861D861E861F868F
:10B5B000188A198A1A8A1B8A1C8A1D8A1E8A1F8A5F
:10B5C000188EAE014F5F5F4FBA018CE998E50E947B
:10B5D000BE866896CDBFDEBFDF91CF910895CF9331
:10B5E000DF93CDB7DEB72797CDBFDEBF97E0E9ED9C
:10B5F000F0E2DE01119601900D929A95E1F7873005
:10B6000050F4E1E0F0E0EC0FFD1FE80FF11D87FDC5
:10B61000FA95808101C080E22796CDBFDEBFDF9121
:10B62000CF910895EF92FF920F931F93CF93DF93E3
:10B630001F92CDB7DEB77C018B01642F70E080E0F4
:10B6400090E049830E94C2D8F7016187728783879F
:10B65000948782E087834981E42FF0E0EE0FFF1F9B
:10B66000E00FF11F659174914FE450E081E59DE397
:10B670000E9435E4BC01C7010F90DF91CF911F916B
:10B680000F91FF90EF900C94FB65CF93DF93EC014B
:10B690000E949D4E482F61EB73E1CE01DF91CF9167
:10B6A0000C94125B4091533262E773E10C94125B8D
:10B6B0004091543269E473E10C94125B409155322D
:10B6C00065E373E10C94125B4091563267E073E1DD
:10B6D0000C94125B409157326AEE72E10C94125B4B
:10B6E000E0918132F0918232E55BFF4F408164E16D
:10B6F00074E10C94125BE0918132F0918232E45B50
:10B70000FF4F408160E272E10C94125BE091813264
:10B71000F0918232448166E871E10C94125BE09111
:10B720008132F0918232E65BFF4F408163E571E147
:10B730000C94125BE0918132F0918232E25BFF4F18
:10B74000408169E071E10C94125BE0918132F091EB
:10B750008232E15BFF4F408168EC70E10C94125B38
:10B76000E0918132F0918232E75BFF4F408169E5E1
:10B7700070E10C94125BCF93DF93EC01E091813286
:10B78000F0918232E05BFF4F608170E080E090E0FA
:10B790000E94C2D869877A878B879C8782E08F83D3
:10B7A00080E0DF91CF910895CF93DF93EC0160911A
:10B7B00083327091843280918532909186320E94DA
:10B7C000C2D869877A878B879C8782E08F8380E0E5
:10B7D000DF91CF910895CF93DF93EC01E091813217
:10B7E000F091823260817181828193810E94C2D8FE
:10B7F00069877A878B879C8782E08F8380E0DF91DF
:10B80000CF910895CF93DF93EC0180915532811150
:10B8100005C019861A861B861C8614C00E942A9AA7
:10B8200069877A878B879C872091CB5621110AC024
:10B8300025E832E441E25DE30E94C7DA69877A874E
:10B840008B879C878C819D81FC01EE0FFF1FE80F89
:10B85000F91FEE0FFF1FEE0FFF1FEE0FFF1FEA5F36
:10B86000F94E85919491888784E08F8380E0DF9101
:10B87000CF910895CF93DF93EC01209181323091E5
:10B880008232F901FD96608171818281938169879D
:10B890007A878B879C873E96208121110AC025E8F4
:10B8A00032E441E25DE30E94C7DA69877A878B87D9
:10B8B0009C878C819D81FC01EE0FFF1FE80FF91F13
:10B8C000EE0FFF1FEE0FFF1FEE0FFF1FEA5FF94E97
:10B8D00085919491888784E08F8380E0DF91CF9178
:10B8E0000895CF93DF93EC018C819D810E94AF4C32
:10B8F000682F80918132909182320E941E50698718
:10B900007A878B879C878C819D81FC01EE0FFF1FBE
:10B91000E80FF91FEE0FFF1FEE0FFF1FEE0FFF1FC7
:10B92000EA5FF94E85919491888784E08F8380E067
:10B93000DF91CF910895CF93DF93EC018C819D81AE
:10B940000E94AF4C20918132309182322358324391
:10B9500069F4E82FF0E0EE0FFF1FEE0FFF1FE45237
:10B96000FD4C608171818281938102C00E94339A73
:10B9700069877A878B879C878C819D81FC01EE0F7C
:10B98000FF1FE80FF91FEE0FFF1FEE0FFF1FEE0F57
:10B99000FF1FEA5FF94E85919491888784E08F8339
:10B9A00080E0DF91CF910895CF93DF93EC018C81FC
:10B9B0009D810E94AF4CE0918132F091823294E0FF
:10B9C000899FE00DF11D1124458D568D678D70A165
:10B9D00049875A876B877C878C819D81FC01EE0F9C
:10B9E000FF1FE80FF91FEE0FFF1FEE0FFF1FEE0FF7
:10B9F000FF1FEA5FF94E85919491888784E08F83D9
:10BA000080E0DF91CF910895CF93DF93EC010E9406
:10BA1000966169857A858B859C850E9496D8462F8C
:10BA200060E474E1CE01DF91CF910C94125BCF936F
:10BA3000DF93EC018C819D810E94AF4C833054F4E4
:10BA40008F3FA9F407C0CE010E94406280E01CC075
:10BA50008DE61AC020E030E040E450E469857A8544
:10BA60008B859C850E9425DA181694F3ECCF20E094
:10BA700030E040E050E469857A858B859C850E94A2
:10BA800025DA18162CF3DFCFDF91CF91089595E3D7
:10BA9000899FF0011124EB5DFE4C608171818281F0
:10BAA00093810895CF92DF92EF92FF92CF93DF932D
:10BAB0006A017B0125E3829FC0011124805B9F4CBA
:10BAC000FC01EB52FF4F4083518362837383EC018F
:10BAD000C352DF4F20E034E244E759E4C701B60126
:10BAE0000E94C7DA9B01AC0160E070E080E89FE350
:10BAF0000E9429D8688379838A839B83DF91CF91C1
:10BB0000FF90EF90DF90CF900895CF92DF92EF9269
:10BB1000FF92CF93DF93EC01C984DA84EB84FC8439
:10BB200020E034E244E759E4C701B6010E9425DA77
:10BB3000181664F420E034E244E759E4C701B60182
:10BB40000E9429D869877A878B879C87CE010E94BB
:10BB50001567C984DA84EB84FC848C819D810E9402
:10BB6000AF4C25E3829FC0011124805B9F4CFC01F8
:10BB7000EB52FF4FC082D182E282F382EC01C352CA
:10BB8000DF4F20E034E244E759E4C701B6010E94E8
:10BB9000C7DA9B01AC0160E070E080E89FE30E949F
:10BBA00029D8688379838A839B8380E0DF91CF9152
:10BBB000FF90EF90DF90CF900895CF92DF92EF92B9
:10BBC000FF92CF93DF93EC01C984DA84EB84FC8489
:10BBD00020E034E244E759E4C701B6010E9425DAC7
:10BBE000181664F420E034E244E759E4C701B601D2
:10BBF0000E9429D869877A878B879C87CE010E940B
:10BC0000156780E0DF91CF91FF90EF90DF90CF90AC
:10BC1000089581E080937B3280E008952CEA35EC32
:10BC200047E257E3FC0161857285838594850E9414
:10BC300025DA181614F40E94136F80E008956091BD
:10BC40007D3270917E3280917F3290918032089562
:10BC50000E94256380E00E94967180E008950E9412
:10BC6000256381E00E94967180E008950E9425631B
:10BC700082E00E94967180E008950E94256383E02F
:10BC80000E94967180E00895CF93DF93EC01E091DC
:10BC90008132F0918232E55BFF4FE081F0E0EE0F00
:10BCA000FF1FED58FB4E659174914FE450E081E524
:10BCB0009DE30E9435E4AC0162E470E1CE01DF91C6
:10BCC000CF910C9463C5CF93DF93EC01E091813267
:10BCD000F0918232E55BFF4FE081F0E0EE0FFF1F55
:10BCE000ED58FB4E659174914FE450E081E59DE382
:10BCF0000E9435E4AC016AE270E1CE01DF91CF91A0
:10BD00000C9463C5CF93DF93EC018BEE90E20E941D
:10BD10009AE5CE010E94445ECE010E94635E66E118
:10BD200070E1CE010E942AC56DEF7FE0CE010E9436
:10BD3000F5C464EE7FE0CE010E94F5C46BEC7FE0B9
:10BD4000CE010E94F5C462EB7FE0CE010E94F5C4F3
:10BD500069E97FE0CE010E94F5C460E87FE0CE0192
:10BD60000E94F5C467E67FE0CE010E94F5C46EE450
:10BD70007FE0CE010E94F5C465E37FE0CE010E9422
:10BD8000F5C46CE17FE0CE010E94F5C463E07FE082
:10BD9000CE010E94F5C46AEE7EE0CE010E94F5C499
:10BDA00061ED7EE0CE010E94F5C468EB7EE0CE013D
:10BDB0000E942AC580E0DF91CF91089566E170E18D
:10BDC0000C942AC56DEF7FE00C94F5C464EE7FE01F
:10BDD0000C94F5C46BEC7FE00C94F5C462EB7FE04F
:10BDE0000C94F5C469E97FE00C94F5C460E87FE049
:10BDF0000C94F5C467E67FE00C94F5C46EE47FE034
:10BE00000C94F5C465E37FE00C94F5C46CE17FE02D
:10BE10000C94F5C463E07FE00C94F5C46AEE7EE018
:10BE20000C94F5C461ED7EE00C94F5C468EB7EE003
:10BE30000C942AC56CE37EE00C942AC56BE07EE08E
:10BE40000C942AC566ED7DE00C942AC56BE97DE073
:10BE50000C942AC567E67DE00C942AC5CF93DF9346
:10BE6000EC01E0918132F0918232E55BFF4FE0819D
:10BE7000F0E0EE0FFF1FED58FB4E659174914FE41B
:10BE800050E081E59DE30E9435E4AC0163E47DE090
:10BE9000CE01DF91CF910C9463C5CF93DF93EC017A
:10BEA000E0918132F0918232E55BFF4FE081F0E07A
:10BEB000EE0FFF1FED58FB4E659174914FE450E07B
:10BEC00081E59DE30E9435E4AC0162E27DE0CE01B4
:10BED000DF91CF910C9463C565E07DE00C940BC5B8
:10BEE000CF93DF93EC01E0918132F0918232E55BF8
:10BEF000FF4FE081F0E0EE0FFF1FED58FB4E659124
:10BF000074914FE450E081E59DE30E9435E4AC017B
:10BF100066EE7CE0CE01DF91CF910C9463C50F9368
:10BF20001F93CF93DF938C01FC016185728583851C
:10BF300094850E9496D8E62FF0E0EE0FFF1FE05C9C
:10BF4000FB4E659174914FE450E081E59DE30E94C2
:10BF500035E4E8012D969F938F93F80161857285F2
:10BF6000838594850E9496D81F926F93DF93CF9319
:10BF70000F5E1F4F1F930F93DF93CF938AEC9CE0CC
:10BF80009F938F93E7E3FAE581818F9380818F936D
:10BF90000E94FCE4EDB7FEB73E96EDBFFEBFDF9119
:10BFA000CF911F910F91089562EA7CE00C94214D8E
:10BFB0006AE77CE00C94214D68E57CE00C94214D0F
:10BFC00066E37CE00C94214D64E07CE00C94214D10
:10BFD00063ED7BE00C94214D6AE97BE00C94214DEC
:10BFE0006AE77BE00C94214D68E37BE00C94EF4C16
:10BFF00066EF7AE00C94EF4C6FEC7AE00C94214DF4
:10C0000069EA7AE00C94214D68E87AE00C94214DBD
:10C0100068E67AE00C94214D6BE47AE00C94744D60
:10C020006CE27AE00C94744DBC01675F7F4F209105
:10C03000CE3242EA5EE0FC01848195810C94CB4DC6
:10C04000BC01675F7F4F21E048E85EE0FC0184812E
:10C0500095810C94CB4DBC01675F7F4F21E04FE68B
:10C060005EE0FC01848195810C94CB4D0F931F936E
:10C07000CF93DF93EC010C811D810E94E0680817CB
:10C080001907C0F48C819D81FC01EE0FFF1FE80FA2
:10C09000F91FEE0FFF1FEE0FFF1FEE0FFF1FE55FF3
:10C0A000F94E25913491CE01F901DF91CF911F9185
:10C0B0000F91199485E1DF91CF911F910F91089510
:10C0C0000F931F93CF93DF93EC010C811D810E948E
:10C0D000E06808171907C0F48C819D81FC01EE0F00
:10C0E000FF1FE80FF91FEE0FFF1FEE0FFF1FEE0FF0
:10C0F000FF1FE75FF94E25913491CE01F901DF91E1
:10C10000CF911F910F91199485E1DF91CF911F91EC
:10C110000F9108950F931F93CF93DF93EC010C8140
:10C120001D810E94E06808171907C0F48C819D8169
:10C13000FC01EE0FFF1FE80FF91FEE0FFF1FEE0FC0
:10C14000FF1FEE0FFF1FE95FF94E25913491CE01DD
:10C15000F901DF91CF911F910F911994DF91CF9148
:10C160001F910F910895CF93DF93EC018C819D81F6
:10C170000E94F3688823C9F08C819D81FC01EE0F39
:10C18000FF1FE80FF91FEE0FFF1FEE0FFF1FEE0F4F
:10C19000FF1FEB5FF94EE491E1FF05C0CE01DF9197
:10C1A000CF910C94978480E001C085E1DF91CF911D
:10C1B00008950F931F93CF93DF93EC0181E00E94CA
:10C1C00024531C821D8280E090E08E010F5E1F4F81
:10C1D00047C08C819D819C01220F331FF901E80F1C
:10C1E000F91FEE0FFF1FEE0FFF1FEE0FFF1FEB5F9C
:10C1F000F94EE491E0FF2EC0280F391F220F331FA4
:10C20000220F331F220F331F215F394EF901459151
:10C2100055916591749149875A876B877C87BC01DA
:10C22000660F771F680F791F660F771F660F771FDE
:10C23000660F771F61507A4E45E050E0C8010E94BA
:10C2400035E4CE010E943660CE010E94B3602C819D
:10C250003D8101C09C012F5F3F4F2C833D83C9016D
:10C260000E94E3688111B5CF0E94E2ABDF91CF91CC
:10C270001F910F910C949AABCF93DF93EC012CEAB2
:10C2800035EC47E257E369857A858B859C850E946A
:10C2900022D887FF05C0CE01DF91CF910C94917D0C
:10C2A000CE010E94D96082E08F8340E050E060E8D8
:10C2B0007FE349875A876B877C8780E0DF91CF9146
:10C2C00008958091463A9091473A8F3E924111F0FD
:10C2D0008AE508958091883A9091893A8F3E9241FB
:10C2E000B9F780911C3590911D358F3E924181F7B1
:10C2F00080913E3890913F388F3E924149F780912E
:10C300004038909141388F3E924111F78091443AE4
:10C310009091453A8F3E9241D9F68091A03D81118E
:10C32000D7CF0895FC01178289E60895CF93DF9354
:10C33000EC018C819D81FC01EE0FFF1FE80FF91FBE
:10C34000EE0FFF1FEE0FFF1FEE0FFF1FE35FF94E13
:10C35000A591B4916C9170E080E090E00E94C2D809
:10C3600069877A878B879C8782E08F8380E0DF9163
:10C37000CF910895CF93DF93EC018C819D81FC01D7
:10C38000EE0FFF1FE80FF91FEE0FFF1FEE0FFF1F4D
:10C39000EE0FFF1FE35FF94EA591B4916D917D9172
:10C3A0008D919C910E94C2D869877A878B879C87E0
:10C3B00082E08F8380E0DF91CF910895CF93DF9368
:10C3C000DC0114968D919C911597FC01EE0FFF1FD7
:10C3D000E80FF91FEE0FFF1FEE0FFF1FEE0FFF1FFD
:10C3E000E35FF94EC591D491488159816A817B817F
:10C3F00019964D935D936D937C931C9783E01796EC
:10C400008C9380E0DF91CF910895CF93DF93DC018F
:10C4100014968D919C911597FC01EE0FFF1FE80F6C
:10C42000F91FEE0FFF1FEE0FFF1FEE0FFF1FE35F61
:10C43000F94EC591D491488159816A817B811996C1
:10C440004D935D936D937C931C97FC01EE0FFF1F42
:10C45000E80FF91FEE0FFF1FEE0FFF1FEE0FFF1F7C
:10C46000EA5FF94E8591949118968C93189784E021
:10C4700017968C9380E0DF91CF91089588E6089518
:10C480000F931F93CF93DF93EC018C819D81FC016F
:10C49000EE0FFF1FE80FF91FEE0FFF1FEE0FFF1F3C
:10C4A000EE0FFF1FE35FF94E0591149169857A85C0
:10C4B0008B859C850E9496D8F801608382E08F83EB
:10C4C00080E0DF91CF911F910F910895CF93DF937B
:10C4D000EC0169857A858B859C850E9496D86230AF
:10C4E000B0F48C819D81FC01EE0FFF1FE80FF91F56
:10C4F000EE0FFF1FEE0FFF1FEE0FFF1FE35FF94E62
:10C50000A591B4916C9382E08F8380E001C08EE6A8
:10C51000DF91CF910895CF93DF93EC0169857A8500
:10C520008B859C850E9496D86330B0F48C819D8168
:10C53000FC01EE0FFF1FE80FF91FEE0FFF1FEE0FBC
:10C54000FF1FEE0FFF1FE35FF94EA591B4916C93AF
:10C5500082E08F8380E001C08EE6DF91CF91089565
:10C56000CF93DF93EC0169857A858B859C850E944A
:10C5700096D86430B0F48C819D81FC01EE0FFF1FD2
:10C58000E80FF91FEE0FFF1FEE0FFF1FEE0FFF1F4B
:10C59000E35FF94EA591B4916C9382E08F8380E0C4
:10C5A00001C08EE6DF91CF9108950F931F93CF9333
:10C5B000DF93EC018C819D81FC01EE0FFF1FE80FE2
:10C5C000F91FEE0FFF1FEE0FFF1FEE0FFF1FE35FC0
:10C5D000F94E0591149169857A858B859C850E9419
:10C5E00096D8F801608371838283938382E08F837E
:10C5F00080E0DF91CF911F910F910895CF93DF934A
:10C60000DC0114968D919C911597FC01EE0FFF1F94
:10C61000E80FF91FEE0FFF1FEE0FFF1FEE0FFF1FBA
:10C62000E35FF94EC591D49119964D915D916D914D
:10C630007C911C97488359836A837B8383E0179698
:10C640008C9380E0DF91CF910895CF93DF93DC014D
:10C6500014968D919C911597FC01EE0FFF1FE80F2A
:10C66000F91FEE0FFF1FEE0FFF1FEE0FFF1FE35F1F
:10C67000F94EC591D49119964D915D916D917C9132
:10C680001C97488359836A837B83FC01EE0FFF1F4D
:10C69000E80FF91FEE0FFF1FEE0FFF1FEE0FFF1F3A
:10C6A000EA5FF94E8591949118968C93189784E0DF
:10C6B00017968C9380E0DF91CF9108951F93CF93CD
:10C6C000DF93EC018091A43A8823D1F01DE10A8028
:10C6D000DB81C02D209711F480E013C08F818F3F44
:10C6E000D9F3811104C0CE010E94606006C0CE0162
:10C6F0000E943660CE010E94B360115041F7ECCF2A
:10C7000085E6DF91CF911F910895CF93DF93EC01E0
:10C71000BC0189EF90E20E946EE4892B41F0BE01DA
:10C720008CEF90E20E946EE421E0892B09F420E076
:10C73000822FDF91CF9108950F931F93CF93DF93B3
:10C74000CDB7DEB72997CDBFDEBF8B0144E050E007
:10C75000BC01CE0101960E948EE446E050E0B80193
:10C76000CE0101960E947EE40E94E068009709F4E1
:10C770003FC07981AA81BB811C810D812FEF35E1FA
:10C7800040E050E0F9016491671327C03196E491CD
:10C79000E11103C0A11121C029C0EA131EC0F90193
:10C7A0003296E491E11103C0B11117C01FC0EB1321
:10C7B00014C0F9013396E491E11103C011110DC0C9
:10C7C00015C0E1130AC0F9013496E491E11103C0E8
:10C7D000011103C00BC0E01749F04F5F5F4F285EA7
:10C7E0003F4F4817590709F0CDCF02C0CA0102C018
:10C7F0008FEF9FEF2996CDBFDEBFDF91CF911F91C5
:10C800000F910895CF93DF93FC012189222371F1C9
:10C81000EC016196BE0180E091E20E946EE4892BFA
:10C8200039F1BE0189EF90E20E946EE4892B11F18B
:10C83000BE0183E091E20E946EE4892BD9F0BE0133
:10C8400087EE90E20E946EE4892BB1F0BE0186E093
:10C8500091E20E946EE4892B79F0BE0187EE91E2AD
:10C860000E946EE4892B51F485E009C080E007C086
:10C8700082E005C083E003C084E001C081E0DF9175
:10C88000CF910895FC018FEF878314821582118662
:10C890001286138614861086118A1586178A108EC2
:10C8A000A081B181109711F416820DC017968C915A
:10C8B0001797873029F416968C918F5F868303C073
:10C8C00016968C918683CF010895EF92FF920F9375
:10C8D0001F93CF93DF93EC010C811D810E94E068D0
:10C8E0000817190708F06FC00C811D81CE010E9446
:10C8F00042640C831D837E0181E1E80EF11CB801C6
:10C90000660F771F600F711F660F771F660F771F07
:10C91000660F771F61507A4EC7010E9416E48E01A0
:10C92000035F1F4F2C813D81B901660F771F620F96
:10C93000731F660F771F660F771F660F771F65508F
:10C940007A4EC8010E9416E48D85882311F18C81EE
:10C950009D81FC01EE0FFF1FE80FF91FEE0FFF1F77
:10C96000EE0FFF1FEE0FFF1FEB5FF94EE491E2FFAA
:10C9700002C01D8610C0F80101900020E9F7BF0138
:10C98000601B710B605F7F4F6C0F7D1FC7010E94A2
:10C9900077E48C819D81FC01EE0FFF1FE80FF91FEA
:10C9A000EE0FFF1FEE0FFF1FEE0FFF1FE75FF94EA9
:10C9B00025913491CE01F901DF91CF911F910F9113
:10C9C000FF90EF901994DF91CF911F910F91FF90FD
:10C9D000EF9008958F929F92AF92BF92CF92DF9285
:10C9E000EF92FF920F931F93CF93DF9300D01F928C
:10C9F000CDB7DEB76C015C0181E1A80EB11C87E008
:10CA0000F6018783ABEFEA2EA5E1FA2E00E010E0F5
:10CA10001DC0B701CE0101960E9416E4BE016F5FF2
:10CA20007F4FC5010E946EE4892B59F44601F9E15C
:10CA30008F0E911CF601058F168FC4010E9465644C
:10CA400064010F5F1F4FF8E1EF0EF11CC8010E9457
:10CA5000E3688111DECF2496CDBFDEBFDF91CF9199
:10CA60001F910F91FF90EF90DF90CF90BF90AF900C
:10CA70009F908F900895CF93DF9310924238109239
:10CA80004338A5E0B5E3EEE1F5E391E08FEFA08355
:10CA9000B18379965B96ED93FC935C975D961D92BE
:10CAA0001C925E97EF0163979883229618822197D4
:10CAB00088832A961882599628E3EE33F20739F7CD
:10CAC000109227381092283810921E3510921F3578
:10CAD0001092243587E08093253582E790E080939B
:10CAE0002F359093303587E395E3DF91CF9108950B
:10CAF0000F931F93CF93DF930E943B65EC018FEE62
:10CB000092E18093463A9093473A8093883A909383
:10CB1000893A80931C3590931D3580933E389093CD
:10CB20003F3880934038909341388093443A9093B3
:10CB3000453A81E00E9424531C821D82CE010E944E
:10CB40006E842091903A3091913A4091923A50916E
:10CB5000933A69857A858B859C850E9422D88823A3
:10CB600039F0CE01DF91CF911F910F910C94D960D4
:10CB70000E949FAB1C821D8280E090E08E010F5EC0
:10CB80001F4F2FC06C817D819B01220F331FF90144
:10CB9000E60FF71FEE0FFF1FEE0FFF1FEE0FFF1F39
:10CBA000EB5FF94EE491E0FF17C0620F731F660F51
:10CBB000771F660F771F660F771F61507A4E45E02B
:10CBC00050E0C8010E9435E4CE010E946E84CE017F
:10CBD0000E9436606C817D816F5F7F4F6C837D83A7
:10CBE000CB010E94E3688111CDCFDF91CF911F91DE
:10CBF0000F910C94E2ABEF92FF920F931F93CF93A0
:10CC0000DF938C012091423830914338EB01099039
:10CC10000020E9F72197C61BD70BAE01420F531F27
:10CC200041305240D8F4F901EC5BF74C7F01AE0182
:10CC30004F5F5F4FCF010E944FE4409142385091C7
:10CC400043384F5F5F4F4C0F5D1F40934238509306
:10CC50004338F801E78AF08E80E001C08DE0DF9173
:10CC6000CF911F910F91FF90EF900895CF93DF9395
:10CC70002EE1C7E3D5E33F813F3F59F00A80DB81D6
:10CC8000C02D209719F480E090E010C0215099F752
:10CC9000FACFBC0180E593E20E949C638C839D8364
:10CCA000019689F3CE010E946564CE01DF91CF9198
:10CCB0000895EF92FF920F931F93CF93DF938B0111
:10CCC0002EE1C7E3D5E33F813F3F59F00A80DB8186
:10CCD000C02D209719F480E090E01DC0215099F7F5
:10CCE000FACF7E0121E1E20EF11C45E050E0BC01EB
:10CCF000C7010E948EE4B801CE010E94FB6581113C
:10CD0000EACFB70180E593E20E949C638C839D8308
:10CD100085E08F83CE01DF91CF911F910F91FF901E
:10CD2000EF9008952091A43A213021F420914D3DB7
:10CD3000213029F4BC0187EE90E20C94596680E022
:10CD400090E008959091A43A913019F4642F0C94D6
:10CD5000EA820C9475C4CF93DF93EC018091BD29D6
:10CD6000811103C00E94F2D402C00E94EECB682F52
:10CD700070E080E090E00E94C2D869877A878B8754
:10CD80009C8782E08F8380E0DF91CF9108950F939D
:10CD90001F93CF93DF93CDB7DEB7C058D109CDBF76
:10CDA000DEBFFC0161857285838594850E9496D8DB
:10CDB0008FEF860F863030F08AE391E20E94926610
:10CDC0008EE62AC06093B82981E08093B929E62FC6
:10CDD000F0E0EE0FFF1FEA53FA4E659174914FE4B5
:10CDE00050E081E59DE30E9435E49F938F9386E8B0
:10CDF00094E19F938F938E010F5F1F4F1F930F93AB
:10CE00000E94F0E5C8010E9492660F900F900F906B
:10CE10000F900F900F9080E0C058DF4FCDBFDEBF66
:10CE2000DF91CF911F910F9108950F931F93CF938F
:10CE3000DF93EC0183E892E30E94F94E882329F006
:10CE400009851A858B859C8511C023E333E34BEC60
:10CE500051E469857A858B859C850E94C7DA8B01B0
:10CE6000AB01BC0149875A876B877C872C813D8148
:10CE7000F901EE0FFF1FE20FF31FEE0FFF1FEE0F82
:10CE8000FF1FEE0FFF1FE35FF94EA591B491A801BC
:10CE9000BC014D935D936D937C931397F901EE0F55
:10CEA000FF1FE20FF31FEE0FFF1FEE0FFF1FEE0F2E
:10CEB000FF1FEA5FF94E85919491888784E08F8304
:10CEC00080E0DF91CF911F910F91089567E975E19F
:10CED0000C940BC563E775E10C940BC567E375E132
:10CEE0000C940BC56CEF74E10C940BC56FEA74E104
:10CEF0000C940BC51F93CF93DF93EC0110E0888156
:10CF0000882301F10E943B6545E050E0BE0188E4C2
:10CF100095E30E948EE468E475E380E593E20E9465
:10CF20009C6380933B3590933C3587E395E30E9467
:10CF3000656442E063E080E00E94A2661F5F26967F
:10CF40001D31E9F684E0DF91CF911F910895CF93D1
:10CF5000DF93CDB7DEB7EC97CDBFDEBF8CE3E8E162
:10CF6000F0E2DE01119601900D928A95E1F7CE0173
:10CF700001960E947A67EC96CDBFDEBFDF91CF911C
:10CF80000895CF93DF93CDB7DEB7AA97CDBFDEBFAD
:10CF90008AE2E4E5F0E2DE01119601900D928A95B5
:10CFA000E1F7CE0101960E947A67AA96CDBFDEBF57
:10CFB000DF91CF910895CF93DF93CDB7DEB76E9712
:10CFC000CDBFDEBF8EE1EEE7F0E2DE01119601900B
:10CFD0000D928A95E1F7CE0101960E947A676E96CE
:10CFE000CDBFDEBFDF91CF910895CF93DF93EC01EA
:10CFF00043E759E763E770E0498B5A8B6B8B7C8B77
:10D000000E94EA6442E063E080E00E94A266CE01F2
:10D010000E94DB67CE010E94C16720E731E340E058
:10D02000298B3A8B4B8BCE010E94EA6442E063E08D
:10D0300080E00E94A266CE01DF91CF910C94A76799
:10D04000CF92DF92EF92FF92CF93DF93EC01C984EE
:10D05000DA84EB84FC8420E030E040E85FE3C70141
:10D06000B6010E9425DA18161CF1C701B6010E940C
:10D0700096D86093BA2989859A85AB85BC85BC0111
:10D08000CD019F772CEA35EC47E257E30E9425DA81
:10D0900018163CF460E470E080E00E949BCA80E0D7
:10D0A00008C060E870E080E00E949BCA80E001C098
:10D0B0008EE6DF91CF91FF90EF90DF90CF900895B3
:10D0C000CF92DF92EF92FF92CF93DF93EC01C9846E
:10D0D000DA84EB84FC8420E030E040E050E4C701D7
:10D0E000B6010E9425DA18161CF1C701B6010E948C
:10D0F00096D86093BC2989859A85AB85BC85BC018F
:10D10000CD019F772CEA35EC47E257E30E9425DA00
:10D1100018163CF464E070E080E00E949BCA80E056
:10D1200008C068E070E080E00E949BCA80E001C017
:10D130008EE6DF91CF91FF90EF90DF90CF90089532
:10D14000CF92DF92EF92FF92CF93DF93EC01C984ED
:10D15000DA84EB84FC8420E030E040E85FE3C70140
:10D16000B6010E9425DA18161CF1C701B6010E940B
:10D1700096D86093BB2989859A85AB85BC85BC010F
:10D18000CD019F772CEA35EC47E257E30E9425DA80
:10D1900018163CF460E170E080E00E949BCA80E0D9
:10D1A00008C060E270E080E00E949BCA80E001C09D
:10D1B0008EE6DF91CF91FF90EF90DF90CF900895B2
:10D1C0008CE891E0089521E08334914008F020E05C
:10D1D000822F08959C012F55314081E0293231057D
:10D1E00008F080E0089521E08036914008F020E0CA
:10D1F000822F0895CF92DF92EF92FF92CF93DF9329
:10D20000EC01C984DA84EB84FC84A7019601C70190
:10D21000B6010E94E8DB81113CC0E894F7F82FEFDB
:10D220003FEF4FE75FE7C701B6010E94E8DB8111DE
:10D230000AC02FEF3FEF4FE75FE7C701B6010E943B
:10D2400022D8181634F18C819D81FC01EE0FFF1F4E
:10D25000E80FF91FEE0FFF1FEE0FFF1FEE0FFF1F6E
:10D26000EB5FF94EE491E3FF14C083E892E30E9480
:10D27000F94E81110EC025E832E441E25DE3698593
:10D280007A858B859C850E94C7DA69877A878B8728
:10D290009C87DF91CF91FF90EF90DF90CF90089522
:10D2A0008091B929882349F01092B9296091B82951
:10D2B00080E00E94A3CA80E0089583E00895CF93A0
:10D2C000DF93E091C33AF091C43A04C0E093C33ACB
:10D2D000F093C43AEF018191982F9D7F9032B1F382
:10D2E0008930A1F34FE450E0BE0187EC9CE30E943B
:10D2F0008EE46881611105C08091A43A81115DC0FE
:10D3000028C0613221F4DF91CF910C94A559653288
:10D3100021F4DF91CF910C94A9596E3721F4DF915C
:10D32000CF910C94AD596B3741F481E08093A43ACE
:10D33000CE01DF91CF910C94E77D70E08AE691E217
:10D340000E9463E4892B59F01092A43ACE010E9406
:10D35000CDC067EC7CE3DF91CF910C940DC280913E
:10D36000A43A811109C0CE010E94627467EC7CE38B
:10D37000DF91CF910C940DC247EF50E0BE0187ECD6
:10D380009AE30E948EE487EC9AE39F938F938FE653
:10D3900091E29F938F93DF93CF930E94C7E50F9005
:10D3A0000F900F900F900F900F908091C33A909133
:10D3B000C43ADF91CF910C94E77DDF91CF9108952E
:10D3C000FF920F931F93CF93DF931F921F92CDB7BE
:10D3D000DEB7F82EEAE8FAE32FE832E0DF01C90110
:10D3E0001D920197E9F72FEE32E1208331832093DC
:10D3F000173D3093183D06EF18E82CED33E4009309
:10D40000903A1093913A2093923A3093933A0CEEDB
:10D4100011E528E73FE30093943A1093953A20935F
:10D42000963A3093973A00E010E020EA30E4009317
:10D43000983A1093993A20939A3A30939B3A00E0A5
:10D4400010E020E83FE300939C3A10939D3A20932C
:10D450009E3A30939F3A83E08093A63A8F2D4A8379
:10D4600069830E94B3CA6981862F0E94BECA4A811D
:10D47000842F0E94C9CAF092B729F092B5290F9063
:10D480000F90DF91CF911F910F91FF900895CF934F
:10D49000DF931F921F92CDB7DEB780E6F82E01E032
:10D4A00010E00E944F7C8230E1F30E94567C823073
:10D4B000C1F30E94D84E863009F0C6C00E9497C8BA
:10D4C0008090AC3A9090AD3AA090AE3AB090AF3A1E
:10D4D00086169706A806B90620F70E9497C86C59C9
:10D4E0007F4F8F4F9F4F6093AC3A7093AD3A8093CC
:10D4F000AE3A9093AF3A0E94C57BD3CF0E94A0BFB3
:10D50000882329F08CEC0E941053823051F20E9443
:10D51000FE59823031F20E9427A1823011F20E941E
:10D5200061618093A13D81112EC080918A3A9091D2
:10D530008B3A8F3E924109F08DC08091173D9091BA
:10D54000183D8F3E924109F085C08AC00E944385F4
:10D550008093A13D811117C00E94C4B58093A13D65
:10D56000811111C00E942D748093A13D81110BC0C7
:10D570000E94B5C98093A13D811105C00E945DB68E
:10D58000823031F48ECF0E9410538230B9F789CFA8
:10D590000E9496AD823009F484CF0E9402AF82309F
:10D5A00009F47FCF0E94C9AF823009F47ACF098392
:10D5B0001A8365EC7AE3CE0101960E94D8CA809363
:10D5C000C33A9093C43A892B11F00E945F690E947C
:10D5D000868F823009F465CF0E94626F823009F431
:10D5E00060CF0E942172823009F45BCF0E940874E0
:10D5F000823009F456CF0E94A750823009F44FCFF1
:10D600000E94F8858430B0F54ACF8091A63A8430E4
:10D6100038F484E08093A63A0E94A9590E94A4ABF2
:10D6200083E090E089839A8365EC7AE3CE010196EA
:10D630000E94D8CA8093C33A9093C43A892B09F4C4
:10D640002ECF0E945F692BCF0E94D84E823009F402
:10D650005ECF54CFF092A13D80E60E94105395CF4B
:10D660001092A13D0E94D5528093A13D882309F4D8
:10D670006DCF89CF8091CD289091CE280E9466D31E
:10D68000682F70E080E090E00E94C4D823E333E389
:10D690004BE451E40E9425DA87FF01CF0E945069D4
:10D6A000823009F0B2CFFBCE8091B7298093B529A3
:10D6B00008958093B52908958093B6290895CF934E
:10D6C000C82F80919B23882379F040E050E0BA0175
:10D6D0008C2F0E942154EC2FFF27E7FDF095E85A8C
:10D6E000FD4C81E080830AC06C2F80E896E50E94A3
:10D6F0001E50AB01BC018C2F0E9421544091C223CB
:10D700005091C3236091C4237091C5238C2F0E9434
:10D71000525D88E29DE680939C2390939D2382E056
:10D72000CF910895CF92DF92EF92FF920F931F93C4
:10D73000CF93DF93CDB7DEB7E097CDBFDEBF98E1E3
:10D740007E01A9E1EA0EF11CF701A92F1192AA9519
:10D75000E9F7FE0131966F0111929A95E9F7F6010A
:10D7600094E08902E00DF11D1124408F518F628FEA
:10D77000738F80E090E0A0E8BFE380839183A28371
:10D78000B3830093C0321093C1322093C2323093DE
:10D79000C3320E947B860E94AD59B601C7010E9428
:10D7A00077578093A13D811101C082E0E096CDBF03
:10D7B000DEBFDF91CF911F910F91FF90EF90DF902F
:10D7C000CF9008950F931F93E0919523FF27E7FDD6
:10D7D000F095E35DFF4C9381913099F40091A6237D
:10D7E0001091A7232091A8233091A9234091AE2323
:10D7F0005091AF236091B0237091B1230E94926B3E
:10D800001DC0E0919623FF27E7FDF095E35DFF4CF7
:10D810009381913099F40091A6231091A723209130
:10D82000A8233091A9234091AE235091AF2360915A
:10D83000B0237091B12370580E94926B88E29CE6ED
:10D8400080939C2390939D2382E01F910F910895D4
:10D850000F931F93CF93C82F85E3C802F0011124C3
:10D86000E75DFE4C40815181628173818C2F0E9463
:10D87000525D0091A6231091A7232091A8233091F7
:10D88000A9234091A2235091A3236091A4237091D6
:10D89000A5238C2F0E94926B87EB9CE680939C23A0
:10D8A00090939D2382E0CF911F910F9108950F9344
:10D8B0001F930091A6231091A7232091A8233091B4
:10D8C000A9234091B2235091B3236091B423709166
:10D8D000B5230E94926B8FE59BE680939C239093E7
:10D8E0009D2382E01F910F9108950E947B86809175
:10D8F000BB230E948A538091BA230E9424538091B3
:10D90000BC230E9428538091BD230E9463578091BD
:10D91000BE239091BF23A091C023B091C1238093D7
:10D92000C0329093C132A093C232B093C33264E04C
:10D9300083E892E30E94164F0E945A5A1092543282
:10D9400080E00895CF93C82F4091C2235091C32304
:10D950006091C4237091C5230E94525D8C2F0E9458
:10D96000756C80E00E9464AD80EFCF9108950F93B5
:10D970001F93E0919523FF27E7FDF095E35DFF4CB2
:10D980009381913039F082EA9CE680939C239093B6
:10D990009D2318C00091AA231091AB232091AC23A2
:10D9A0003091AD234091AE235091AF236091B023CD
:10D9B0007091B1230E94926B87E59CE680939C2333
:10D9C00090939D2382E01F910F910895FF920F93F2
:10D9D0001F93CF93DF93CDB7DEB7C058D109CDBF2A
:10D9E000DEBFF82E0E943B658EEFF81205C08CE773
:10D9F00091E20E94926619C08F2D0E94EF5A1F92E9
:10DA00008F932BE13BE33F932F938E010F5F1F4FCB
:10DA10001F930F930E94F0E5C8010E9492660F9039
:10DA20000F900F900F900F900F9042E062E080EF08
:10DA30000E94A2668F2D0E94756C80EFC058DF4F48
:10DA4000CDBFDEBFDF91CF911F910F91FF90089561
:10DA50004F925F926F927F929F92AF92BF92CF92BE
:10DA6000DF92EF92FF920F931F93CF93DF938F3F3D
:10DA700009F045C02CEA35EC47E257E36091B93331
:10DA80007091BA338091BB339091BC330E9425DAF8
:10DA900018160CF469C12CEA35EC47E257E36091A3
:10DAA000B1337091B2338091B3339091B4330E940B
:10DAB00025DA18160CF45DC12CEA35EC47E257E381
:10DAC0006091B5337091B6338091B7339091B8338C
:10DAD0000E9425DA18160CF455C12CEA35EC47E201
:10DAE00057E36091BD337091BE338091BF33909105
:10DAF000C0330E9425DA18160CF43FC171C1823080
:10DB0000A1F52CEA35EC47E257E36091B13370910F
:10DB1000B2338091B3339091B4330E9425DA181652
:10DB20000CF427C12CEA35EC47E257E36091B5339A
:10DB30007091B6338091B7339091B8330E9425DA53
:10DB400018160CF41FC12CEA35EC47E257E360913C
:10DB5000BD337091BE338091BF339091C0330E942A
:10DB600025DA18160CF409C131C18823D9F28130A5
:10DB700051F32CC17E018DEEE80EF11CF70180817E
:10DB80009181A281B381BC01CD019F772CEA35EC54
:10DB900047E257E30E9422D887FD46C06E01F1EFAD
:10DBA000CF0ED11CF601408051806280738020E04E
:10DBB00030E0A901C301B2010E9422D887FD34C020
:10DBC000FE01EF52FF4F2081318142815381349712
:10DBD00060817181828193810E94B3D69B01AC01E7
:10DBE0005F77C301B2010E94B4D62B013C019F773D
:10DBF0002CEA35EC47E257E30E9422D887FD14C097
:10DC0000AB2CAA0C8A2D0E949ABF8093932399244F
:10DC100093949A0C892D0E949ABF8093942320910B
:10DC20009323822780FD02C08B2DDBC0B09292230C
:10DC3000F80180819181A281B381BF778093A6236F
:10DC40009093A723A093A823B093A923F701408121
:10DC50005181628173817F774093AA235093AB23D4
:10DC60006093AC237093AD2320FF2DC0A092952329
:10DC70009092962377FA709477F870944092A2234A
:10DC80005092A3236092A4237092A523F601808171
:10DC90009181A281B3818093AE239093AF23A0930F
:10DCA000B023B093B123CB50DF4F88819981AA81F3
:10DCB000BB818093B2239093B323A093B423B093FA
:10DCC000B5238A2D2AC090929523A0929623409244
:10DCD000A2235092A3236092A4237092A523F6015D
:10DCE00080819181A281B381B0588093AE239093BB
:10DCF000AF23A093B023B093B123CB50DF4F8881E3
:10DD00009981AA81BB81B0588093B2239093B323A9
:10DD1000A093B423B093B523892D0E949ABF8D7F21
:10DD2000813039F088E29DE680939C2390939D2377
:10DD300069C0809196230E949ABF811103C08FEF22
:10DD4000809396238B2D0E94475D6093C22370932E
:10DD5000C3238093C4239093C52382EE9BE68093D4
:10DD60009C2390939D234EC082E090E032E0B32E3E
:10DD70000DC080E090E0B12C09C083E090E023E08A
:10DD8000B22E04C081E090E0BB24B394FC01E85AB9
:10DD9000FD4C108225E3289FE001299FD00D11241E
:10DDA000C05BDF4C8E0107511F4FF80180819181CC
:10DDB000A281B381BC01CD019F772CEA35EC47E20B
:10DDC00057E30E9422D887FFD5CE2ECF81E08093E3
:10DDD000573285E79CE680939C2390939D2312C045
:10DDE0008EEFDF91CF911F910F91FF90EF90DF9019
:10DDF000CF90BF90AF909F907F906F905F904F902B
:10DE00000C94E66C82E0DF91CF911F910F91FF900F
:10DE1000EF90DF90CF90BF90AF909F907F906F90EA
:10DE20005F904F900895CF93DF93C1E8D2E388814C
:10DE300099810E94F94E8093BA23888199810E942A
:10DE4000F44E8093BB23888199810E94034F809375
:10DE5000BC23888199810E94084F8093BD238881CB
:10DE600099810E940F4F6093BE237093BF238093CC
:10DE7000C0239093C12381E00E94245381E00E943B
:10DE8000285380E00E948A5381E00E94635781E01A
:10DE900080939B238FEF8093922388E29DE680936B
:10DEA0009C2390939D2383E08093543210925732A9
:10DEB00080E0DF91CF9108950E94136F10929B2311
:10DEC00080E0089580915432833059F40E940D4FC0
:10DED000813049F0E0919C23F0919D238091922321
:10DEE000199483E0089582E008958DE79FE680937A
:10DEF000D7239093D82382E008952F923F924F9298
:10DF00005F926F927F928F929F92AF92BF92CF92C9
:10DF1000DF92EF92FF920F931F93CF93DF93CDB7D2
:10DF2000DEB7CA54D109CDBFDEBF98E19E01275E9E
:10DF30003F4F29AB3AABD901E92F1D92EA95E9F79A
:10DF4000285131091901D9011D929A95E9F724E068
:10DF50008202F00111242B96EEAFFFAF2B97E20D5A
:10DF6000F31D80E090E0A0E8BFE380839183A2836B
:10DF7000B383C090CF23D090D023E090D123F090F2
:10DF8000D2234090CB235090CC236090CD2370902F
:10DF9000CE238090C7239090C823A090C923B0902F
:10DFA000CA23A5019401C301B2010E9422D8181608
:10DFB0005CF080E090E0A0E8BFE329968CAF9DAFD5
:10DFC000AEAFBFAF29970AC080E090E0A0E8BFEBFA
:10DFD00029968CAF9DAFAEAFBFAF2997A301920139
:10DFE000C501B4010E94B3D60E9491D89B0177FF6E
:10DFF00004C022273327261B370BB901882777FD5A
:10E000008095982F0E94C4D825966CAF7DAF8EAFB7
:10E010009FAF2597C092C032D092C132E092C232F7
:10E02000F092C3320E947B860E94AD5920E030E01E
:10E0300040E050E425966CAD7DAD8EAD9FAD25974B
:10E040000E9425DA18166CF08091D3239091D42386
:10E05000A091D523B091D6238BAF9CAFADAFBEAF0F
:10E06000DBC02AE037ED43E25CE325966CAD7DAD85
:10E070008EAD9FAD25970E9425DA18162CF709E181
:10E0800010E08AE0882E87ED982E83E2A82E8CE39C
:10E09000B82E412C512C32012B96AEADBFAD2B9733
:10E0A000A20DB31D58962196AEAFBFAF21974BAAD4
:10E0B0005CAA6DAA7EAA8FAA98AEA9AEBAAE29961E
:10E0C0002CAD3DAD4EAD5FAD29976FA978AD89AD53
:10E0D0009AAD0E94C7DA9B01AC016091CB2370918D
:10E0E000CC238091CD239091CE230E94B4D621964B
:10E0F000EEADFFAD21976083718382839383C092DD
:10E10000C032D092C132E092C232F092C332B10139
:10E11000CE0149960E9477578093A13D8111AAC0F4
:10E1200020E030E040E85FE36BA97CA98DA99EA9BF
:10E130000E94B4D66BAB7CAB8DAB9EAB20E030E0E5
:10E1400048EC51E40E9429D89B01AC0160E070E0EA
:10E1500080E291E40E942ADB2B013C018091D323D1
:10E160009091D423A091D523B091D6238BAF9CAFAF
:10E17000ADAFBEAFC090CF23D090D023E090D123DD
:10E18000F090D223A7019601BC01CD010E94B3D625
:10E190004B015C0120E030E040E251E4C301B201F8
:10E1A0000E9429D89B01AC01C501B4010E94C7DAC5
:10E1B0009B01AC01C701B6010E94B4D66B017C0182
:10E1C0002BA93CA94DA95EA9CA01B9010E94B4D6E8
:10E1D00020E030E048EC51E40E9429D89B01AC01DA
:10E1E0006FA978AD89AD9AAD0E94B4D66FAB78AF08
:10E1F00089AF9AAF9B01AC0125966CAD7DAD8EAD1C
:10E200009FAD25970E9425DA181634F401501109A4
:10E210000115110509F053CF8BAD9CADADADBEAD71
:10E220008093C0329093C132A093C232B093C33274
:10E230002B96EEADFFAD2B97E20DF31D8091C7231A
:10E240009091C823A091C923B091CA23808F918F48
:10E25000A28FB38FB101CE0149960E947757809368
:10E26000A13D811107C081E591E78093D723909369
:10E27000D82382E0C65BDF4FCDBFDEBFDF91CF91F9
:10E280001F910F91FF90EF90DF90CF90BF90AF90D4
:10E290009F908F907F906F905F904F903F902F90C6
:10E2A0000895CF93DF931F92CDB7DEB789830E9485
:10E2B0007B864091E1235091E2236091E3237091AA
:10E2C000E42389810E94525D8091DE230E948A535B
:10E2D0008091DD230E9424538091DF230E942853E4
:10E2E0008091E0230E9463578091D9239091DA2393
:10E2F000A091DB23B091DC238093C0329093C13294
:10E30000A093C232B093C33264E083E892E30E94E8
:10E31000164F0E945A5A1092543288EA91E20E9493
:10E320009AE580E00F90DF91CF9108950F931F93AE
:10E33000CF93C82F01E812E3F801808191810E94F8
:10E34000F94E8093DD23F801808191810E94F44E83
:10E350008093DE23F801808191810E94034F809396
:10E36000DF23F801808191810E94084F8093E02390
:10E37000F801808191810E940F4F6093D92370939F
:10E38000DA238093DB239093DC238C2F0E94475D5C
:10E390006093E1237093E2238093E3239093E4233B
:10E3A00081E00E94245380E00E94285380E00E9474
:10E3B0008A5381E00E94635740E050E060E271E4DC
:10E3C0004093CF235093D0236093D1237093D223D3
:10E3D00085E3C89FF0011124E75EFE4C4081518126
:10E3E000628173814093D3235093D4236093D523C8
:10E3F0007093D6236C2F80E896E50E940B506093B3
:10E40000CB237093CC238093CD239093CE230E9473
:10E410001F5E6093C7237093C8238093C923909392
:10E42000CA23C093C62385E79FE68093D7239093A2
:10E43000D82384E08093543280E0CF911F910F91D4
:10E44000089580915432843059F40E940D4F8130E8
:10E4500049F0E091D723F091D8238091C6231994F5
:10E4600083E0089582E00895E091E723F0E0E35D22
:10E47000FF4C8381882341F08FE492E78093E5236A
:10E480009093E62382E0089564E374E28CE194E2E1
:10E490000E9477578093A13D882371F308951F93BD
:10E4A000CF93DF93E091E723F0E0E35DFF4C81E061
:10E4B0009381913009F080E080935E32CFE5D2E322
:10E4C00010E0612F80E896E50E941E50AB01BC0170
:10E4D000812F0E942154612F80918132909182324C
:10E4E0000E940B5069937993899399931F5F16301B
:10E4F00041F782EB91E20E94E77D8DEB92E78093FA
:10E50000E5239093E62382E0DF91CF911F91089558
:10E510001F93CF93DF930E947B868091E8238093A3
:10E520002D30E091E723F0E08091E923E35DFF4C9B
:10E5300083870E94B7BFCCEED3E210E04991599196
:10E5400069917991812F0E94525D1F5F1630B1F75A
:10E550008091EB230E948A538091EA230E942853E2
:10E5600064E083E892E30E94164F0E945A5A109288
:10E570005432DF91CF911F9108950E94887280E0FC
:10E5800008950F931F93CF93DF93CDB7DEB7C05895
:10E59000D109CDBFDEBF182F0E943B651E3F29F475
:10E5A0008FEB91E20E94926619C0812F0E94EF5A70
:10E5B0001F928F9389E49BE39F938F938E010F5F4C
:10E5C0001F4F1F930F930E94F0E5C8010E949266AF
:10E5D0000F900F900F900F900F900F9042E062E01D
:10E5E0008AEF0E94A2660E9488728AEFC058DF4FAD
:10E5F000CDBFDEBFDF91CF911F910F910895FF92A4
:10E600000F931F93CF93DF9310925E3282E080933B
:10E6100054320CEE13E2C9E2D1E3F12C8F2D0E94AB
:10E62000475DF80161937193819391938F014881C4
:10E6300059816A817B818F2D0E94525D6F2D80915F
:10E640008132909182320E940B50F801648B758B5D
:10E65000868B978BF394E596F6E0FF12DFCF6CE1A3
:10E6600074E284E094E20E949AC52AE43CE042E825
:10E670005EE30E9422D887FF03C08EEF0E94C17222
:10E68000C0E1D4E213E069917991899199912C8943
:10E690003D894E895F890E94B3D69F772CEA35EC7D
:10E6A00047E257E30E9425DA18161CF4812F0E94D6
:10E6B000C1721F5F163039F784E08093E7238091A1
:10E6C0003C308093E92381E080933C3080912D3071
:10E6D0008093E82310922D300E94B7BF8091813241
:10E6E000909182320E94F44E8093EB23809181328C
:10E6F000909182320E94034F8093EA2380E00E942F
:10E70000285380E00E948A5380E00E94AAB184E3EB
:10E7100092E78093E5239093E62382E0DF91CF9107
:10E720001F910F91FF9008950F931F93CF93DF9345
:10E730008C01EB018091CC32882399F08091C0321A
:10E740009091C132A091C232B091C332BC01CD01CF
:10E750009F772CEA35EC47E257E30E9422D887FDE9
:10E760004FC088819981AA81BB81BC01CD019F776F
:10E770002CEA35EC47E257E30E9425DA1816F4F448
:10E780008C819D81AE81BF81BC01CD019F772CEA38
:10E7900035EC47E257E30E9425DA18167CF48885A9
:10E7A0009985AA85BB85BC01CD019F772CEA35EC04
:10E7B00047E257E30E9425DA181624F188E1F801B0
:10E7C000ACE1B4E201900D928A95E1F788E1FE0197
:10E7D000A4E3B4E201900D928A95E1F788E1EFE5B8
:10E7E000F2E3DF011D928A95E9F782E080935E32C1
:10E7F0008FEF92E78093E5239093E62380E003C0B8
:10E800008EE801C086E8DF91CF911F910F910895A6
:10E8100080915432823021F080915E32823049F40E
:10E820000E940D4F813039F0E091E523F091E6230D
:10E83000199483E0089582E00895E9E1FDE380E220
:10E84000DF011D928A95E9F78FEE92E18093373DC3
:10E850009093383D8083918308958091373D9091C6
:10E86000383D8F3E924111F08CE508958091193D1D
:10E8700090911A3D8F3E9241B9F780E00895CF9371
:10E88000DF93C82FCB01BA010E9476DB27E0C29F3D
:10E89000E0011124C75ED24C0E9491D86D837E8323
:10E8A0008F839887DF91CF91089597E0899FF0013A
:10E8B0001124E75EF24C65817681878190850E9404
:10E8C000C4D808952F923F924F925F926F927F9299
:10E8D0008F929F92AF92BF92CF92DF92EF92FF9270
:10E8E0000F931F93CF93DF93CDB7DEB72797CDBF9D
:10E8F000DEBF8C011B8280915332823009F4A6C6A0
:10E90000D801BC90B110CFC680E06E01B3E0CB0E51
:10E91000D11C3DC0F6018081811108C0B72CD70100
:10E920001C926E01B3E0CB0ED11CBAC6883239F40A
:10E93000B72CF7011082FFEFCF1ADF0AB1C68B3375
:10E94000B9F3A82EB12CC5010E94EAE3892B39F452
:10E95000B50189EE91E20E9463E4892B51F04701F1
:10E960008FEF881A980AC5010E940EE4D7018C9394
:10E970007401BFEFCB1ADB0AF70180818111CACF86
:10E98000B72CD8018C916E01B3E0CB0ED11CF801ED
:10E990001CC08E32E1F090E0C0970A9790F0818120
:10E9A000803391F4828190E0C0970A9760F4DF0190
:10E9B000119611968C9111978D938111FACF8081C8
:10E9C00004C0818101C080E331968111E2CFF6015C
:10E9D000A080A11007C036C0D6011196AC90BFEF41
:10E9E000CB1ADB0A76018A2C912CC4010E94FEE32B
:10E9F000892B91F7C4010E9406E48D369105A1F49C
:10EA0000F601818190E00E9406E48337910561F46C
:10EA1000D60112968C9190E00E9406E4873691050B
:10EA200019F4F601339602C0FE013396AA2061F074
:10EA30008A2DD701893209F41C9211968C9181118B
:10EA4000F9CF02C0FE013396BFE2BB1609F400C63F
:10EA50008081882319F0CF010E94A05980E1E9E369
:10EA6000FDE3DF011D928A95E9F78AE5EAEAF3E31F
:10EA7000DF01982F1D929A95E9F7E0E5F3E3DF01B6
:10EA80001D928A95E9F783E892E30E94F14E809304
:10EA90005133812C912C80E8A82E8FE3B82E552479
:10EAA000539492E0492E24E0322EBDC3C701B60133
:10EAB0000E9496D8862F90E08F35910508F0CCC53E
:10EAC000FC01EC50FF4F0C946DE0109251335092CA
:10EAD000AB3380913A3D8F5F80933A3DA4C350920F
:10EAE00051335092AB3380913A3D8F5F80933A3DE2
:10EAF0009AC3409251335092AB3380913A3D8F5F2D
:10EB000080933A3D90C383E0809351335092AB336E
:10EB100080913A3D8F5F80933A3D85C38DE080932D
:10EB200050335092AA337FC388E0B2C01092803332
:10EB30005092DA3380913B3D8F5F80933B3D73C3AE
:10EB4000509280335092DA3380913B3D8F5F8093B7
:10EB50003B3D69C3409280335092DA3380913B3D14
:10EB60008F5F80933B3D5FC3109281335092DB33C4
:10EB700080913E3D8F5F80933E3D55C350928133DF
:10EB80005092DB3380913E3D8F5F80933E3D4BC37F
:10EB9000C701B6010E94E1DB6C837D838E839F8376
:10EBA00020E030E040E251E4C701B6010E94C7DA3C
:10EBB0006B017C0120E030E040E251E46C817D811A
:10EBC0008E819F810E94C7DA9B01AC01C701B6010B
:10EBD0000E94B3D60E9496D8623001F128F46623D1
:10EBE00041F0613089F038C56330E9F0643001F1FB
:10EBF00033C5B5E0B09350335092AA338091393D7C
:10EC00008F5F8093393D0FC3309250336093AA33A6
:10EC10008091393D8F5F8093393D05C350925033C9
:10EC20005092AA3300C3409250335092AA33FBC291
:10EC300083E0809350335092AA33F5C2C701B601E6
:10EC40000E94E1DB6C837D838E839F8320E030E034
:10EC500040E251E4C701B6010E94C7DA6B017C01B2
:10EC600020E030E040E251E46C817D818E819F8123
:10EC70000E94C7DA9B01AC01C701B6010E94B3D65E
:10EC80000E9496D8662319F0613061F0E5C487E0F0
:10EC9000809350335092AA338091393D8F5F809397
:10ECA000393DC1C2E6E0E09350336093AA338091CE
:10ECB000393D8F5F8093393DB6C2C701B6010E94CE
:10ECC000E1DB6C837D838E839F8320E030E040E234
:10ECD00051E4C701B6010E94C7DA6B017C0120E054
:10ECE00030E040E251E46C817D818E819F810E9401
:10ECF000C7DA9B01AC01C701B6010E94B3D60E94DE
:10ED000096D8623009F0A8C48EE0809350335092B8
:10ED1000AA3389C2509283335092DD3384C2509219
:10ED200082335092DC338091423D8F5F8093423D2D
:10ED30007AC2409282335092DC338091423D8F5FA1
:10ED40008093423D70C283E016C03092823350926D
:10ED5000DC338091423D8F5F8093423D64C2F5E099
:10ED6000F09382335092DC338091423D8F5F8093E9
:10ED7000423D59C286E0809382335092DC338091C9
:10ED8000423D8F5F8093423D4EC2C701B6010E9453
:10ED9000E1DB6C837D838E839F8320E030E040E263
:10EDA00051E4C701B6010E94C7DA6B017C0120E083
:10EDB00030E040E251E46C817D818E819F810E9430
:10EDC000C7DA9B01AC01C701B6010E94B3D60E940D
:10EDD00096D8662319F0613059F03EC410928533FD
:10EDE0005092DF338091433D8F5F8093433D1BC240
:10EDF000609385336093DF338091433D8F5F8093D1
:10EE0000433D11C2409285335092DF338091433DA0
:10EE10008F5F8093433D07C2309251335092AB33A2
:10EE200080913A3D8F5F80933A3DFDC110928633C9
:10EE30005092E03380913C3D8F5F80933C3DF3C125
:10EE4000509286335092E03380913C3D8F5F8093A7
:10EE50003C3DE9C1C701B6010E94E1DB6C837D83C3
:10EE60008E839F8320E030E040E251E4C701B60189
:10EE70000E94C7DA6B017C0120E030E040E251E4FF
:10EE80006C817D818E819F810E94C7DA9B01AC01DC
:10EE9000C701B6010E94B3D60E9496D8613089F0AE
:10EEA00028F06230A1F06330C1F0D6C399E09093AE
:10EEB00050335092AA338091393D8F5F8093393D12
:10EEC000B2C1AAE0A09350336093AA33ACC1BBE0B7
:10EED000B09350335092AA33A6C1ECE0E093503384
:10EEE0005092AA33A0C110927B335092D5338091B7
:10EEF0003D3D8F5F80933D3D96C150927B33509254
:10EF0000D53380913D3D8F5F80933D3D8CC1C701DE
:10EF1000B6010E9496D8862F90E08D33910508F0B7
:10EF200099C3FC01ED5AFE4F0C946DE010925233E0
:10EF30005092AC338091443D8F5F8093443D73C1C8
:10EF4000509252335092AC338091443D8F5F809306
:10EF5000443D69C150928C335092E6338091463DD6
:10EF60008F5F8093463D5FC140928C335092E63371
:10EF70008091463D8F5F8093463D55C110928C3302
:10EF80005092E6338091463D8F5F8093463D4BC162
:10EF9000509289335092E33346C150928A33509253
:10EFA000E4338091473D8F5F8093473D3CC1509251
:10EFB0008B335092E5338091473D8F5F8093473D7F
:10EFC00032C110928B335092E5338091473D8F5F71
:10EFD0008093473D28C150927E335092D833809120
:10EFE000483D8F5F8093483D1EC110927E33509202
:10EFF000D8338091483D8F5F8093483D14C1509233
:10F000007C335092D6338091483D8F5F8093483D4A
:10F010000AC1509295335092EF338091483D8F5FF3
:10F020008093483D00C1C701B6010E94E1DB0E9408
:10F0300096D8609388335092E233F5C0C0926F3314
:10F04000D0927033E0927133F09272338092C93370
:10F050009092CA33A092CB33B092CC33E4C0C0922A
:10F060009633D0929733E0929833F092993380920E
:10F07000F0339092F133A092F233B092F333D3C0D5
:10F08000C0928D33D0928E33E0928F33F0929033D2
:10F090008092E7339092E833A092E933B092EA335A
:10F0A000C2C0C0925733D0925833E0925933F09295
:10F0B0005A338092B1339092B233A092B333B0926C
:10F0C000B433B1C0C0925B33D0925C33E0925D3315
:10F0D000F0925E338092B5339092B633A092B733FC
:10F0E000B092B833A0C0C0925F33D0926033E09248
:10F0F0006133F09262338092B9339092BA33A09226
:10F10000BB33B092BC338FC0C0926333D0926433B0
:10F11000E0926533F09266338092BD339092BE33B5
:10F12000A092BF33B092C0337EC0C0926733D092FA
:10F130006833E0926933F0926A338092C1339092DF
:10F14000C233A092C333B092C4336DC0C0926B334C
:10F15000D0926C33E0926D33F0926E338092C5336F
:10F160009092C633A092C733B092C8335CC0C092AD
:10F170009E33D0929F33E092A033F092A1338092DD
:10F18000F8339092F933A092FA33B092FB334BC02C
:10F19000C092A233D092A333E092A433F092A5336D
:10F1A0008092FC339092FD33A092FE33B092FF33F5
:10F1B0003AC0C092A633D092A733E092A833F0921F
:10F1C000A9338092003490920134A0920234B0921C
:10F1D000033429C0C0929A33D0929B33E0929C337F
:10F1E000F0929D338092F4339092F533A092F633EF
:10F1F000B092F73318C0C701B6010E9496D8609349
:10F20000533370935433809355339093563381E046
:10F2100090E0A0E0B0E08093AD339093AE33A09344
:10F22000AF33B093B033D8012C90222009F416C22A
:10F23000822D90E00E94F5E3892B09F421C2380168
:10F24000BFEF6B1A7B0AF8018181803349F4828118
:10F25000883531F40E5F1F4FC12CD12C760114C2BA
:10F26000BE016F5F7F4FC3010E948DE06B017C0187
:10F2700009811A816016710609F006C203C28091E5
:10F280007B330E946357182F01C010E06091C9338F
:10F290007091CA338091CB339091CC330E9496D831
:10F2A000662359F060916F337091703380917133A0
:10F2B000909172330E943257182F6091CD33709124
:10F2C000CE338091CF339091D0330E9496D866236D
:10F2D00071F06091733370917433809175339091B4
:10F2E00076330E9496D8862F0E940E59182F60916F
:10F2F000D1337091D2338091D3339091D4330E9423
:10F3000096D8662371F0609177337091783380914D
:10F31000793390917A330E9496D8862F0E944D5966
:10F32000182F6091E7337091E8338091E933909121
:10F33000EA330E9496D8662359F060918D3370911C
:10F340008E3380918F33909190330E94DEB1182FCD
:10F350006091EB337091EC338091ED339091EE330B
:10F360000E9496D8662371F0609191337091923328
:10F3700080919333909194330E9496D8862F0E9467
:10F380008C59182F8091E233882329F0809188339B
:10F390000E94CB57182F8091E333882329F0809166
:10F3A00089330E94FF57182F8091E633882329F074
:10F3B00080918C330E94AAB1182F8091E433882366
:10F3C00029F080918A330E943458182F8091E533B8
:10F3D000882329F080918B330E946858182F8091E0
:10F3E000D633882329F080917C330E94E358182F6C
:10F3F0008091D733882329F080917D330E94225950
:10F40000182F8091EF33882329F0809195330E9443
:10F410006159182F8091D833882329F080917E3349
:10F420000E94DB58182F809150338D3029F0809145
:10F43000DA338823A9F00FC0609196337091973327
:10F4400080919833909199330E946B578093A13D9E
:10F45000882369F32DC1809180330E942053182F97
:10F460008091DB33882329F0809181330E942453DB
:10F47000182F8091DC33882329F0809182330E94F9
:10F480008A53182F8091DF33882329F080918533A8
:10F490000E946757182F8091E033882329F08091CC
:10F4A00086330E942853182F4091503350E04F303C
:10F4B000510508F0B4C0FA01E057FE4F0C946DE01E
:10F4C0000E94B456182FABC061EB73E387E593E35A
:10F4D0000E94BF56182FA3C00E94F356182F9FC03A
:10F4E00061EB73E387E593E30E94FE56182F97C004
:10F4F0000E94136F182F93C061EB73E387E593E3CA
:10F500000E945154182F8BC00E945C6F182F87C027
:10F5100061EB73E387E593E30E949473182F7FC038
:10F52000609196337091973380919833909199338D
:10F530000E9496D8862F41EB53E367E573E30E9460
:10F540002C53182F6CC061EB73E387E593E30E94A3
:10F55000FB54182F64C00E94AE55182F60C00E9443
:10F560001556182F5CC00E944C56182F58C0609139
:10F57000833383E892E30E948C4F8091513384302F
:10F5800038F48230D8F4882349F0813079F047C0CC
:10F59000843009F044C08093873241C061EB73E34B
:10F5A00087E593E30E948456182F39C061EB73E31B
:10F5B00087E593E30E947757182F31C0A090A633B8
:10F5C000B090A733C090A833D090A933E090A23375
:10F5D000F090A3330091A4331091A53320919E3372
:10F5E00030919F334091A0335091A1338F938091FC
:10F5F0009D338F9380919C338F9380919B338F9316
:10F6000080919A338F9361EB73E387E593E30E94D4
:10F610000B88182F0F900F900F900F900F9060E0B5
:10F6200083E892E30E948C4F8091AC33813061F487
:10F6300080915233811104C00E948D5A812F38C0AD
:10F640000E94BE5A812F34C0812F32C08BEC30C053
:10F6500083E02EC084E82CC083E82AC01092A13D2C
:10F660006091533370915433809155339091563358
:10F670000E94264F8091D533882309F406CEFFCD12
:10F6800085E616C086E614C0822D90E0FC01E154A8
:10F69000F109EA31F10500F7E156FE4F0C946DE0F7
:10F6A000D8018C9174C968018B2D78017B2C3EC9DF
:10F6B0002796CDBFDEBFDF91CF911F910F91FF90B5
:10F6C000EF90DF90CF90BF90AF909F908F907F9002
:10F6D0006F905F904F903F902F900895CF93DF935E
:10F6E000EC0167EC7CE30E94FB658093A13D8111F6
:10F6F00002C095E09F83DF91CF910895FC01878937
:10F70000908D0C94627483FF06C0E0912530F091D7
:10F71000263090E2958382FF06C0E0912730F09179
:10F72000283090E2958381FF06C0E0912930F09166
:10F730002A3090E2958380FF06C0E0912B30F09153
:10F740002C3080E28583089583FF06C0E091253048
:10F75000F091263090E2968382FF06C0E091273038
:10F76000F091283090E2968381FF06C0E091293025
:10F77000F0912A3090E2968380FF06C0E0912B3012
:10F78000F0912C3080E2868308958091A73A811110
:10F7900007C084E00E94837B81E08093A73A0895AC
:10F7A00084E00E94A47B1092A73A0895CF92DF9242
:10F7B000EF92FF920F931F93CF93DF93C12C26E01C
:10F7C000D22EC0921530D092163030EAE32E36E0B9
:10F7D000F32EE0921730F092183000E816E0009314
:10F7E000193010931A30C0E6D6E0C0931B30D09386
:10F7F0001C30C0921D30D0921E30C0931F30D09369
:10F8000020300093213010932230E0922330F09288
:10F8100024302DEC3CEC4CED50E40E9425DAC092F3
:10F820002530D0922630E0922730F09228301816FA
:10F830004CF4C0932930D0932A3000932B3010938E
:10F840002C3008C00093293010932A30C0932B30FD
:10F85000D0932C30DF91CF911F910F91FF90EF90BB
:10F86000DF90CF9008950E9406D660E070E080E0BF
:10F8700091E40E94D67B0C9425D681E08093B03A27
:10F88000089520E093E088ED08B618BE84BF9093F9
:10F8900080002091820021FDFCCF08BEFFCF809127
:10F8A000B03A81110E94417C83E008958091B13A81
:10F8B000882341F0F89461E089E790E00E9408D63F
:10F8C00082E0089583E00895CF93DF93CDB7DEB74C
:10F8D000AD97CDBFDEBF21E2ECEEF1E2DE01119685
:10F8E00001900D922A95E1F722E02093CA01DE01F2
:10F8F0009296E8E0F0E024912D933196EE30F105F8
:10F90000D1F72DE228A7E0E1F0E0E491EF7121E0EA
:10F9100030E02C0F3D1F2E0F311DF901208129A74A
:10F92000E2E1F0E0E491EF719E012E0F311DF9014B
:10F9300021812AA7E4E1F0E0E491EF719E012E0F0E
:10F94000311DF90121812BA71CA61092CA0125E0C7
:10F95000FC012783BE016E5D7F4F0E94FB65809393
:10F96000A13DAD96CDBFDEBFDF91CF91089581E07F
:10F970008093B13A80E00895CF93DF93EC0120E0CB
:10F9800030E040E051E469857A858B859C850E9452
:10F9900025DA18166CF0CE010E94256369857A85F8
:10F9A0008B859C850E94D67B0E94B7BF80E001C0FA
:10F9B0008DE6DF91CF9108956BEE7BE30C944AC501
:10F9C0006DEC7BE30C944AC56EEA7BE30C944AC56C
:10F9D00060E97BE30C944AC56CE77BE30C94F5C4C7
:10F9E000CF93DF9381E397E49F938F93C7E3DAE5A7
:10F9F00089818F9388818F930E94FCE48BEF94E43C
:10FA00009F938F9389818F9388818F930E94FCE4C9
:10FA100083E794E49F938F9389818F9388818F9359
:10FA20000E94FCE489EA93E49F938F9389818F93EA
:10FA300088818F930E94FCE40E94A4AB8DB79EB78F
:10FA400040968DBF9EBF80E0DF91CF910895CF9308
:10FA5000DF9384E893E49F938F93C7E3DAE589818A
:10FA60008F9388818F930E94FCE486E192E49F93B8
:10FA70008F9389818F9388818F930E94FCE48BE818
:10FA800090E49F938F9389818F9388818F930E94B5
:10FA9000FCE483E794E49F938F9389818F9388811B
:10FAA0008F930E94FCE489EA93E49F938F9389816A
:10FAB0008F9388818F930E94FCE48DB79EB7449604
:10FAC0008DBF9EBF80E0DF91CF910895CF93DF93EC
:10FAD0008AE690E49F938F93C7E3DAE589818F9359
:10FAE00088818F930E94FCE48CEE9CE39F938F931C
:10FAF00089818F9388818F930E94FCE489EA93E443
:10FB00009F938F9389818F9388818F930E94FCE4C8
:10FB10008DB79EB70C968DBF9EBF80E0DF91CF91D1
:10FB20000895CF93DF9384EC9CE39F938F93C7E377
:10FB3000DAE589818F9388818F930E94FCE483E5C5
:10FB40009CE39F938F9389818F9388818F930E94E9
:10FB5000FCE489EA93E49F938F9389818F93888152
:10FB60008F930E94FCE48DB79EB70C968DBF9EBF0D
:10FB700080E0DF91CF910895CF93DF9380E39CE302
:10FB80009F938F93C7E3DAE589818F9388818F9361
:10FB90000E94FCE487E09CE39F938F9389818F937D
:10FBA00088818F930E94FCE489EA93E49F938F936A
:10FBB00089818F9388818F930E94FCE48DB79EB7D3
:10FBC0000C968DBF9EBF80E0DF91CF9108952F925C
:10FBD0003F924F925F926F927F928F929F92AF92DD
:10FBE000BF92CF92DF92EF92FF920F931F93CF932A
:10FBF000DF93CDB7DEB76A97CDBFDEBF5C010E9451
:10FC00003B652C011F86188A198A1A8AF501019012
:10FC10000020E9F73197EA19FB09E130F24008F0DA
:10FC200002C2D5018C91882359F17501BFEFEB1AFF
:10FC3000FB0A850120E0211115C0883229F08132AC
:10FC4000C8F08F37B9F001C021E06801EFEFCE1A9C
:10FC5000DE0A90E02A8F0E9406E4D8018C93860188
:10FC60002A8D08C021E0893209F420E0F801808360
:10FC70000F5F1F4FD7018D917D018111DCCF01C036
:10FC80008501F80110821092A13DFDE19F2EAAE3AB
:10FC90006A2EA2E27A2E812CB6E02B2E03C09A9413
:10FCA00009F49CC18BE79CE2A2E2B0E08B879C87C1
:10FCB000AD87BE876B8A7C8A8D8A8DE79CE2A2E243
:10FCC000B0E08F839887A987BA87EDE0F2E2DE0182
:10FCD0001196822D01900D928A95E1F7C2010E9442
:10FCE00042648501075F1F4F75019FEFA91AB90A8A
:10FCF000D7016C9170E0CE010B960E9463E4892BD2
:10FD000021F487010E5D1F4F04C0A016B10661F7F4
:10FD100093C16501BFEFAB1ABB0AF601608170E0C9
:10FD2000CE0143960E9463E4892B91F0D6011D9287
:10FD30008D0192012F5E3F4F288F398F46E050E0B2
:10FD4000B701C9010E948EE43AE0C30ED11C04C081
:10FD5000A016B106F1F670C15801D8013D908D0191
:10FD6000E32CF12CC7010E94EAE3892B59F4B70177
:10FD7000CE0101960E9463E4892B21F40C151D0528
:10FD800059F75AC18501BEE63B1641F0E2E23E1248
:10FD90000CC0D50111968C918232A9F5F20117821F
:10FDA0001186128613861486A3C0B0E3EB1AF108FD
:10FDB000EAE0EE16F10418F0FDE23F1217C0BE01B2
:10FDC0006A5E7F4FC5010E948DE0D20119966D9346
:10FDD0007D938D939C931C978E899F898A159B0593
:10FDE00009F42DC1E4E01796EC9382C0FBE73F12C3
:10FDF0004FC0E7E0D2011796EC93FFEFAF1ABF0AAE
:10FE0000E2E0FE2E95C02FEFA21AB20AE5E0D20181
:10FE10001796EC9362E270E0C5010E9463E48E8B5A
:10FE20009F8B009709F408C1DC011C92F501019039
:10FE30000020E9F73197EA19FB093397C8F0F80178
:10FE400081818033A9F48281883791F440E050E0C9
:10FE500060E070E0C5010E94FEE1D20119966D9349
:10FE60007D938D939C931C9783E017968C9308C089
:10FE7000B501C2010E94FB658093A13D811153C071
:10FE8000AE88BF88BFEFAB1ABB0AAE8ABF8A30C04C
:10FE9000E4E73E120EC0E1E0D2011796EC9380E059
:10FEA00090E0A0E8BFE3F20181879287A387B4873F
:10FEB0001FC0F6E63F120CC0E1E0D2011796EC93AA
:10FEC000179719961D921D921D921C921C9710C097
:10FED000BBE53B12B1C0F2012782B501C2010E940D
:10FEE000FB658093A13D81111EC077E6F72E7DC092
:10FEF000BE01695F7F4FC5010E94A8E45C010097C5
:10FF000009F49AC0DC018C918D3729F411968C91FB
:10FF1000F50131965F018C3209F48BC0FFEFAF1A07
:10FF2000BF0AF12C05C0F82E22E0281708F45DC0A6
:10FF30008F858201035F1F4F882341F043E050E02B
:10FF4000BE01615F7F4FC8010E948EE4688D798D8C
:10FF5000C8010E949C63D20114968D939C931597BF
:10FF60008F3FBFEF9B07B9F10E94EA68882371F0C9
:10FF7000888D998D0E948563882341F043E050E08D
:10FF8000688D798DCE010F960E948EE4F201428039
:10FF900053804114510411F1F11081CE80913E350E
:10FFA000811108C087E395E30E9460608093A13DC2
:10FFB000F82E1BC080915332823099F087E395E38D
:10FFC0000E9436608093A13D81110EC087E395E3C6
:10FFD0000E94B3600AC064E6F62E07C050E7F52E13
:10FFE00004C04BECF42E01C0F82E42E060E08F2DEF
:10FFF0000E94A26681E00E9464AD6A96CDBFDEBF1A
:020000021000EC
:10000000DF91CF911F910F91FF90EF90DF90CF90F4
:10001000BF90AF909F908F907F906F905F904F9028
:100020003F902F9008958BE68093A13D3BE6F32E01
:10003000DCCF22E0F22E7CCF9FE6F92ED6CF86E6EB
:10004000F82ED3CF2F923F924F925F926F927F9272
:100050008F929F92AF92BF92CF92DF92EF92FF92D8
:100060000F931F93CF93DF9300D000D0CDB7DEB7AF
:100070008C0169837A834B835C835A0128E0A21A3E
:10008000B108A60EB71EDC0116967C907B01BFEF6F
:10009000EB1AFB0A8BE7FB01808380E0912C95E053
:1000A000692E27E1422E22E2522E33E1232E32E244
:1000B000332E4DE7842EED82FE82D80117969C9157
:1000C0009F3F09F429C1882339F02CE2ED81FE819C
:1000D00020833196ED83FE8380914B3D811119C0C1
:1000E000C80141969F938F933F922F923E813F93F9
:1000F0008D818F930E94C7E5AD81BE81A80FB91F86
:10010000AD83BE830F900F900F900F900F900F90C4
:1001100018C0C80141969F938F935F924F92BE8102
:10012000BF93ED81EF930E94C7E52D813E81280F9B
:10013000391F2D833E830F900F900F900F900F90DB
:100140000F90D80117968C911797843059F519960E
:10015000CD90DD90ED90FC901C97A7019601C70112
:10016000B6010E94E8DB811117C0E894F7F82FEF81
:100170003FEF4FE75FE7C701B6010E94E8DB81115F
:1001800021C12FEF3FEF4FE75FE7C701B6010E94A4
:1001900022D818160CF016C1F801118612861386A3
:1001A000148610C1811113C0EDE1F2E2AD81BE8170
:1001B000862D01900D928A95E1F72D813E812C5F6D
:1001C0003F4F2D833E83D80117968C9199C0823082
:1001D00061F4F80184858F9383858F9382858F9353
:1001E00081858F93A2E2B2E214C0833029F5D80151
:1001F0001C968C911C978F931B968C911B978F93B9
:100200001A968C911A978F9319968C918F93A8E2D6
:10021000B2E2BF93AF93FE81FF932D812F930E9493
:10022000C7E5AD81BE81A80FB11DAD83BE83F801C6
:100230008781CDBFDEBF64C0853059F4D8015896A0
:100240008C9158978F9357968C918F93A0E3B2E23D
:100250000CC0863009F5D80158968C9158978F9329
:1002600057968C918F93A5E3B2E2BF93AF93FE8133
:10027000FF932D812F930E94C7E5AD81BE81A80F0A
:10028000B11DAD83BE83F80187810F900F900F9051
:100290000F900F900F9034C0813091F52CEA35EC1F
:1002A00047E257E3D80119966D917D918D919C910C
:1002B0001C970E9422D887FF12C0EAE3F2E2AD81C8
:1002C000BE8186E001900D928A95E1F7ED81FE8175
:1002D0003596ED83FE83D80117968C9111C0E0E42A
:1002E000F2E2AD81BE81862D01900D928A95E1F7F3
:1002F000ED81FE813496ED83FE83D80117968C91B3
:10030000873049F42BE7ED81FE8120833196ED8320
:10031000FE8380E001C081E0AD81BE81AA15BB05EE
:1003200018F08FEF9FEF65C0F8010281138101156E
:10033000110549F0D80116969C912FEF290D9915BA
:100340003CF0992EBACEED80FE807914B4F020C036
:10035000ED81FE81D801CF010196808216969C9096
:1003600016973FEF320F92161CF4232FFC01F3CFA8
:100370008D839E838D0181E0A0CEF7012DE7CF0113
:10038000019620839A94791414F4FC01F8CF7C012F
:100390008DE79AE0A0E0F70180839183A283F2E0E9
:1003A000EF0EF11C89819A812B813C81820F931F72
:1003B0008E159F0508F4B5CFC701A981BA818A1BA4
:1003C0009B0B17C0C8010E94FA68F801418552854D
:1003D0006385748520858D819E810E948EC72D81C5
:1003E0003E81280F311D2D833E83D80117968C91B5
:1003F00087CF2696CDBFDEBFDF91CF911F910F91A2
:10040000FF90EF90DF90CF90BF90AF909F908F9034
:100410007F906F905F904F903F902F90089540E0B5
:1004200052E067EC7AE30E9422806091375A709123
:10043000385A87EC9AE30C944BE5EF92FF920F93B6
:100440001F93CF93DF93CDB7DEB76297CDBFDEBFEB
:10045000F82E9091493D992309F4B2C08FE6F81225
:1004600012C00E943B6567EC7CE38091C33A909197
:10047000C43A0E946EC7BC0186E091E20E945966B0
:1004800007E315E34AC08091533207E315E388235D
:1004900009F443C0EE24EA94C8010E940264882350
:1004A000E1F1823029F48091503D811120C01DC0BE
:1004B000843029F480914D3D811119C016C08530DA
:1004C000B1F480914F3D882381F0F80181859285B8
:1004D000A385B485BC01CD019F772CEA35EC47E2BA
:1004E00057E30E9422D887FF02C0F801E782F80193
:1004F000028113810115110579F60FC0F8010281FF
:1005000013810115110549F440E052E067EC7AE3EC
:100510008EE195E30E94228053C0F80197819F3FAE
:1005200069F78091BD2981111AC08091C63A8F93D5
:100530008091C53A8F931F92FF9285E492E29F9338
:100540008F93CE0101967C01FF928F930E94C7E5A5
:100550001092C53A1092C63ACDBFDEBF13C00E94BA
:10056000EECB1F928F931F92FF928DE492E29F93A6
:100570008F93CE0101967C01FF928F930E94C7E575
:10058000CDBFDEBFB701C8010E94FB65F80116822E
:1005900086E0878386E690E0818B928B12821382BD
:1005A00040E052E067EC7AE38EE195E30E9422801E
:1005B0006091375A7091385A87EC9AE30E944BE564
:1005C0006296CDBFDEBFDF91CF911F910F91FF905B
:1005D000EF900895613019F0623029F0089587E3B3
:1005E00095E30C940F820C941D82CF92DF92EF92D0
:1005F000FF92FC01C184D284E384F48420E030E0E3
:1006000040EA50E4C701B6010E9425DA18160CF43E
:1006100053C0C701B6010E9496D86093493D10921D
:100620004C3D10924D3D10924E3D10924F3D109218
:10063000503D20E030E040E85FE3C701B6010E9492
:1006400025DA87FD03C081E080934C3D20E030E057
:1006500040E050E4C701B6010E9425DA87FD03C0DF
:1006600081E080934D3D20E030E040E450E4C7015C
:10067000B6010E9425DA87FD03C081E080934E3DDC
:1006800020E030E040E850E4C701B6010E9425DADE
:1006900087FD03C081E080934F3D20E030E040EAD9
:1006A00050E4C701B6010E9425DA87FD07C081E04A
:1006B0008093503D80E003C08EE601C080E0FF9053
:1006C000EF90DF90CF90089563ED77E40C940BC525
:1006D0006CE777E40C940BC568E477E40C940BC5E5
:1006E000BF92CF92DF92EF92FF920F931F93CF931F
:1006F000DF93CDB7DEB76897CDBFDEBF6B0128E1D2
:10070000FC01DE01119601900D922A95E1F784E13A
:10071000E82E81E3F82E8E010F5F1F4FB12CF701F9
:100720008081823029F4F8011082118212821382B2
:100730008091B9588B1114C02091CC583091CD586C
:100740004091CE585091CF58F801608171818281DB
:1007500093810E94C7DAF601608371838283938359
:100760008091D8588B1114C02091EB583091EC58DF
:100770004091ED585091EE58F8016081718182816D
:1007800093810E94C7DAF601648375838683978319
:100790008091F7588B1114C020910A5930910B5950
:1007A00040910C5950910D59F801608171818281FD
:1007B00093810E94C7DAF6016087718782879387E9
:1007C000809116598B1114C02091295930912A59C2
:1007D00040912B5950912C59F8016081718182818F
:1007E00093810E94C7DAF6016487758786879787A9
:1007F000B394F5E3EF0EF11C0C5F1F4F86E0B812C7
:100800008ECF6896CDBFDEBFDF91CF911F910F9144
:10081000FF90EF90DF90CF90BF900895F8940E94E2
:10082000337C0E9465840E9425D60E946AC90E947A
:1008300009B60E941D740E94B7BF0E942BA940E018
:1008400060E080E00E94E0690E9478650E94538425
:100850000E9457860E94C0530E941DD68091A2001C
:1008600084608093A2008091A20082608093A200A5
:100870008091A20081608093A20078940E94A4AB32
:100880000E94CCC00E94476AFDCFE82FF0E0EE0F37
:10089000FF1FE150F84B659174914FE450E081E502
:1008A0009DE30C9435E48091A53A823041F440E018
:1008B00060E081E00E94E06980E00E945C6B0C9443
:1008C000ECCC682F81E00C945DCA1092A23D10928E
:1008D000A33D1092A43D1092A53D0895CF93DF93C0
:1008E000EC018C819D81880F991F880F991F2091A1
:1008F000A43D3091A53D820F931F8093A63D909318
:10090000A73D44E050E06CEA7DE30E941DD5409194
:10091000AC3D5091AD3D6091AE3D7091AF3D49878A
:100920005A876B877C8780E0DF91CF9108958F9203
:100930009F92AF92BF92CF92DF92EF92FF92CF93AE
:10094000DF93EC0180915432882369F089E0DF91D4
:10095000CF91FF90EF90DF90CF90BF90AF909F909E
:100960008F900C942CAB89859A85AB85BC85809340
:10097000A83D9093A93DA093AA3DB093AB3DCE0175
:100980000E946E848093A13D81116EC0C984DA8477
:10099000EB84FC84A7019601C701B6010E94E8DB45
:1009A00081112FC046015701E894B7F82FEF3FEFB0
:1009B0004FE75FE7C501B4010E94E8DB81110AC07F
:1009C0002FEF3FEF4FE75FE7C501B4010E9422D848
:1009D0001816BCF08090A83D9090A93DA090AA3D2B
:1009E000B090AB3DA5019401C701B6010E94B3D6FA
:1009F0009F772CEA35EC47E257E30E9425DA181678
:100A000074F58091A83D9091A93DA091AA3DB09127
:100A1000AB3D8093AC3D9093AD3DA093AE3DB09384
:100A2000AF3D8C819D81880F991F880F991F209160
:100A3000A43D3091A53D820F931F8093A63D9093D6
:100A4000A73D44E050E06CEA7DE30E94AED5809083
:100A5000A83D9090A93DA090AA3DB090AB3D89865D
:100A60009A86AB86BC8680E0DF91CF91FF90EF90B5
:100A7000DF90CF90BF90AF909F908F9008950E948D
:100A800029BB80E008958091B03D9091B13D8F3EAB
:100A9000924111F08EE508958091D63D9091D73D19
:100AA0008F3E9241B9F78091D83D9091D93D8F3ECC
:100AB000924181F780914155909142558F3E9241EC
:100AC00049F780914355909144558F3E924111F7DB
:100AD0008091D5569091D6568F3E9241D9F680E0BE
:100AE000089594E0899FF0011124E055F24C42836F
:100AF000538364837583089594E0899FF0011124E2
:100B0000ED5BFA4A45AB56AB67AB70AF08955F92A9
:100B10006F927F928F929F92AF92BF92CF92DF920D
:100B2000EF92FF920F931F93CF93DF93CDB7DEB772
:100B30006097CDBFDEBFBE016F5F7F4F88E795E551
:100B40000E947083CE0101964C0180EFA82E85E5AE
:100B5000B82E90E0C92E96E5D92E20E1E22E26E5AA
:100B6000F22E00E316E530E5632E39E5732E512CA5
:100B7000F40141915191619171914F01F5014193BE
:100B80005193619371935F01F60141935193619386
:100B900071936F01F70141935193619371937F01B9
:100BA000852D0E943F74F8011192119211921192B9
:100BB0008F01F30110821182128213825394F8E1A3
:100BC0006F0E711C84E05812D3CF6096CDBFDEBF8C
:100BD000DF91CF911F910F91FF90EF90DF90CF9019
:100BE000BF90AF909F908F907F906F905F9008958F
:100BF0008091DA3D08951F93CF93DF938BE697E1C1
:100C0000E8EDFDE3DF019C011D9221503040E1F74A
:100C10008FEE92E18093D83D9093D93D80934155DA
:100C200090934255C1EEDDE3C093DB3DD093DC3DB4
:100C3000C093DD3DD093DE3DC093DF3DD093E03DDA
:100C400081E090E066E874E520E030E01BEB129F65
:100C5000A001139F500D1124FA01E852F24CD90162
:100C600011961A9F90011B9F300D11242F51324C69
:100C70002387348761877287BA016F51724C9C0158
:100C800001968032910519F78BEB829FF001839FCB
:100C9000F00D1124E852F24CC387D4876187728724
:100CA00080E28093DA3DDF91CF911F910895CF9339
:100CB000DF93E3E4F5E584E991E0DF01EC011D92C7
:100CC0002197E9F7A0EBBDE388E2ED0119928A953F
:100CD000E9F78FEE92E18D939C938093D63D9093AC
:100CE000D73D808391838093D5569093D656DF91DC
:100CF000CF910C94FB850E9452900E94FB8580E06E
:100D00000C94DB4EE091DB3DF091DC3D848581115C
:100D10001BC022813381808191814BEBDF011D92C9
:100D20004A95E9F7228333838083918381E0848726
:100D30008091DA3D81508093DA3D82819381809366
:100D4000DB3D9093DC3D05C08CE10E942CABE0E0E4
:100D5000F0E0CF010895ADEDBDE3ED91FC91119769
:100D6000858781E0878782E08487828193818D9364
:100D70009C9381E00E94B5AE0C946FB8EF92FF9205
:100D80000F931F93CF93DF9300D01F92CDB7DEB7A1
:100D90008C014B835C8369837A830E948286FC0189
:100DA0004B815C8169817A81009761F48EE02496A1
:100DB000CDBFDEBFDF91CF911F910F91FF90EF90DC
:100DC0000C94105383E085878FE395E884839583A3
:100DD000068317838B017A0126E0D8014D915D913E
:100DE0006D917D918D01CF0185599F4FDC014D9310
:100DF0005D936D937C931397D7014D915D916D91A8
:100E00007D917D01418B528B638B748B2150349685
:100E10002111E3CF83E02496CDBFDEBFDF91CF91D8
:100E20001F910F91FF90EF900C94AB86CF92DF92C1
:100E3000EF92FF926B017C010E948286009739F449
:100E40008EE0FF90EF90DF90CF900C94105329E943
:100E500037E8FC0124833583E556FF4FC082D182F9
:100E6000E282F38221E0FC01278782E00E94AB86C8
:100E700080E0FF90EF90DF90CF9008958091DF3D6C
:100E80009091E03DFC0124853EEF320F323018F4A2
:100E900024E024870895243011F080E090E0089544
:100EA000E091DF3DF091E03D2281338180819181AD
:100EB0004BEBDF011D924A95E9F722833383808350
:100EC0009183E091DF3DF091E03D0280F381E02DE0
:100ED000E093DF3DF093E03D8485823011F483E0C0
:100EE00084878091DA3D8F5F8093DA3D8FEF0E9497
:100EF000B5AE81E04091DB3D5091DC3D2091DF3D7E
:100F00003091E03D4217530709F080E00895BC019D
:100F10006F5E7F4FDC011696ED91FC911797855916
:100F20009F4F19950E94508781110E945A5A80E064
:100F3000089585569F4F20E034E244E759E4FC01D0
:100F400060817181828193810E94C7DA0E9496D864
:100F50000E94C2D80E9433BB0E94508781110E9418
:100F60005A5A80E008958091DF3D9091E03DFC0168
:100F700024853EEF320F323018F424E024870895A0
:100F8000243011F080E090E00895CF93DF93C0917A
:100F9000DF3DD091E03D8C859EEF980F923018F4A4
:100FA00084E08C8705C0843019F080E090E010C0A8
:100FB0002097D9F3DE011296ED91FC911397878566
:100FC000882329F0EC17FD0711F0DF01F4CFCD01E4
:100FD000DF91CF910895CF93DF93EC012A813B817C
:100FE000888199814BEBFB01DE0101900D924A95BE
:100FF000E1F72A833B8388839983DF91CF9108951A
:101000008FEE92E18093D7569093D8568093935762
:101010009093945708952F923F924F925F926F92C0
:101020007F928F929F92AF92BF92CF92DF92EF9278
:10103000FF920F931F93CF93DF93CDB7DEB76B97DC
:10104000CDBFDEBF4C011B0129013A01EB86FC86B6
:101050000D871E871A2D0B2DE9A8BAA8ABA82CA9BD
:1010600029838091CC32882399F08091C03290916D
:10107000C132A091C232B091C332BC01CD019F7781
:101080002CEA35EC47E257E30E9422D887FDEFC6F1
:101090008091F4339091F533A091F633B091F7330A
:1010A000BC01CD019F7731E039872CEA35EC47E26E
:1010B00057E30E9425DA181614F0198610C02DEC9B
:1010C0003CEC4CEC5DE360919A3370919B338091E2
:1010D0009C3390919D330E9422D887FDCAC6F101AE
:1010E00080819181A281B381BC01CD019F77F1E024
:1010F000FD832CEA35EC47E257E30E9425DA181607
:101100000CF01D82F10184819581A681B781BC011B
:10111000CD019F77F1E0FF872CEA35EC47E257E3FA
:101120000E9425DA18160CF01F86F1018085918542
:10113000A285B3852091F8333091F9334091FA3389
:101140005091FB332F8B388F498F5A8F2091FC336E
:101150003091FD334091FE335091FF332B8B3C8B0C
:101160004D8B5E8B4091003450910134609102347C
:1011700070910334F090CD32F11021C010922357BA
:1011800081E08093245782E080932557398533236B
:1011900041F04D81411171C65F8551116EC68CE9D8
:1011A0009FC6CB01BA019F772CEA35EC47E257E3A3
:1011B0000E9425DA18160CF065C68BE991C6BC01B1
:1011C000CD019F77A1E0AB8F2CEA35EC47E257E3E6
:1011D0000E9425DA18160CF01B8EB1E0FB1216C027
:1011E0001092235782E080932457F0922557E98587
:1011F000EE2339F0FD81F11140C62B8D222379F2C7
:101200003CC66B897C898D899E89CDCF32E0F312F3
:1012100017C081E080932357F092245710922557EE
:101220004985442341F05F85511127C68B8D882362
:1012300009F4B5CF22C66F89788D898D9A8DB3CF89
:10124000B101C4010E942A519985992309F451C022
:10125000209188323091893240918A3250918B327C
:101260006091DC327091DD328091DE329091DF321C
:101270000E94B3D69F772CEA35EC47E257E30E94F1
:1012800022D887FF36C020918C3230918D32409128
:101290008E3250918F326091E0327091E1328091C4
:1012A000E2329091E3320E94B3D69F772CEA35EC7C
:1012B00047E257E30E9422D887FF1BC0209190325B
:1012C0003091913240919232509193326091E43258
:1012D0007091E5328091E6329091E7320E94B3D668
:1012E0009F772CEA35EC47E257E30E9422D887FD2E
:1012F000C2C58DA98093873283E892E30E94324F62
:1013000085E5E3E8F2E3AEE3B7E501900D928A9557
:10131000E1F788E1ECEDF2E3AAEDB6E501900D927C
:101320008A95E1F78091CE328111B1C523E333E391
:101330004BEC51E46E2D7B2D8A2D99810E94C7DAEA
:101340004B015C0160930E5770930F5780931057B9
:101350009093115723E333E34BEC51E4C301B20103
:101360000E94C7DA6093F2567093F3568093F45656
:101370009093F55623E333E34BEC51E46B857C8586
:101380008D859E850E94C7DA6093F6567093F75656
:101390008093F8569093F95623E333E34BEC51E4F2
:1013A000612F702FC6010E94C7DA162F072F412F19
:1013B000502FBC014093FA565093FB566093FC5655
:1013C0007093FD568091963390919733A091983306
:1013D000B0919933BC01CD019F770E94FFD80E9444
:1013E00096D82B013C0160931F5770932057809330
:1013F0002157909322571091235780912457A82F5B
:10140000B0E0AB87BC877D01EE0CFF1CEE0CFF1C2F
:10141000F101EE0DFF1D80819181A281B381BC019C
:10142000CD019F772CEA35EC47E257E30E9422D8A2
:10143000881F8827881F8983E12FF0E0E987FA87D2
:101440008F01000F111F000F111FF101E00FF11F9D
:1014500080819181A281B381BC01CD019F772CEA6B
:1014600035EC47E257E30E9422D8881F8827881F5F
:10147000F981F823F983F0931E572CEA35EC47E203
:1014800057E3C501B4019F770E9425DA181624F0AE
:101490000D831E83870105C1E985FA85EE0FFF1FC5
:1014A000EE0FFF1FE857FD4CA985BA85AA0FBB1F99
:1014B000AA0FBB1FA452BD4C2D913D914D915C9143
:1014C00060817181828193810E94B3D66F87788B0E
:1014D000898B9A8BEB85FC85EE0FFF1FEE0FFF1FAC
:1014E000E857FD4CAB85BC85AA0FBB1FAA0FBB1FDD
:1014F000A452BD4C2D913D914D915C9160817181C3
:10150000828193810E94B3D66B8B7C8B8D8B9E8B5B
:10151000A5019401C501B4010E94C7DA20E030E0C2
:1015200040E850E40E94C7DA6D837E838F839887FA
:101530002F85388949895A89CA01B9010E94C7DAB9
:101540006B017C012B893C894D895E89CA01B901F7
:101550000E94C7DA9B01AC01C701B6010E94B4D654
:101560009B01AC016D817E818F8198850E94B3D6ED
:101570006B017C0120E030E0A9010E9425DA1816F9
:10158000D4F4C701B6010E94A0DB6B017C012B895A
:101590003C894D895E896F85788989899A890E94FD
:1015A00032DA9B01AC01C701B60190580E9429D8DC
:1015B0006B017C0103C0C12CD12C76018091873254
:1015C000833021F4F7FAF094F7F8F09420E030E05B
:1015D000A901C501B4010E9422D887FF04C0F7FA0F
:1015E000F094F7F8F09429853A85220F331F220FE3
:1015F000331F2D833E8389010952194AA7019601A1
:101600006B897C898D899E890E94C7DA9B01AC0118
:101610006F85788989899A890E94B3D620E030E065
:1016200040E05FE30E94C7DAD8015B966D937D933B
:101630008D939C935E970B851C85000F111F000FE7
:10164000111FF801E952F94A5F01A70196016F8560
:10165000788989899A890E94C7DA9B01AC016B89D4
:101660007C898D899E890E94B4D620E030E040E0DC
:101670005FE30E94C7DAD5015B966D937D938D93EE
:101680009C935E97E0912557F0E0EE0FFF1FEE0F61
:10169000FF1FE952F94A138E148E158E168E109282
:1016A000A13DF801E952F94AC38CD48CE58CF68C43
:1016B000F7FAF094F7F8F094ED81FE81E952F94AD7
:1016C000838D948DA58DB68DBC01CD019058A70159
:1016D00096015F770E9429D80E9418D74B015C01C0
:1016E00020E030E0A901C701B6010E9425DA1816F2
:1016F000C4F020E030E0A901B401C5010E9425DA60
:101700009401A50118162CF46BED7FE089E490E4B8
:1017100004C06BED7FE089E490EC0E94B3D64B01EE
:101720005C01C401D5018093065790930757A0939D
:101730000857B09309579401A501B401C5010E944F
:10174000E8DB8111C8C3B981BB23B1F1C301B20188
:101750000E94C2D86B017C012CEA35EC47E257E3CA
:101760000E9422D887FD11C0B09087322BED3FE058
:1017700049EC50E4C701B6010E94C7DA9B01AC01F5
:10178000C12CD12CE12CF12CEFC081E090E0A0E045
:10179000B0E080931F5790932057A0932157B093A8
:1017A0002257B09087322BED3FE049EC50E4C12C3A
:1017B000D12CE12CF12CD8C0EB85FC85EE0FFF1F5E
:1017C000EE0FFF1FED5BF84A98012952394A790163
:1017D000D9015B962D913D914D915C915E97608111
:1017E0007181828193810E94B3D6F7012381348174
:1017F000458156810E94B3D66B017C01E985FA854B
:10180000EE0FFF1FEE0FFF1FED5BF84A2D813E81AB
:101810002952394A1901D9015B962D913D914D917B
:101820005C915E9760817181828193810E94B3D6C1
:10183000F10123813481458156810E94B3D6A701ED
:1018400096015F770E9429D80E9418D71B018983CF
:101850009F8720E030E0A901C701B6010E9425DA88
:101860001816E4F020E030E0A901B10189819F85DC
:101870000E9425DA910149815F8518162CF46BEDE1
:101880007FE089E490E404C06BED7FE089E490ECB4
:101890000E94B3D61B01F82EE92E02C0F980EF8416
:1018A000C101AF2DBE2D80930A5790930B57A09383
:1018B0000C57B0930D5791014F2D5E2DB1018F2D17
:1018C0009E2D0E94E8DB811106C391014F2D5E2DF4
:1018D000B401C5010E9425DA1816B4F42BED3FE0DF
:1018E00049EC50E4B1018F2D9E2D0E94B4D61B010E
:1018F000AB01BC0140930A5750930B5760930C57B0
:1019000070930D57F82EE92E9401A501B1018F2D8A
:101910009E2D0E94B3D66B017C01B0908732F3E01C
:10192000BF1669F0C301B2010E94C2D82BED3FE09F
:1019300049EC50E40E94C7DA9B01AC0115C02BEDC5
:101940003FE049EC50E40E94B3D66B017C01C30137
:10195000B2010E94C2D82BED3FE049EC50E40E9456
:10196000C7DA9B01AC0108C082E0B81205C0B6011D
:10197000C7010E94B4D604C0B601C7010E94B3D605
:101980006B01AB01BC014093125750931357609306
:101990001457709315577C01F801E952F94A238DC9
:1019A000348D458D568DED81FE81E952F94A638D66
:1019B000748D858D968D0E9432DA2B013C016093E7
:1019C0000E5770930F5780931057909311571091A3
:1019D0002557A12FB0E0FD01EE0FFF1FEE0FFF1FF7
:1019E000ED5BF84AAA0FBB1FAA0FBB1FA952B94A49
:1019F00013962D913D914D915C9116976081718167
:101A0000828193810E94B3D64B015C01609316578B
:101A10007093175780931857909319579601A70101
:101A2000C301B2010E94C7DA6B017C0160931A57AF
:101A300070931B5780931C5790931D57A5019401D9
:101A40000E9432DA69837A838B839C836093FE568B
:101A50007093FF56809300579093015720915F3009
:101A60003091603040916130509162302D833E83DF
:101A70004F8358870E9422D887FD2FC28091CC3295
:101A8000811118C03091C0323B8F4091C1324F87D5
:101A90005091C2325B8B8091C3328F8B1092C032D7
:101AA0001092C1321092C2321092C33281E0809300
:101AB000CC3212C02091C0323091C1324091C2323A
:101AC0005091C33269817A818B819C810E9429D88F
:101AD0006B8F7F878B8B9F8B85E3A985BA858A9FC8
:101AE000F0018B9FF00D1124EB5EFE4C20813181C3
:101AF00042815381C701B6010E9429D86987072F07
:101B0000382E292E2B8D3F854B895F89832D922D71
:101B10000E9422D887FF03C0BB8DB98703C00F87FF
:101B20003B8A2F8A85E32B853C85829FF001839F2A
:101B3000F00D1124EB5EFE4C2081318142815381F6
:101B4000C701B6010E9429D8F62E072F382E292E5C
:101B5000262F372F482F592F69857F858B899F899D
:101B60000E9425DA181624F40F853B882F8801C0BF
:101B7000F9868985902FA32DB22D809302579093DB
:101B80000357A0930457B093055720E030E0A90114
:101B9000C501B4019F770E9425DA18167CF535E35C
:101BA000139FF0011124EB5EFE4C208131814281B4
:101BB0005381C501B4010E9429D86B017C01E894CE
:101BC000F7F8A70196016985702F832D922D0E9449
:101BD00025DA181614F4198504C01C2D0D2D3E2C81
:101BE0002F2C812F902FA32DB22D809302579093ED
:101BF0000357A0930457B093055701C01985C090AF
:101C00005630D0905730E0905830F090593020E066
